:020000040800F2
:1000000000060020E1010008CD0D0008D10D000818
:10001000290E0008D10D0008FD0D0008E3010008BD
:10002000E3010008E3010008E30100083D210008A6
:10003000E3010008E3010008E3010008E301000810
:10004000E3010008E3010008E3010008E301000800
:10005000E3010008E30100081D32000849320008EE
:1000600075320008A1320008CD320008E301000813
:10007000E3010008E3010008E3010008E3010008D0
:10008000E3010008E3010008E3010008E3010008C0
:10009000E3010008E3010008E3010008F932000869
:1000A000E3010008E3010008E3010008E3010008A0
:1000B00091300008E3010008E3010008E3010008B3
:1000C000E3010008E3010008E3010008E301000880
:1000D000E3010008E3010008E3010008E301000870
:1000E00061330008E3010008E3010008E3010008B0
:1000F000E3010008E3010008E3010008E301000850
:10010000E3010008E3010008E3010008E30100083F
:10011000E3010008E3010008E3010008E30100082F
:10012000E3010008E3010008E3010008E30100081F
:10013000E3010008E3010008E3010008E30100080F
:10014000E3010008E3010008E3010008812800083A
:10015000E3010008E3010008E3010008E3010008EF
:10016000E3010008E3010008E3010008E3010008DF
:10017000E3010008E3010008E3010008E3010008CF
:10018000E3010008E3010008E3010008E3010008BF
:10019000E3010008E3010008E3010008E3010008AF
:1001A000E3010008E3010008E3010008E30100089F
:1001B000E3010008E3010008E3010008E30100088F
:1001C000E3010008E3010008E3010008E30100087F
:1001D000E3010008E3010008E3010008E30100086F
:1001E00002E000F000F8FEE772B6394880F30888B4
:1001F000384880F3098838484EF60851CEF200019D
:10020000086040F20000CCF200004EF63471CEF2ED
:1002100000010860BFF34F8FBFF36F8F40F2000003
:10022000C0F2F0004EF68851CEF200010860BFF334
:100230004F8FBFF36F8F4FF00000E1EE100A4EF6C4
:100240003C71CEF200010860062080F31488BFF3F1
:100250006F8F01F0D1FF02F077FE4FF055301F494C
:100260001B4A91423CBF41F8040BFAE71C49194A6A
:1002700091423CBF41F8040BFAE71A491A4A1B4B5A
:100280009A423EBF51F8040B42F8040BF8E70020F5
:100290001749184A91423CBF41F8040BFAE701F0B4
:1002A000AFFF02F0ADFE144C144DAC4203DA54F82B
:1002B000041B8847F9E700F041F8114C114DAC429E
:1002C00003DA54F8041B8847F9E701F097BF0000F0
:1002D000000600200022002000000008000000208E
:1002E0000006002090370008002200203C22002059
:1002F00040220020A42D0020E0010008E0010008B9
:10030000E0010008E00100082DE9F04F2DED108A12
:10031000C1F80CD0C3689D46BDEC108ABDE8F08FD3
:10032000002383F311882846A047002001F004FB36
:10033000FEE701F085FA00DFFEE7000038B501F0C6
:10034000CFFE044601F0F4FE0546D8B90F4B9C429F
:100350001AD001339C4218BF054641F2883404BFCD
:1003600001250024002001F0C5FE0DB100F058F871
:1003700000F000FD00F09EFB204600F0AFF800F01A
:100380004FF8F9E70024EDE70446EBE7010007B07A
:1003900008B500F061FBA0F120035842584108BDA8
:1003A00007B5054B02211B88ADF8043001A800F009
:1003B00071FB03B05DF804FB5C34000810B520232A
:1003C00083F311881248C3680BB101F051FB00237D
:1003D000104A0F484FF47A7101F0F8FA002383F3C2
:1003E00011880D4C236813B12368013B23606368B7
:1003F00013B16368013B6360084B1B7833B96368D2
:1004000023B9022000F02CFC3223636010BD00BF32
:1004100040220020BD0300085C230020542200205D
:1004200010B5254B254953F8042F013200D110BDDA
:100430008B42F8D1224C234B22689A423AD9224B64
:100440009B6803F1006303F540439A4232D20020D7
:1004500000F04AFB1D4B0220187000F0FFFB1C4B04
:100460001A6C00221A64196E1A66196E596C5A6455
:10047000596E5A665A6E5A6942F080025A615A6938
:1004800022F080025A615A691A6942F000521A61D8
:100490001A6922F000521A611B6972B60D4A0E4B9E
:1004A00013601B682268202181F311889D4683F325
:1004B0000888104710BD00BFFCBF00081CC0000822
:1004C00004C00008FFBF00080022002054220020C2
:1004D0000038024008ED00E000C000082DE9F04FB0
:1004E00099B0B94D00902022FF2110A8AC6800F00F
:1004F000E3FBB64A01951378A3B9B5480121C3605F
:100500001170202383F31188C3680BB101F0B0FA96
:100510000023B04AAE484FF47A7101F057FA002335
:1005200083F31188009BAC4A03B11360AB4B009D71
:10053000029300261E705660B2463746B14601202F
:1005400000F08CFB002D00F02582A34B1B68002BD4
:1005500040F0208219B0BDE8F08F0220FFF718FFAD
:10056000002840F01082009B002E08BF1D469C4BC7
:1005700002211B88ADF82C300BA800F08BFADEE7C7
:100580004FF47A7000F068FAB0F10008EBDB02205B
:10059000FFF7FEFE0028E6D008F1FF38B8F1040F9F
:1005A00000F2F381DFE808F0031E2124270018A8D9
:1005B000052340F8343D042100F06CFA012303FACE
:1005C00008F848EA0A0A5FFA8AFA4FF0000900F0D0
:1005D000C7FB27B10AF00B030B2B08BF0025FFF761
:1005E000DFFEACE704217848E6E704217D48E3E735
:1005F00004217D48E0E74FF01C09484600F076FAF8
:1006000009F104090B9004210BA800F043FAB9F199
:100610002C0FF2D1D2E7002FA5D00AF00B030B2B41
:10062000A1D10220FFF7B4FE804600289BD0012014
:100630006A4E00F059FA0220307000F00FFB0027DC
:100640005FFA87FB584600F05FFA054688B15846C6
:1006500000F06AFA01370028F2D146460025634BC4
:1006600002211B88ADF82C300BA800F013FA474686
:1006700065E701230220337000F0EEFA2C46019B5F
:100680009B689C4206D2204600F030FA0130E4D14B
:100690000434F4E7029B00241C704F4B46465C6018
:1006A0004746254693E7002F3FF45DAF0AF00B0362
:1006B0000B2B7FF458AF029B0220187000F0CEFA8B
:1006C000322000F0C9F9B0F1000BFFF64CAF1BF07F
:1006D00003087FF448AF019B996804EB0B028A4240
:1006E0003FF641AFBBF5807F3FF63DAF404A0392F6
:1006F000D8450FDA4FF47A7000F0AEF904900499FF
:100700000029FFF630AF039A049908F8021008F1A7
:100710000108ECE7C820FFF73BFE804600283FF4C5
:1007200022AF1F2C11D8C4F120075F4528BF5F46B8
:1007300010AB24F003003A462D49184400F092FA19
:100740003A46FF212A4800F0B7FA4FEAAB03DAB283
:1007500027490393204600F0B7FA074600283FF4E4
:100760007EAF039B04EB830431E70220FFF710FE0A
:1007700000283FF4F8AE00F0FDF900283FF4F3AE96
:100780004FF000084346019A9268904532D2B8F182
:100790001F0F12D8109A01320FD028F0030218A9A7
:1007A0000A4452F8202C0B92184604220BA900F0A0
:1007B0004FFB08F104080346E5E74046039300F0C9
:1007C00095F9039B0B90EFE70022002058230020AF
:1007D00040220020BD0300085C230020542200209A
:1007E0005E34000804220020082200206034000843
:1007F0005822002018A8042140F84C3D00F04AF986
:10080000E5E618A8002340F8343D642100F038F9EB
:1008100000287FF4A8AE0220FFF7BAFD00283FF4BD
:10082000A2AE0B9800F092F918AB43F8480D0421E2
:100830001846E3E718A8002340F8343D642100F08F
:100840001FF900287FF48FAE0220FFF7A1FD0028DA
:100850003FF489AE0B9800F087F918AB43F8440DCC
:10086000E5E70220FFF794FD00283FF47CAE00F09E
:1008700091F918AB43F8400DD9E70220FFF788FD46
:1008800000283FF470AE0BA9142000F089F98046CF
:1008900018A8042140F83C8D00F0FCF841460BA854
:1008A000ACE7322000F0D8F8B0F10008FFF65BAEFC
:1008B00018F0030F7FF457AE019A926808EB090312
:1008C00093423FF650AE0220FFF762FD00283FF44E
:1008D0004AAE28F00308C844C1453FF478AE484604
:1008E00000F004F904210A900AA800F0D3F809F1F5
:1008F0000409F1E74FF47A70FFF74AFD00283FF44E
:1009000032AE00F037F9002842D0109B01330BD0F3
:10091000082210A9002000F0D7F9002838D02022A2
:10092000FF2110A800F0C8F9FFF73AFD364801F0A2
:1009300009F80FE6002F3FF416AE0AF00B030B2B5D
:100940007FF411AE18A8002340F8343D642100F074
:1009500097F8804600287FF406AE0220FFF718FDC6
:1009600000283FF400AE0390FFF71AFD41F28830F3
:1009700000F0E8FF0B9800F027FA00F0F1F9039B74
:1009800045461F46DBE5074621E64FF00009EAE54C
:10099000B84664E6002000F05FF80490049B002B4A
:1009A000FFF6D0AD012000F057F9049B213B122B3C
:1009B0003FF6C5AD01A252F823F000BF5B05000869
:1009C00081050008170600083F0500083F050008DC
:1009D0003F050008A7060008A30800086B070008E9
:1009E0000308000835080008630800083F050008F0
:1009F0007B0800083F050008F5080008CF0500083F
:100A00003F05000835090008A086010070B50F4BAE
:100A10000C4619780131C9B2012906460FD80C4895
:100A200003681D6A4FF47A73534331462246A84740
:100A3000844204D1074B00221A70012070BD4FF48C
:100A4000FA7000F07FFF002070BD00BF0C22002074
:100A5000502500209023002007B502AB002203F8A8
:100A6000012D012102461846FFF7D0FF20B19DF865
:100A7000070003B05DF804FB4FF0FF30F9E700001A
:100A80000A4608B50421FFF7C1FF80F00100C0B29B
:100A9000404208BD30B4054C2368DD69044B0A466A
:100AA000AC460146204630BC604700BF50250020C0
:100AB000A086010070B501F017FA094C094E20809C
:100AC000002530682388834208D901F007FA33688B
:100AD00005440133B5F5404F3360F2D370BD00BF1C
:100AE000922300206423002001F0ACBA00F10060E2
:100AF00000F540400068704700F10060920000F58A
:100B0000404001F037BA0000054B1A68054B1B88BE
:100B10009B1A834202D9104401F0E0B900207047CB
:100B2000642300209223002038B5074D044628682E
:100B3000204401F0DBF928B928682044BDE838409A
:100B400001F0ECB938BD00BF6423002010F00303AE
:100B500008D1B0F5047F05D200F10050A0F508409F
:100B60000068704700207047014BC058704700BFB5
:100B7000107AFF1F064991F8243033B10023082270
:100B8000086A81F82430FFF7B7BF0120704700BF23
:100B900068230020014B1868704700BF002004E064
:100BA00070B52A4B1C68C4F30B03240C63B140F2EC
:100BB0001342934231D040F2194293422FD040F277
:100BC000214293422DD10323214A0C2505FB032307
:100BD0005D6893F9082042F201039C4224D0B4F5E9
:100BE000805F23D041F201039C4221D041F20303F4
:100BF0009C421FD041F207039C4208BF3122441E91
:100C00000C44013D0B46A3421ED215F9016F581C3E
:100C100096B1034600F8016CF5E70123D4E70223FF
:100C2000D2E73F220B4DD6E73322E3E74122E1E74B
:100C30005A22E4E75922E2E72C2584421D7001D9AB
:100C4000981C5A70401A70BD1846FBE7002004E05B
:100C500070340008643400087047000070470000DA
:100C60007047000010B50023934203D0CC5CC454FD
:100C70000133F9E710BD000030B5441E14F9010F2F
:100C80000B4660B193F90050854201F1010106D194
:100C90001AB993F90020801A30BD013AEEE7002A14
:100CA000F7D1104630BD000002460346981A13F9EA
:100CB000011B0029FAD1704702440346934202D037
:100CC00003F8011BFAE770472DE9F047234C94F82D
:100CD000243005468846174683BB2E46DFF87C90B5
:100CE000C7B394F824302BB92022FF21484626624E
:100CF000FFF7E2FF94F82400C0F10805BD4228BFC9
:100D00003D465FFA85FAAD0041462A4604EB800075
:100D1000FFF7A8FF94F82430A7EB0A079A445FFA7C
:100D20008AFABAF1080F2E44A844FFB284F824A02E
:100D3000D6D1FFF71FFF0028D2D108E0266A06EBC4
:100D40008306B042CAD0FFF715FF0028C5D10020A6
:100D5000BDE8F0870120BDE8F08700BF68230020D0
:100D6000024B1A78024B1A70704700BF9023002084
:100D70000C22002038B5104D104C284600F0F8F831
:100D80002146284600F020F924680D48626DD2F80B
:100D9000043843F00203C2F8043800F0D3FD0949D7
:100DA000204600F01DFA626DD2F8043823F00203E9
:100DB000C2F8043838BD00BF502500206435000853
:100DC00040420F008C35000870470000FEE700002D
:100DD00000B59BB0EFF3098168226846FFF742FF38
:100DE000EFF30583044B9A6BDA6A9A6A9A6A9A6AF5
:100DF0009A6A9A6A9B6AFEE700ED00E000B59BB034
:100E0000EFF3098168226846FFF72CFFEFF30583B3
:100E1000044B9A6B9A6A9A6A9A6A9A6A9A6A9B6A65
:100E2000FEE700BF00ED00E000B59BB0EFF30981E5
:100E300068226846FFF716FFEFF30583034B5A6BF2
:100E40009A6A9A6A9A6A9A6A9B6AFEE700ED00E0DB
:100E500030B5084D0A4491420BD011F8013B0924EA
:100E60005840013CF7D040F300032B4083EA500088
:100E7000F7E730BD2083B8ED026843681143016095
:100E800003B118477047000013B5446BD4F894348D
:100E90001A681178042915D1217C022912D11979F7
:100EA000128901238B4013420CD101A904F14C009B
:100EB00001F04EFFD4F89444019B2179024620684A
:100EC00000F0DAF902B010BD143001F0D1BE00001C
:100ED0004FF0FF33143001F0CBBE00004C3001F076
:100EE000A3BF00004FF0FF334C3001F09DBF000066
:100EF000143001F09FBE00004FF0FF31143001F0BC
:100F000099BE00004C3001F06FBF00004FF0FF327F
:100F10004C3001F069BF0000D0F8942438B5136854
:100F200019780429054601D0012038BD017C022929
:100F3000FAD112795C89012090400440F4D105F186
:100F4000140001F031FE02460028EDD0D5F894548B
:100F50004FF480732868697900F07CF9204638BD29
:100F6000406BFFF7D9BF00000020704770470000BA
:100F70007FB5124B0360002343608360C36001258B
:100F800002260F4B057404460290019300F184027F
:100F9000294600964FF48073143001F0E1FD094BAF
:100FA0000193029400964FF4807304F5237229464E
:100FB00004F14C0001F0A8FE04B070BDC03400087C
:100FC000610F0008890E00080B68202282F3118847
:100FD0000A7903EB820290614A79093243F82200D0
:100FE0008A7912B103EB8203986102230374C0F87B
:100FF0009414002383F311887047000038B5037FF1
:10100000044613B190F85430ABB9201D01250221DC
:10101000FFF732FF04F1140025776FF0010100F0B3
:10102000B9FC84F8545004F14C006FF00101BDE8A4
:10103000384000F0AFBC38BD10B501210446043083
:10104000FFF71AFF0023237784F8543010BD000007
:1010500038B504460025143001F09AFD04F14C0027
:10106000257701F069FE201D84F854500121FFF717
:1010700003FF2046BDE83840FFF74EBF90F84430EC
:1010800003F06003202B19D190F84520212A0AD0C3
:10109000222A4FF000030ED0202A0FD1084A826383
:1010A0000722C26304E0064B83630723C363002364
:1010B0000364012070478363C363F9E7002070472E
:1010C0000D220020D0F8943437B51A68117804291D
:1010D00004461AD1017C022917D1197912890123FA
:1010E0008B40134211D100F14C05284601F0E4FE7B
:1010F00058B101A9284601F02BFED4F89444019B75
:1011000021790246206800F0B7F803B030BD000036
:1011100000EB8103F7B59C6905460E46F4B1202328
:1011200083F3118805EB8607201D0821FFF7A4FE35
:10113000FB685B691B684C3413B1204601F016FE56
:1011400001A9204601F004FE024648B1019B314648
:10115000284600F091F8002383F3118803B0F0BD16
:10116000FB685A691268002AF5D01B8A013B1340BC
:10117000F1D105F14402EAE7093138B550F82140D0
:10118000DCB1202383F31188D4F8942413685279B6
:1011900003EB8203DB689B695D6845B1042160183D
:1011A000FFF76AFE294604F1140001F007FD20460E
:1011B000FFF7B2FE002383F3118838BD70470000AB
:1011C00001F0B0B80123037000234360C361836260
:1011D0000362C3624362036303814381704700007B
:1011E00038B50446202383F3118800254160C5608B
:1011F00005614561856101F0A5F80223237085F33F
:10120000118838BD70B500EB810305465069DA607E
:101210000E46144618B110220021FFF74DFDA069BB
:1012200018B110220021FFF747FD31462846BDE8DE
:10123000704001F051B90000028902F00102028100
:10124000428902F001024281002202614261826110
:1012500001F0D6B9F0B400EB81044789E4680125B8
:10126000A4698D403D43458123600023A2606360F3
:10127000F0BC01F0F1B90000F0B400EB8104078983
:10128000E468012564698D403D43058123600023A6
:10129000A2606360F0BC01F06BBA000070B502237D
:1012A000002504460370A0F84C5080F84E5080F89A
:1012B0004F5005814581C56005614561856180F8B4
:1012C000345001F0A5F863681B6823B12946204615
:1012D000BDE87040184770BD037880F85030052392
:1012E000037043681B6810B504460BB1042198478E
:1012F00000232381638110BD436890F850201B6850
:1013000002700BB1052118477047000090F8343087
:1013100070B5044613B1002380F8343004F1440260
:10132000204601F08FF963689B6863BB94F84450D2
:1013300015F0600615D194F8453005F07F0545EAB3
:10134000032540F202339D4200F00E815BD8022D4E
:1013500000F0DC803FD8002D00F08780012D00F0E8
:10136000CF800021204601F0C7FB0021204601F07C
:10137000B9FB63681B6813B1062120469847062312
:1013800084F8343070BD204698470028CED094F8B9
:101390004B2094F84A3043EA0223E26B934238BF71
:1013A000E36394F94430E56B002B4FF0200380F2A7
:1013B000FD80002D00F0EC80092284F8342083F3B6
:1013C00011880021E36BA26B2046FFF755FF002335
:1013D00083F3118870BDB5F5817F00F0B180B5F55C
:1013E000407F49D0B5F5807FBBD194F84630012BC2
:1013F000B7D1B4F84C3023F00203A4F84C30A66304
:10140000E6632664C3E740F201639D421ED8B5F54A
:10141000C06F3BD2B5F5A06FA3D1B4F84430B3F59B
:10142000A06F0ED194F8463084F84E30204601F07B
:1014300047F863681B6813B10121204698470323CE
:1014400023700023A363E3632364A0E7B5F5106F63
:1014500032D040F602439D4252D0B5F5006F80D1A4
:1014600004F14F03A363012324E004F14C03A363BD
:101470000223E36325648AE794F84630012B7FF466
:1014800070AFB4F84C3043F00203B6E794F849204B
:10149000616894F848304D6894F8471043EA022395
:1014A000204694F84620A84700283FF45AAF4368E6
:1014B000A3630368E363A4E72378042B10D12023FC
:1014C00083F311882046FFF7B7FE86F3118863681F
:1014D00084F84F601B68032121700BB120469847A8
:1014E00094F84630002BACD084F84F30042323709E
:1014F00063681B68002BA4D0022120469847A0E710
:10150000374BA3630223E36300239DE794F848105D
:1015100011F0800F204601F00F010ED001F084F889
:10152000012806D002287FF41CAF2E4BA363E06392
:1015300067E72D4BA363E56363E701F067F8EFE727
:1015400094F84630002B7FF40CAF94F8483013F039
:101550000F013FF476AF1A06204602D501F0E0FAFB
:101560006FE701F0D3FA6CE794F84630002B7FF474
:10157000F8AE94F8483013F00F013FF462AF1B0649
:10158000204602D501F0B8FA5BE701F0ABFA58E764
:10159000142284F8342083F311882B462A462946E6
:1015A0002046FFF757FE85F3118870BD5DB1152207
:1015B00084F8342083F311880021E36BA26B20466A
:1015C000FFF748FE03E70B2284F8342083F31188E9
:1015D0002B462A4629462046FFF74EFEE3E700BF8A
:1015E000F0340008E8340008EC34000838B590F80E
:1015F00034300446152B29D8DFE803F03E2828288C
:1016000028283E28280B293928282828282828284F
:101610003E3E90F84B1090F84A20C36B42EA0122FC
:101620009A4214D9C268128AB3FBF2F502FB15354F
:101630006DB9202383F311882B462A462946FFF7EC
:101640001BFE85F311880A2384F8343038BD142337
:1016500084F83430202383F3118800231A46194676
:101660002046FFF7F7FD002383F3118838BD036C94
:1016700003B198470023E7E7002101F03DFA00217C
:10168000204601F02FFA63681B6813B1062120463B
:1016900098470623D8E7000090F83420152A38B57B
:1016A000044622D80123934040F6416213421DD1E3
:1016B00013F480150FD19B0217D50B2380F834301B
:1016C000202383F311882B462A462946FFF7D4FDB1
:1016D00085F3118838BDC3689B695B682BB9036CBF
:1016E00003B19847002384F8343038BD002101F05D
:1016F00003FA0021204601F0F5F963681B6813B175
:101700000621204698470623EDE70000024B002201
:101710001B605B609A607047942300200023037471
:101720008268054B1B6899689142FBD25A68036036
:1017300042601060586070479423002008B5202351
:1017400083F31188037C032B05D0042B0DD02BB918
:1017500083F3118808BD436900221A604FF0FF33FC
:101760004361FFF7DBFF0023F2E790E80C001A600B
:1017700002685360F2E70000002303748268054B9F
:101780001B6899689142FBD85A68036042601060F8
:101790005860704794230020054B19690874186835
:1017A00002681A605360186101230374FEF7ACBD30
:1017B0009423002030B54B1C87B005460A4C10D04E
:1017C00023690A4A01A800F001F92846FFF7E4FF5F
:1017D000049B13B101A800F04BF92369586907B0C5
:1017E00030BDFFF7D9FFF8E7942300203D1700082C
:1017F00038B50C4D41612B6981689A689142044665
:1018000003D8BDE83840FFF789BF1846FFF7B4FF9B
:1018100001232C61014623742046BDE83840FEF7C1
:1018200073BD00BF94230020044B1A681B699068A5
:101830009B68984294BF00200120704794230020A9
:1018400010B5084C236820691A6822605460012290
:1018500023611A74FFF790FF01462069BDE810402C
:10186000FEF752BD94230020FEE7000010B50C4C9B
:10187000FFF74CFF00F09CF880220A49204600F058
:1018800021F8012344F8180C037400F067FC0023CE
:1018900083F3118862B60448BDE8104000F034B804
:1018A000BC230020F4340008FC34000800F01AB90E
:1018B000034B59685A68521A9042FBD8704700BFD0
:1018C000001000E08260022202740022427470471D
:1018D0008368A3F17C0243F80C2C026943F83C2C8A
:1018E000426943F8382C074A43F81C2CC26843F875
:1018F000102C022203F8082C002203F8072CA3F175
:10190000180070472103000810B5202383F31188C5
:10191000FFF7DEFF00210446FFF76AFF002383F391
:101920001188204610BD0000024B1B6958610F2032
:10193000FFF732BF94230020202383F31188FFF7A1
:10194000F3BF000008B50146202383F31188082067
:10195000FFF730FF002383F3118808BD49B1064B20
:1019600042681B6918605A60136043600420FFF7E7
:1019700021BF4FF0FF307047942300200368984246
:1019800006D01A680260506059611846FFF7C6BE5B
:101990007047000038B504460D462068844200D1E7
:1019A00038BD036823605C604561FFF7B7FEF4E76C
:1019B000054B03F114025A619A614FF0FF32DA616C
:1019C00000221A62704700BF94230020F8B5274F09
:1019D0000361C2600D46044601F0A2FA3B46022DA7
:1019E00053F8142F294638BF02219A423E461D461D
:1019F0000AD138627C61BC61084422606260A160E7
:101A0000BDE8F84001F07ABAD7F820E0A0EB0E0369
:101A10005F181FD300279068834217D8376AAA42FD
:101A20001F44376201D0C01A906073699A6891426E
:101A300019D85A682360626014605C60A16098687D
:101A4000411A99604FF0FF33F361F8BD97601B1A9C
:101A50001268E0E793689F4203D20EEB070001F0A3
:101A60005BFA3946E1E7891A1B68DFE79423002017
:101A700038B51B4B01685A6990421D4603F11402A8
:101A80000CD0446821600368002193425C60C1600F
:101A900025D09A6881680A449A6038BD59614A60C5
:101AA0005B6900219342C16003D1BDE8384001F079
:101AB0002DBA9A6881680A449A602C6A01F030FA5B
:101AC0006A699268001B824209D9111A012998BFDC
:101AD000821C286ABDE83840104401F01DBA38BDA8
:101AE000942300202DE9F84F204C0027656904F16C
:101AF0001406B84601F014FA236AA0EB030AAB6897
:101B000053451DD84FF02009236AAA68D5F80CB0B8
:101B100013442362AB68AAEB030A2B68B3425E60EE
:101B20006361EF6001D101F0F1F988F31188286950
:101B3000D84789F311886569AB689A45E4D2D9E73B
:101B40006369B34210D020629A68A2EB0A029A60DD
:101B5000226AAB68821A9B1A022B2CBFC018023073
:101B6000BDE8F84F01F0D8B9BDE8F88F9423002004
:101B700000207047FEE70000704700004FF0FF3084
:101B800070470000022906D0032906D00129064823
:101B900018BF0020704705487047032A9ABF0448C1
:101BA00000EBC20000207047E83500089C350008B3
:101BB0001C22002070B59AB001AD064608462946A1
:101BC000144600F0BDF82846FFF76EF8C0B2431C7B
:101BD0005B0086E81800237003236370002302343F
:101BE0001946DAB2904204F1020401D81AB070BD6D
:101BF000EA5C04F8022C04F8011C0133F1E7000050
:101C000008B5202383F311880348FFF75BFA00230C
:101C100083F3118808BD00BF5025002090F84430A0
:101C200003F01F02012A07D190F845200B2A03D1A7
:101C300000238363C36312E003F06003202B11D100
:101C4000B0F8483073B990F84520212A03D0222AF1
:101C5000EFD0202A06D1044A82630722C2630364BC
:101C600001207047FFF70ABA1422002010B504467D
:101C7000052916D8DFE801F016150316161D2023D6
:101C800083F311880E4A0121FFF7BCFA20460D4A62
:101C90000221FFF7B7FA0C48FFF7DAF9002383F3C4
:101CA000118810BD202383F311880748FFF7A6F998
:101CB000F4E7202383F311880348FFF7BDF9EDE72C
:101CC0001C350008403500085025002038B50C4D63
:101CD0000C4C0D492A4604F10800FFF76BFF05F193
:101CE000CA0204F110000949FFF764FF05F5CA7242
:101CF00004F118000649BDE83840FFF75BBF00BF9C
:101D0000182A00201C2200206C35000876350008B7
:101D10008135000870B5044608460D46FEF7C4FF3D
:101D2000C6B22046013403780BB9184670BD32465E
:101D30002946FEF7A1FF0028F3D1012070BD000065
:101D40002DE9F04704460D46FEF7AEFF2D49C6B219
:101D50002046FFF7DFFF08B10836F6B22A492046D1
:101D6000FFF7D8FF08B11036F6B2632E0BD8DFF8B4
:101D70009480DFF89490254FDFF89CA0267846B930
:101D80002E70BDE8F08721462846BDE8F04701F0F7
:101D90005DBB252E31D1072241462046FEF76CFF60
:101DA00080B91B4B2A4603F10C0153F8040B42F88F
:101DB000040B8B42F9D119889B78118093700734FA
:101DC0000F35DBE7082249462046FEF755FFA0B94C
:101DD000104BAA1C13F8011F09095345C95D02F8ED
:101DE000021C197801F00F0102F10202C95D02F82C
:101DF000031CEFD118350834C0E72E7001340135CB
:101E0000BCE700BF0836000881350008203600080E
:101E1000103600080F7AFF1F1B7AFF1FBFF34F8F8A
:101E2000024AD368DB03FCD4704700BF003C024089
:101E300008B5094B1B7873B9FFF7F0FF074B1A6918
:101E4000002ABFBF064A5A6002F188325A601A68F7
:101E500022F480621A6008BD762C0020003C02400B
:101E60002301674508B50B4B1B7893B9FFF7D6FFE5
:101E7000094B1A6942F000421A611A6842F4805212
:101E80001A601A6822F480521A601A6842F480625A
:101E90001A6008BD762C0020003C02400B2870B56B
:101EA00013D80B4A0B4C137863B90B4E4FF00061FB
:101EB00044F8231056F8235001330C2B2944F7D152
:101EC0000123137054F8200070BD002070BD00BFC6
:101ED000A82C0020782C002034360008014B53F841
:101EE00020007047343600080C2070470B2810B5CE
:101EF000044601D9002010BDFFF7D0FF064B53F870
:101F000024301844C21A0BB9012010BD12680132E6
:101F1000F0D1043BF6E700BF343600080B2810B5BB
:101F2000044621D8FFF77AFFFFF782FF0F4AF32319
:101F3000D360C300DBB243F4007343F002031361C8
:101F4000136943F480331361FFF768FFFFF7A6FFBF
:101F5000074B53F8241000F0DDF8FFF783FF20460D
:101F6000BDE81040FFF7C2BF002010BD003C02409A
:101F7000343600082DE9F84312F00103154640D12C
:101F80008218B2F1016F3CD22C4B1B6813F0010395
:101F900037D02B4CFFF74CFFF323E360FFF73EFFF6
:101FA00040F20127032D01D9830713D0244C0F469B
:101FB000401A40F20118EB1B0B44012B00EB070603
:101FC000236924D823F001032361FFF74BFF01208D
:101FD000BDE8F883236923F44073236123693B43FD
:101FE000236151F8046B0660BFF34F8FFFF716FFB4
:101FF00003689E4208D0236923F001032361FFF7A1
:1020000031FF0020BDE8F883043D0430CAE723F423
:1020100040732361236943EA08032361B94637F813
:10202000023B3380BFF34F8FFFF7F8FE3688B9F8D5
:102030000030B6B2B342BED0DDE700BF0038024088
:10204000003C0240084908B50B7828B153B9FFF7A6
:10205000EFFE01230B7008BD23B1BDE808400870F6
:10206000FFF700BF08BD00BF762C002010B502446A
:10207000064B0439D2B2904200D110BD441C00B2CC
:1020800053F8200041F8040FE0B2F4E75028004074
:10209000104B30B51C6F240407D41C6F44F400743B
:1020A0001C671C6F44F400441C670B4C236843F40A
:1020B000807323600244094B0439D2B2904200D1AC
:1020C00030BD441C00B251F8045F43F82050E0B228
:1020D000F4E700BF00380240007000405028004084
:1020E00007B5012201A90020FFF7C0FF019803B046
:1020F0005DF804FB13B50446FFF7F2FFA04206D0DB
:1021000002A9012241F8044D0020FFF7C1FF02B0EF
:1021100010BD000070470000034B1B689B0042BFCE
:10212000024B01221A70704774380240A92C00201B
:10213000014B1878704700BFA92C0020EFF30983EA
:1021400005494A6822F001024A60683383F309882E
:10215000002383F31188704730EF00E0202080F3E4
:10216000118862B60B4B0C4AD96821F4E06109046E
:10217000090C0A430949DA60CA6842F08072CA60F1
:1021800007490A6842F001020A601022DA7783F8F0
:102190002200704700ED00E00003FA05F0ED00E0DA
:1021A000001000E010B5202383F311880E4B5B680C
:1021B00013F4006314D0F1EE103AEFF30984683C95
:1021C0004FF08073E361094BDB68236684F3098871
:1021D000FFF72AFB10B1064BA36110BD054BFBE7CF
:1021E00083F3118810BD00BF00ED00E030EF00E088
:1021F000330300083603000870470000FEE70000C4
:10220000084A094B09498B4204D3094A00219342E9
:1022100005D3704752F8040F43F8040BF3E743F873
:10222000041BF4E7C8370008A42D0020A42D0020CB
:10223000A42D0020836D70B5446D9E6800214FF081
:10224000FF354A01A3180131D3F800090028BEBFA9
:10225000D3F8000940F08040C3F80009D3F8000B20
:102260000028BEBFD3F8000B40F08040C3F8000B3D
:10227000A3188E42C3F80859C3F8085BE1D24FF0A7
:102280000113C4F81C3870BD890141F020010161BF
:1022900003699B06FCD41220FFF70ABB204B03EB1B
:1022A00080022DE9F047D2F80CE05D6DDEF81420D5
:1022B000461CD2F800C005EB063605EB4018516805
:1022C00061450BD3D5F83428012303FA00F022EA44
:1022D0000000C5F834081846BDE8F087BEF8104085
:1022E000ACEB0103A34228BF2346D8F81849A4B297
:1022F000B3EB840F10D894681F46A4F1040959F871
:1023000004AFC6F800A0042F01D9043FF7E71C442E
:102310000B4494605360D2E70020BDE8F08700BF13
:10232000AC2C002010B5054C2046FEF74BFF4FF0BB
:10233000A0436365024BA36510BD00BFAC2C002019
:10234000883600080378012B70B5054650D12A4B1A
:10235000446D98421BD1294B5A6B42F080025A635C
:102360005A6D42F080025A655A6D5A6942F08002F5
:102370005A615A6922F080025A610E2143205B693A
:1023800000F0D8FB1E4BE3601E4BC4F8003800235E
:10239000C4F8003EC02323606E6D4FF40413A363A2
:1023A0003369002BFCDA012333610C20FFF780FA3C
:1023B0003369DB07FCD41220FFF77AFA3369002B6C
:1023C000FCDA0026A6602846FFF734FF6B68C4F8E5
:1023D0001068DB68C4F81468C4F81C684BB90A4B71
:1023E000A3614FF0FF336361A36843F00103A3606F
:1023F00070BD064BF4E700BFAC2C00200038024053
:102400004014004003002002003C30C0083C30C0B3
:10241000F8B5446D054600212046FFF735FFA96D4C
:1024200000234FF001128F68C4F834384FF0006673
:10243000C4F81C284FF0FF3004EB431201339F42D5
:10244000C2F80069C2F8006BC2F80809C2F8080BAC
:10245000F2D20B686A6DEB65636210231361166933
:1024600016F01006FBD11220FFF722FAD4F800383C
:1024700023F4FE63C4F80038A36943F4402343F017
:102480001003A3610923C4F81038C4F814380A4BA8
:10249000EB604FF0C043C4F8103B084BC4F8003B5E
:1024A000C4F81069C4F80039EB6D03F1100243F46D
:1024B0008013EA65A362F8BD64360008408000100E
:1024C000426D90F84E10D2F8003823F4FE6343EAD0
:1024D0000113C2F8003870472DE9F0410EB200EB4D
:1024E00086080D46D8F80C100F6807F00303022B7E
:1024F00050D0032B50D03D4A3D4F012B18BF1746FB
:10250000446D4FEA451E04EB0E030022C3F8102B66
:102510008A6905F1100C002A40D04A8A05F1580357
:102520005B013A43E2500123D4F81C2803FA0CF370
:102530001343A6444A69C4F81C380023CEF8103966
:1025400005F13F03002A39D00A8A898B92080129B4
:1025500088BF4A43C16D04EB8303561841EA024227
:10256000C66529465A602046FFF78EFED8F80C3023
:102570001B8A43EA85531F4305F148035B01E7507B
:102580000123D4F81C2803FA05F51543C4F81C5898
:10259000BDE8F081174FB3E7174FB1E704EB4613DF
:1025A000D3F8002B22F40042C3F8002BD4F81C28E7
:1025B000012303FA0CF322EA0303BAE704EB8303D3
:1025C0000E4A5A6004EB461629462046FFF75CFE89
:1025D000D6F8003923F40043C6F80039D4F81C3883
:1025E000012202FA05F523EA0505CFE70080001075
:1025F000008004100080081000800C10000400020D
:10260000826D1268C265FFF715BE00005831436D38
:1026100049015B5813F4004004D013F4001F14BFA9
:1026200001200220704700004831436D49015B588A
:1026300013F4004004D013F4001F14BF0120022043
:102640007047000000EB8101CB68196A0B681360CA
:102650004B6853607047000000EB810330B5DD68C4
:10266000AA691368D36019B9402B84BF4023136053
:102670006B8A1468426D1C44013CB4FBF3F4634361
:10268000033323F0030302EB411043EAC44343F056
:10269000C043C0F8103B2B6803F00303012B09B2C1
:1026A0000ED1D2F8083802EB411013F4807FD0F835
:1026B000003B14BF43F0805343F00053C0F8003B8D
:1026C00002EB4112D2F8003B43F00443C2F8003B56
:1026D00030BD00002DE9F041244D6E6D06EB401336
:1026E0000446D3F8087BC3F8087B38070AD5D6F828
:1026F0001438190706D505EB84032146DB68284604
:102700005B689847FA072FD5D6F81438DB072BD526
:1027100005EB8403D968CCB98B69488A5E68B6FB3F
:10272000F0F200FB12628AB91868DA6890420DD2A2
:10273000121A83E81400202383F311880B482146E2
:10274000FFF78AFF84F31188BDE8F081012303FAC3
:1027500004F26B8923EA02036B81CB6823B1214623
:102760000248BDE8F0411847BDE8F081AC2C0020DC
:1027700000EB810370B5DD68436D6C692668E66027
:102780004A0156BB1A444FF40020C2F810092A68C7
:1027900002F00302012A0AB20ED1D3F8080803EBB3
:1027A000421410F4807FD4F8000914BF40F0805028
:1027B00040F00050C4F8000903EB4212D2F80009BF
:1027C00040F00440C2F80009D3F83408012202FAAC
:1027D00001F10143C3F8341870BD19B9402E84BF0C
:1027E0004020206020682E8A841940F00050013C6F
:1027F0001A44B4FBF6F440EAC440C6E7F8B5044610
:102800001E48456D05EB4413D3F80869C3F8086901
:10281000F10717D5D5F81038DA0713D500EB840384
:10282000D9684B691F68DA68974218D2D21B002713
:102830001A605F60202383F311882146FFF798FF19
:1028400087F31188330617D5D5F834280123A34020
:10285000134211D02046BDE8F840FFF71FBD012309
:1028600003FA04F2038923EA020303818B68002B35
:10287000E8D021469847E5E7F8BD00BFAC2C002022
:1028800097482DE9F84F456D6E69AB691E4016F407
:10289000805F6E61044605D0FEF700FDBDE8F84F8D
:1028A000FFF780BC002E12DAD5F8003E8C489B075B
:1028B0001EBFD5F8003E23F00303C5F8003ED5F84F
:1028C000043823F00103C5F80438FEF715FD370579
:1028D00005D58348FFF7AEFC8148FEF7FDFCB00448
:1028E0000CD5D5F8083813F0060FEB6823F47053B5
:1028F0000CBF43F4105343F4A053EB60310704D5ED
:102900006368DB680BB176489847F2025AD4B30289
:102910000CD5D4F85480DFF8C8A100274FF0010986
:10292000A36D9B68F9B28B4280F08780F70619D5BA
:10293000616D0A6AC2F30A1702F00F0302F4F01283
:10294000B2F5802F00F0A180B2F5402F0AD104EB40
:10295000830301F58051DB68186A00231A469F4201
:1029600040F087803003D5F8184813D5E10302D52D
:102970000020FFF7AFFEA20302D50120FFF7AAFE59
:10298000630302D50220FFF7A5FE270302D503202B
:10299000FFF7A0FE750381D5E00702D50020FFF701
:1029A0002DFFA10702D50120FFF728FF620702D5FE
:1029B0000220FFF723FF23077FF570AF0320FFF707
:1029C0001DFF6BE7D4F85480DFF814A100274FF007
:1029D0000109A36D9B685FFA87FB5B4597D308EB02
:1029E0004B13D3F8002902F44022B2F5802F22D1F4
:1029F000D3F80029002A1EDAD3F8002942F09042C9
:102A0000C3F80029D3F80029002AFBDB5946606D82
:102A1000FFF73AFC228909FA0BF322EA0303238128
:102A200004EB8B03DB689B6813B15946504698470B
:102A30005846FFF733FC0137CBE708EB4112D2F8D9
:102A4000003B03F44023B3F5802F10D1D2F8003BB4
:102A5000002B0CDA628909FA01F322EA030363818D
:102A600004EB8103DB68DB680BB150469847013704
:102A700056E79C0708BF0A68072B98BF027003F14E
:102A800001039CBF120A013069E7023304EB8302A1
:102A900001F58051526890690268D0F808C040681A
:102AA000A2EB000E0022104697420AD104EB8304E9
:102AB00063689B699A683A449A605A6817445F60F1
:102AC00050E712F0030F08BF0868964588BF8CF8DE
:102AD000000002F1010284BF000A0CF1010CE3E7DF
:102AE000AC2C0020436D03EB4111D1F8003B43F4C3
:102AF0000013C1F8003B7047436D03EB4111D1F85F
:102B0000003943F40013C1F800397047436D03EBFB
:102B10004111D1F8003B23F40013C1F8003B70478A
:102B2000436D03EB4111D1F8003923F40013C1F8D0
:102B30000039704700F1604300F01F02400903F5BF
:102B4000614309018000C9B200F1604083F80013BD
:102B500000F5614001239340C0F880310360704765
:102B600030B5039C0172043304FB0325C361049B4D
:102B700003630021059B00604060C1604261026107
:102B80008561046242628162C162436330BD0000BC
:102B90000022416A41610161C2608262C2626FF0DB
:102BA0000101FEF7F7BE000003694269934203D1B9
:102BB000C2680AB100207047181D70470369196088
:102BC000C2680132C260C2691344826903619342E0
:102BD00024BF436A03610021FEF7D0BE38B5044626
:102BE0000D46E3683BB16269131D1268A36213448A
:102BF000E362002038BD237A33B929462046FEF728
:102C0000ADFE0028EDDA38BD6FF00100FBE70000F3
:102C1000C368C269013BC36043691344826943616D
:102C2000934224BF436A436100238362036B03B171
:102C30001847704770B52023044683F31188866ACD
:102C40003EB9FFF7CBFF054618B186F31188284639
:102C500070BDA36AE26A13F8015BA362934202D3D8
:102C60002046FFF7D5FF002383F31188EFE700002C
:102C70002DE9F84F04460E4690469946202787F3E3
:102C800011880025AA46D4F828B0BBF1000F09D15D
:102C900049462046FFF7A2FF20B18BF31188284652
:102CA000BDE8F88FA16AE36AA8EB050B5B1A9B45A8
:102CB00028BF9B46BBF1400F1BD9334601F14002B0
:102CC00051F8040B43F8040B9142F9D1A36A403345
:102CD0004036A3624035A26AE36A9A4202D3204694
:102CE000FFF796FF8AF311884545D8D287F31188FC
:102CF000C9E730465A46FDF7B5FFA36A5B445E4418
:102D0000A3625D44E7E7000010B5029C0172043342
:102D100003FB0421C36100238362C362039B03633B
:102D2000049B00604060C460426102618161046292
:102D30004262436310BD0000026AC260426A42619F
:102D4000026100228262C2626FF00101FEF722BEC0
:102D5000436902699A4203D1C2680AB100207047F0
:102D6000184650F8043B0B6070470000C368C26906
:102D70000133C3604369134482694361934224BFB2
:102D8000436A43610021FEF7F9BD000038B50446EF
:102D90000D46E3683BB123691A1DA262E269134440
:102DA000E362002038BD237A33B929462046FEF776
:102DB000D5FD0028EDDA38BD6FF00100FBE700001B
:102DC00003691960C268013AC260C269134482692A
:102DD0000361934224BF436A036100238362036B50
:102DE00003B118477047000070B5202304460E4613
:102DF00083F31188856A35B91146FFF7C7FF10B113
:102E000085F3118870BDA36A1E70A36AE26A01335C
:102E10009342A36204D3E16920460439FFF7D0FF4F
:102E2000002080F3118870BD2DE9F84F04460D464F
:102E300091469A464FF0200888F311880026B34641
:102E4000A76A4FB951462046FFF7A0FF20B187F38C
:102E500011883046BDE8F88FA06AE76AA9EB06033F
:102E60003F1A9F4228BF1F46402F1BD905F1400340
:102E700055F8042B40F8042B9D42F9D1A36A403346
:102E8000A3624036A26AE36A9A4204D3E16920460B
:102E90000439FFF795FF8BF311884E45D9D288F39B
:102EA0001188CDE729463A46FDF7DCFEA36A3B448C
:102EB0003D44A3623E44E5E7026943699A4203D177
:102EC000C3681BB9184670470023FBE7836A002BD1
:102ED000F8D0043B9B1AF5D01360C368013BC36074
:102EE000C3691A44836902619A4224BF436A036139
:102EF000002383620123E5E700F090B84FF08043A0
:102F0000002258631A610222DA6070474FF0804352
:102F10000022DA60704700004FF08043586370472A
:102F20004FF08043586A70474B6843608B688360FA
:102F3000CB68C3600B6943614B6903628B69436271
:102F40000B6803607047000008B5224B22481A69DD
:102F500040F2FF110A431A611A6922F4FF7222F04B
:102F600001021A611A691A6B0A431A631A6D0A433D
:102F70001A651A4A1B6D1146FFF7D6FF184802F171
:102F80001C01FFF7D1FF174802F13801FFF7CCFF12
:102F9000154802F15401FFF7C7FF144802F1700110
:102FA000FFF7C2FF124802F18C01FFF7BDFF114885
:102FB00002F1A801FFF7B8FF0F4802F1C401FFF7C3
:102FC000B3FF0E4802F1E001FFF7AEFFBDE8084095
:102FD00000F0AAB800380240000002409436000811
:102FE0000004024000080240000C024000100240B1
:102FF0000014024000180240001C02400020024061
:1030000008B500F007FAFEF731FCFFF785F8BDE8D8
:103010000840FEF75BBE000070470000104B1A6CC2
:1030200042F001021A641A6E42F001021A660D4A59
:103030001B6E936843F0010393604FF0804353226B
:103040009A624FF0FF32DA6200229A615A63DA60C4
:103050005A6001225A6108211A601C20FFF76ABDDC
:1030600000380240002004E04FF0804208B51369A8
:10307000D1680B40D9B2C9439B07116107D5202302
:1030800083F31188FEF712FC002383F3118808BD37
:1030900008B5FFF7E9FFBDE80840FFF783B8000077
:1030A0001F4B1A696FEAC2526FEAD2521A611A694B
:1030B000C2F308021A614FF0FF301A695A69586169
:1030C00000215A6959615A691A6A62F080521A627B
:1030D0001A6A02F080521A621A6A5A6A58625A6A66
:1030E00059625A6A1A6C42F080521A641A6E42F09F
:1030F00080521A661A6E0B4A106840F48070106095
:10310000186F00F44070B0F5007F1EBF4FF48030A0
:1031100018671967536823F40073536000F05AB9B5
:103120000038024000700040334B4FF080521A6468
:10313000324A4FF4404111601A6842F001021A60AD
:103140001A689207FCD59A6822F003029A602A4B0B
:1031500019469A6812F00C02FBD1186800F0F900C9
:1031600018609A601A6842F480321A600B689B03F8
:10317000FCD54B6F43F001034B671F4B5A6F900711
:10318000FCD51F4A5A601A6842F080721A601B4AC6
:1031900053685904FCD5184B1A689201FCD5194A9A
:1031A0009A60194B1A68194B9A42194B21D1194A46
:1031B0001168194A91421CD140F205121A60144A52
:1031C000136803F00F03052BFAD10B4B9A6842F0FA
:1031D00002029A609A6802F00C02082AFAD15A6C2C
:1031E00042F480425A645A6E42F480425A665B6EE0
:1031F000704740F20572E1E700380240007000407D
:103200000854400700948838002004E0116400202E
:10321000003C024000ED00E041C20F41084A08B501
:10322000536911680B4003F00103536123B1054A50
:1032300013680BB150689847BDE80840FEF7B2BF6D
:10324000003C0140242D0020084A08B5536911684C
:103250000B4003F00203536123B1054A93680BB19D
:10326000D0689847BDE80840FEF79CBF003C01408D
:10327000242D0020084A08B5536911680B4003F05B
:103280000403536123B1054A13690BB15069984790
:10329000BDE80840FEF786BF003C0140242D002019
:1032A000084A08B5536911680B4003F008035361DD
:1032B00023B1054A93690BB1D0699847BDE808402E
:1032C000FEF770BF003C0140242D0020084A08B5DD
:1032D000536911680B4003F01003536123B1054A91
:1032E000136A0BB1506A9847BDE80840FEF75ABF11
:1032F000003C0140242D0020174B10B55C691A6872
:10330000144004F478725A61A30604D5134A936AF0
:103310000BB1D06A9847600604D5104A136B0BB105
:10332000506B9847210604D50C4A936B0BB1D06BB8
:103330009847E20504D5094A136C0BB1506C9847C5
:10334000A30504D5054A936C0BB1D06C9847BDE832
:103350001040FEF727BF00BF003C0140242D002095
:103360001A4B10B55C691A68144004F47C425A6127
:10337000620504D5164A136D0BB1506D98472305AD
:1033800004D5134A936D0BB1D06D9847E00404D572
:103390000F4A136E0BB1506E9847A10404D50C4A26
:1033A000936E0BB1D06E9847620404D5084A136F30
:1033B0000BB1506F9847230404D5054A936F0BB1A6
:1033C000D06F9847BDE81040FEF7ECBE003C0140CE
:1033D000242D0020062108B50846FFF7ABFB062187
:1033E0000720FFF7A7FB06210820FFF7A3FB062114
:1033F0000920FFF79FFB06210A20FFF79BFB062110
:103400001720FFF797FB06212820BDE80840FFF7AB
:1034100091BB000008B5FFF743FE00F00BF8FDF785
:10342000CFFEFDF7A3FDFFF7F7FDBDE80840FFF76E
:1034300063BD0000002304491A465A50C8180833D7
:10344000802B4260F9D17047242D0020034611F8EB
:10345000012B03F8012B002AF9D170471210121327
:103460001211000053544D3332463F3F3F000000DD
:1034700000000000643400083F0000001304000056
:10348000A03400083F00000019040000AA3400081E
:103490003F00000021040000B43400083F00000099
:1034A00053544D3332463430780053544D33324602
:1034B0003432780053544D33324634343658580041
:1034C00000000000E50E0008D10E00080D0F0008F6
:1034D000F90E0008050F0008F10E0008DD0E0008C7
:1034E000C90E0008690F000800000000010000007C
:1034F000000000006D61696E0000000014350008D6
:10350000D823002050250020010000006918000881
:103510000000000069646C6500000000020000000B
:10352000000000001111000879110008400040005F
:10353000E8290020F8290020020000000000000017
:103540000300000000000000BD11000800000000A2
:1035500010000000082A0020000000000100000008
:1035600000000000AC2C00200101020041726475D3
:1035700050696C6F740025424F415244252D424CD6
:10358000002553455249414C250000006D1C0008A0
:10359000851B00081D1C0008011C000843000000DA
:1035A000A435000809024300020100C032090400EA
:1035B00000010202010005240010010524010001A0
:1035C000042402020524060001070582030800FF07
:1035D00009040100020A0000000705010240000082
:1035E000070581024000000012000000F0350008CD
:1035F00012011001020000400912415700020102AD
:10360000030100000403090425424F4152442500F0
:103610004D616D62614634303555532D493243005A
:1036200030313233343536373839414243444546F8
:1036300000000000004000000040000000400000CA
:103640000040000000000100000002000000020035
:103650000000020000000200000002000000020062
:1036600000000200000000000D130008ED15000826
:1036700099160008400040000C2D00200C2D002061
:10368000010000001C2D002080000000400100000F
:10369000030000000000800200000000AAAAAAAAFD
:1036A00000000000FFFF00000000000000A00A0072
:1036B0000000000000000000AAAAAAAA0000000062
:1036C000FFFF0000000000000000000000000050AC
:1036D00000000000AAAAAAAA00000000FF3F000004
:1036E00000000000000000000000000000000000DA
:1036F000AAAAAAAA00000000FFFF00000000000024
:10370000000000000000000000000000AAAAAAAA11
:1037100000000000FFFF00000000000000000000AB
:103720000000000000000000AAAAAAAA00000000F1
:10373000FFFF00000000000000000000000000008B
:1037400000000000AAAAAAAA00000000FFFF0000D3
:103750000000000000000000000000000000000069
:103760000A0000000000000003000000000000004C
:103770000000000000000000000000000000000049
:103780000000000000000000000000000000000039
:103790000E0400000000000000400F00FF00960033
:1037A000000000080096000000000800040000006F
:1037B00004360008000000000000000000000000C7
:1037C000000000000000000000000000FFFFFFFFFD
:1037D000FFFFFFFFFFFFFFFFFFFFFFFFFFFFFFFFF9
:1037E000FFFFFFFFFFFFFFFFFFFFFFFFFFFFFFFFE9
:1037F000FFFFFFFFFFFFFFFFFFFFFFFFFFFFFFFFD9
:10380000FFFFFFFFFFFFFFFFFFFFFFFFFFFFFFFFC8
:10C000000006002089D20008414206089D4106082A
:10C01000094206089D410608D54106088BD2000852
:10C020008BD200088BD200088BD200082D1808088C
:10C030008BD200088BD200088BD200088BD200086C
:10C040008BD200088BD200088BD200088BD200085C
:10C050008BD200088BD20008492A0808712A0808E8
:10C06000992A0808C12A0808E92A0808E5D3070818
:10C070000DD4070839D4070865D4070891D40708F8
:10C08000B9D40708E5D4070869D307088BD200089C
:10C090008BD200088BD200088BD20008112B080825
:10C0A0005D2C0808612C0808752C0808792C0808F4
:10C0B0008BD200087D2C0808912C080871DA07083B
:10C0C00019DC07088BD200088BD200088BD200083D
:10C0D0008BD20008E52B0808F92B08080D2C08085E
:10C0E000752B08088BD200088BD200088BD2000871
:10C0F0008BD200088BD200088BD2000811D507081C
:10C100008BD200088BD20008A52C08088BD200081F
:10C11000212C0808352C08088BD200088BD2000887
:10C120003DD5070865D5070891D50708BDD507088F
:10C13000E9D507088BD200088BD200088BD2000803
:10C140008BD200088BD200088BD20008591F080838
:10C1500011D607083DD6070869D60708492C0808F4
:10C160008BD200088BD200088BD200088BD200083B
:10C170008BD200088BD200088BD200088BD200082B
:10C180008BD200088BD200088BD200088BD200081B
:10C190008BD200088BD200088BD200088BD200080B
:10C1A0008BD200088BD200088BD200088BD20008FB
:10C1B0008BD200088BD200088BD200088BD20008EB
:10C1C0008BD200088BD200088BD200088BD20008DB
:10C1D0008BD200088BD200088BD200088BD20008CB
:10C1E00021E700080DF70008355B010835AD0208AE
:10C1F000112A04087D4404081D910408E1980408EC
:10C20000199C040859FB0408D5160508D9880508A7
:10C21000F53A0608ADCA060801FC0608E55007080D
:10C22000B5770708D981070899AF0708C1B507088E
:10C2300081F0004102E000BF83F0004330B54FEAD7
:10C2400041044FEA430594EA050F08BF90EA020F44
:10C250001FBF54EA000C55EA020C7FEA645C7FEAD7
:10C26000655C00F0E2804FEA5454D4EB5555B8BFFA
:10C270006D420CDD2C4480EA020281EA030382EA6B
:10C28000000083EA010180EA020281EA0303362DFD
:10C2900088BF30BD11F0004F4FEA01314FF4801CD0
:10C2A0004CEA113102D0404261EB410113F0004FE2
:10C2B0004FEA03334CEA133302D0524263EB430399
:10C2C00094EA050F00F0A780A4F10104D5F1200E37
:10C2D0000DDB02FA0EFC22FA05F2801841F1000192
:10C2E00003FA0EF2801843FA05F359410EE0A5F166
:10C2F00020050EF1200E012A03FA0EFC28BF4CF097
:10C30000020C43FA05F3C01851EBE37101F000454C
:10C3100007D54FF0000EDCF1000C7EEB00006EEB59
:10C320000101B1F5801F1BD3B1F5001F0CD34908E3
:10C330005FEA30004FEA3C0C04F101044FEA44523A
:10C3400012F5800F80F09A80BCF1004F08BF5FEAC1
:10C35000500C50F1000041EB045141EA050130BDA1
:10C360005FEA4C0C404141EB0101013C28BFB1F5B3
:10C37000801FE9D291F0000F04BF01460020B1FAFE
:10C3800081F308BF2033A3F10B03B3F120020CDAD1
:10C390000C3208DD02F1140CC2F10C0201FA0CF0AF
:10C3A00021FA02F10CE002F11402D8BFC2F1200C14
:10C3B00001FA02F120FA0CFCDCBF41EA0C019040CA
:10C3C000E41AA2BF01EB0451294330BD6FEA040413
:10C3D0001F3C1CDA0C340EDC04F11404C4F12002FE
:10C3E00020FA04F001FA02F340EA030021FA04F310
:10C3F00045EA030130BDC4F10C04C4F1200220FA67
:10C4000002F001FA04F340EA0300294630BD21FAA4
:10C4100004F0294630BD94F0000F83F4801306BF6A
:10C4200081F480110134013D4EE77FEA645C18BF5E
:10C430007FEA655C29D094EA050F08BF90EA020FF5
:10C4400005D054EA000C04BF1946104630BD91EAED
:10C45000030F1EBF0021002030BD5FEA545C05D1F0
:10C460004000494128BF41F0004130BD14F580042F
:10C470003CBF01F5801130BD01F0004545F0FE41A3
:10C4800041F470014FF0000030BD7FEA645C1ABFD8
:10C49000194610467FEA655C1CBF0B46024650EA0F
:10C4A000013406BF52EA033591EA030F41F400213B
:10C4B00030BD00BF90F0000F04BF0021704730B5C1
:10C4C0004FF4806404F132044FF000054FF0000196
:10C4D00050E700BF90F0000F04BF0021704730B557
:10C4E0004FF4806404F1320410F0004548BF40422C
:10C4F0004FF000013EE700BF42004FEAE2014FEA81
:10C5000031014FEA02701FBF12F07F4393F07F4F5B
:10C5100081F06051704732F07F4208BF704793F05E
:10C520007F4F04BF41F40021704730B54FF4607471
:10C5300001F0004521F000411CE700BF50EA010274
:10C5400008BF704730B54FF000050AE050EA01021D
:10C5500008BF704730B511F0004502D5404261EB8D
:10C5600041014FF4806404F132045FEA915C3FF4CE
:10C57000D8AE4FF003025FEADC0C18BF03325FEA6B
:10C58000DC0C18BF033202EBDC02C2F1200300FA1C
:10C5900003FC20FA02F001FA03FE40EA0E0021FA41
:10C5A00002F11444BDE600BF70B54FF0FF0C4CF42F
:10C5B000E06C1CEA11541DBF1CEA135594EA0C0FE1
:10C5C00095EA0C0F00F0DEF82C4481EA030621EA1C
:10C5D0004C5123EA4C5350EA013518BF52EA033557
:10C5E00041F4801143F4801338D0A0FB02CE4FF009
:10C5F0000005E1FB02E506F00042E0FB03E54FF039
:10C600000006E1FB03569CF0000F18BF4EF0010E30
:10C61000A4F1FF04B6F5007F64F5407404D25FEA2C
:10C620004E0E6D4146EB060642EAC62141EA5551DF
:10C630004FEAC52040EA5E504FEACE2EB4F1FD0C21
:10C6400088BFBCF5E06F1ED8BEF1004F08BF5FEA9F
:10C65000500E50F1000041EB045170BD06F0004651
:10C6600046EA010140EA020081EA0301B4EB5C04FE
:10C67000C2BFD4EB0C0541EA045170BD41F48011F6
:10C680004FF0000E013C00F3AB8014F1360FDEBF1B
:10C69000002001F0004170BDC4F10004203C35DAF7
:10C6A0000C341BDC04F11404C4F1200500FA05F37A
:10C6B00020FA04F001FA05F240EA020001F000421B
:10C6C00021F0004110EBD37021FA04F642EB060191
:10C6D0005EEA430E08BF20EAD37070BDC4F10C04BB
:10C6E000C4F1200500FA04F320FA05F001FA04F27F
:10C6F00040EA020001F0004110EBD37041F100016B
:10C700005EEA430E08BF20EAD37070BDC4F1200575
:10C7100000FA05F24EEA020E20FA04F301FA05F2DD
:10C7200043EA020321FA04F001F0004121FA04F285
:10C7300020EA020000EBD3705EEA430E08BF20EA55
:10C74000D37070BD94F0000F0FD101F0004640008F
:10C7500041EB010111F4801F08BF013CF7D041EA11
:10C76000060195F0000F18BF704703F00046520015
:10C7700043EB030313F4801F08BF013DF7D043EAE6
:10C780000603704794EA0C0F0CEA135518BF95EA9C
:10C790000C0F0CD050EA410618BF52EA4306D1D123
:10C7A00081EA030101F000414FF0000070BD50EA42
:10C7B000410606BF1046194652EA430619D094EACC
:10C7C0000C0F02D150EA013613D195EA0C0F05D1B6
:10C7D00052EA03361CBF104619460AD181EA03010A
:10C7E00001F0004141F0FE4141F470014FF00000C2
:10C7F00070BD41F0FE4141F4780170BD70B54FF05D
:10C80000FF0C4CF4E06C1CEA11541DBF1CEA1355DC
:10C8100094EA0C0F95EA0C0F00F0A7F8A4EB0504BE
:10C8200081EA030E52EA03354FEA013100F08880B5
:10C830004FEA03334FF0805545EA131343EA12637E
:10C840004FEA022245EA111545EA10654FEA002633
:10C850000EF000419D4208BF964244F1FD0404F5EC
:10C86000407402D25B084FEA3202B61A65EB030548
:10C870005B084FEA32024FF480104FF4002CB6EB05
:10C88000020E75EB030E22BFB61A754640EA0C0085
:10C890005B084FEA3202B6EB020E75EB030E22BFC5
:10C8A000B61A754640EA5C005B084FEA3202B6EB06
:10C8B000020E75EB030E22BFB61A754640EA9C00C5
:10C8C0005B084FEA3202B6EB020E75EB030E22BF95
:10C8D000B61A754640EADC0055EA060E18D04FEA53
:10C8E000051545EA16754FEA06164FEAC30343EAF3
:10C8F00052734FEAC2025FEA1C1CC0D111F4801FC0
:10C900000BD141EA00014FF000004FF0004CB6E7B8
:10C9100011F4801F04BF01430020B4F1FD0C88BF57
:10C92000BCF5E06F3FF6AFAEB5EB030C04BFB6EB62
:10C93000020C5FEA500C50F1000041EB045170BD55
:10C940000EF0004E4EEA113114EB5C04C2BFD4EB82
:10C950000C0541EA045170BD41F480114FF0000E06
:10C96000013C90E645EA060E8DE60CEA135594EA82
:10C970000C0F08BF95EA0C0F3FF43BAF94EA0C0F85
:10C980000AD150EA01347FF434AF95EA0C0F7FF4FA
:10C9900025AF104619462CE795EA0C0F06D152EA4E
:10C9A00003353FF4FDAE1046194622E750EA410632
:10C9B00018BF52EA43067FF4C5AE50EA41047FF443
:10C9C0000DAF52EA43057FF4EBAE12E74FF0FF3CA8
:10C9D00006E000BF4FF0010C02E000BF4FF0010C79
:10C9E0004DF804CD4FEA410C7FEA6C5C4FEA430CF2
:10C9F00018BF7FEA6C5C1BD001B050EA410C0CBF41
:10CA000052EA430C91EA030F02BF90EA020F0020A2
:10CA1000704710F1000F91EA030F58BF994208BF09
:10CA200090422CBFD8176FEAE37040F001007047C6
:10CA30004FEA410C7FEA6C5C02D150EA013C07D11D
:10CA40004FEA430C7FEA6C5CD6D152EA033CD3D068
:10CA50005DF8040B704700BF8446104662468C4662
:10CA60001946634600E000BF01B5FFF7B7FF002895
:10CA700048BF10F1000F01BD4DF808EDFFF7F4FFBE
:10CA80000CBF012000205DF808FB00BF4DF808ED49
:10CA9000FFF7EAFF34BF012000205DF808FB00BF6C
:10CAA0004DF808EDFFF7E0FF94BF012000205DF88E
:10CAB00008FB00BF4DF808EDFFF7CEFF94BF012043
:10CAC00000205DF808FB00BF4DF808EDFFF7C4FF3C
:10CAD00034BF012000205DF808FB00BF4FEA410C85
:10CAE0007FEA6C5C02D150EA013C0AD14FEA430C68
:10CAF0007FEA6C5C02D152EA033C02D14FF00000A5
:10CB000070474FF0010070474FEA410212F50012E2
:10CB100015D211D56FF47873B3EB625212D94FEA84
:10CB2000C12343F0004343EA505311F0004F23FA6E
:10CB300002F018BF404270474FF00000704750EAC3
:10CB4000013005D111F0004008BF6FF00040704780
:10CB50004FF00000704700BF4A0011D212F50012DA
:10CB600011D20DD56FF47873B3EB62520ED44FEA45
:10CB7000C12343F0004343EA505323FA02F07047C5
:10CB80004FF00000704750EA013002D14FF0FF3003
:10CB900070474FF0000070474FEA4102B2F1E043A6
:10CBA00024BFB3F5001CDCF1FE5C0DD901F0004C94
:10CBB0004FEAC0024CEA5070B2F1004F40EB8300E4
:10CBC00008BF20F00100704711F0804F21D113F110
:10CBD0003872BCBF01F00040704741F480114FEA49
:10CBE0005252C2F11802C2F1200C10FA0CF320FAD2
:10CBF00002F018BF40F001004FEAC1234FEAD323EF
:10CC000003FA0CFC40EA0C0023FA02F34FEA430358
:10CC1000CCE77FEA625307D150EA01331EBF4FF0E1
:10CC2000FE4040F44000704701F0004040F0FE40FC
:10CC300040F40000704700BF80F0004002E000BFF9
:10CC400081F0004142001FBF5FEA410392EA030FF7
:10CC50007FEA226C7FEA236C6AD04FEA1262D2EB41
:10CC60001363C1BFD218414048404140B8BF5B4246
:10CC7000192B88BF704710F0004F40F4000020F0DF
:10CC80007F4018BF404211F0004F41F4000121F0F5
:10CC90007F4118BF494292EA030F3FD0A2F101023F
:10CCA00041FA03FC10EB0C00C3F1200301FA03F17D
:10CCB00000F0004302D5494260EB4000B0F5000FA0
:10CCC00013D3B0F1807F06D340084FEA310102F15F
:10CCD0000102FE2A51D2B1F1004F40EBC25008BF11
:10CCE00020F0010040EA03007047490040EB0000DB
:10CCF000013A28BFB0F5000FEDD2B0FA80FCACF1DC
:10CD0000080CB2EB0C0200FA0CF0AABF00EBC25008
:10CD100052421843BCBFD0401843704792F0000FF6
:10CD200081F4000106BF80F400000132013BB5E749
:10CD30004FEA41037FEA226C18BF7FEA236C21D0BF
:10CD400092EA030F04D092F0000F08BF0846704724
:10CD500090EA010F1CBF0020704712F07F4F04D1F2
:10CD6000400028BF40F00040704712F100723CBF05
:10CD700000F50000704700F0004343F0FE4040F42F
:10CD8000000070477FEA226216BF08467FEA2363ED
:10CD90000146420206BF5FEA412390EA010F40F4D8
:10CDA000800070474FF0000304E000BF10F0004324
:10CDB00048BF40425FEA000C08BF704743F096430B
:10CDC00001464FF000001CE050EA010208BF704726
:10CDD0004FF000030AE000BF50EA010208BF7047AD
:10CDE00011F0004302D5404261EB41015FEA010CC2
:10CDF00002BF84460146002043F0B64308BFA3F1BA
:10CE00008053A3F50003BCFA8CF2083AA3EBC2539B
:10CE100010DB01FA02FC634400FA02FCC2F12002BA
:10CE2000BCF1004F20FA02F243EB020008BF20F0F1
:10CE30000100704702F1200201FA02FCC2F1200257
:10CE400050EA4C0021FA02F243EB020008BF20EA4C
:10CE5000DC7070477BB972B90029BEBF00204FF06B
:10CE6000004106E008BF00281CBF6FF000414FF0F2
:10CE7000FF3000F007BAADF1080C6DE904CE0029CF
:10CE800009DB002B1ADB00F095F8DDF804E0DDE9A2
:10CE9000022304B07047404261EB4101002B1BDBD1
:10CEA00000F088F8DDF804E0DDE9022304B0404238
:10CEB00061EB4101524263EB43037047524263EB23
:10CEC000430300F077F8DDF804E0DDE9022304B065
:10CED000404261EB41017047524263EB430300F073
:10CEE00069F8DDF804E0DDE9022304B0524263EBA7
:10CEF0004303704753B94AB9002908BF00281CBF33
:10CF00004FF0FF314FF0FF3000F0BCB9ADF1080C2D
:10CF10006DE904CE00F04EF8DDF804E0DDE902230F
:10CF200004B07047430803F05533C01A830803F078
:10CF3000333300F03330184400EB101000F00F30A2
:10CF400000EB002000EB0040000E704707EE900A57
:10CF5000F5EEC07AF1EE10FA01D400F00BB8F1EE64
:10CF6000677A08B517EE900A00F004F8404261EBCA
:10CF7000410108BDD0B5FFF7BFFA0C4B00220646B1
:10CF80000F46FFF711FBFFF7E7FD0446FFF792FAA4
:10CF9000074B0022FFF708FB02460B463046394696
:10CFA000FFF74AF9FFF7D8FD2146D0BD0000F03D5C
:10CFB0000000F0412DE9F047089D04468E46002B05
:10CFC0004DD18A42944669D9B2FA82F252B101FA3D
:10CFD00002F3C2F1200120FA01F10CFA02FC41EA4D
:10CFE000030E94404FEA1C48210CBEFBF8F61FFAD2
:10CFF0008CF708FB16E341EA034306FB07F199426D
:10D000000AD91CEB030306F1FF3080F01F8199421F
:10D0100040F21C81023E63445B1AA4B2B3FBF8F0F9
:10D0200008FB103344EA034400FB07F7A7420AD980
:10D030001CEB040400F1FF3380F00A81A74240F2A8
:10D0400007816444023840EA0640E41B00261DB113
:10D05000D4400023C5E900433146BDE8F0878B4248
:10D0600009D9002D00F0EF800026C5E90001304607
:10D070003146BDE8F087B3FA83F6002E4AD18B42E1
:10D0800002D3824200F2F980841A61EB030301208B
:10D090009E46002DE0D0C5E9004EDDE702B9FFDE77
:10D0A000B2FA82F2002A40F09280A1EB0C014FEA22
:10D0B0001C471FFA8CFE0126200CB1FBF7F307FB7F
:10D0C000131140EA01410EFB03F0884208D91CEB22
:10D0D000010103F1FF3802D2884200F2CB804346BF
:10D0E000091AA4B2B1FBF7F007FB101144EA01449E
:10D0F0000EFB00FEA64508D91CEB040400F1FF312D
:10D1000002D2A64500F2BB800846A4EB0E0440EA1A
:10D1100003409CE7C6F12007B34022FA07FC4CEA23
:10D12000030C20FA07F401FA06F31C43F9404FEA16
:10D130001C4900FA06F3B1FBF9F8200C1FFA8CFE2B
:10D1400009FB181140EA014108FB0EF0884202FA7F
:10D1500006F20BD91CEB010108F1FF3A80F0888040
:10D16000884240F28580A8F102086144091AA4B2FD
:10D17000B1FBF9F009FB101144EA014100FB0EFE7E
:10D180008E4508D91CEB010100F1FF346CD28E45AD
:10D190006AD90238614440EA0840A0FB0294A1EB3E
:10D1A0000E01A142C846A64656D353D05DB1B3EB9B
:10D1B000080261EB0E0101FA07F722FA06F3F140CB
:10D1C0001F43C5E9007100263146BDE8F087C2F172
:10D1D0002003D8400CFA02FC21FA03F391400143EA
:10D1E0004FEA1C471FFA8CFEB3FBF7F007FB103623
:10D1F0000B0C43EA064300FB0EF69E4204FA02F4CF
:10D2000008D91CEB030300F1FF382FD29E422DD921
:10D21000023863449B1B89B2B3FBF7F607FB163356
:10D2200041EA034106FB0EF38B4208D91CEB0101D6
:10D2300006F1FF3816D28B4214D9023E6144C91A56
:10D2400046EA004638E72E46284605E70646E3E666
:10D250001846F8E64B45A9D2B9EB020864EB0C0E70
:10D260000138A3E74646EAE7204694E74046D1E77F
:10D27000D0467BE7023B614432E7304609E764442D
:10D28000023842E7704700BF02E000F000F8FEE716
:10D2900072B6374880F30888364880F309883648E4
:10D2A0003649086040F20000CCF200004EF63471BE
:10D2B000CEF200010860BFF34F8FBFF36F8F40F2D3
:10D2C0000000C0F2F0004EF68851CEF20001086076
:10D2D000BFF34F8FBFF36F8F4FF00000E1EE100AE6
:10D2E0004EF63C71CEF200010860062080F31488EF
:10D2F000BFF36F8F74F0F8FA75F042FA4FF05530C3
:10D300001F491B4A91423CBF41F8040BFAE71D49F3
:10D31000184A91423CBF41F8040BFAE71A491B4AEC
:10D320001B4B9A423EBF51F8040B42F8040BF8E73E
:10D3300000201849184A91423CBF41F8040BFAE713
:10D3400074F0D6FA75F070FA144C154DAC4203DA4D
:10D3500054F8041B8847F9E701F0D2F9114C124D3B
:10D36000AC4203DA54F8041B8847F9E774F0BEBAFC
:10D37000000600200022002000C0000808ED00E0A8
:10D380000000002000060020680E0A08002200208D
:10D39000C8250020C825002098200120E0C10008F1
:10D3A00030C2000830C2000830C200082DE9F04F3A
:10D3B0002DED108AC1F80CD0C3689D46BDEC108AD3
:10D3C000BDE8F08F002383F311882846A047002092
:10D3D00073F00CFAFEE773F069F800DFFEE7000077
:10D3E00001F0FF01102A2BDB10F0070F08D010F816
:10D3F000013B013A8B422DD010F0070F42B3F6D11A
:10D40000F0B441EA012141EA014122F007047FF032
:10D4100000070023F0E80256083C85EA010586EA89
:10D42000010685FA47F5A3FA87F586FA47F6A5FAC5
:10D4300087F68EB9EED1F0BC01F0FF0102F00702D1
:10D4400032B110F8013B013A83EA010313B1F8D17C
:10D450000020704701387047002D06BF354603385D
:10D46000073815F0010F07D1013015F4807F02BF96
:10D47000013015F4C03F0130F0BC0138704700BFE7
:10D4800010F8012B11F8013B012A28BF9A42F7D06E
:10D49000D01A7047034613F8012B002AFBD1181A43
:10D4A0000138704738B50022002304460D46FFF7C7
:10D4B000EDFA28B920462946BDE8384000F00AB800
:10D4C000204605F1004100F005F8404261EB4101C2
:10D4D00038BD00BFD0B50C4B002206460F46FFF703
:10D4E00063F8FFF739FB0446FEF7E4FF074B002221
:10D4F000FFF75AF802460B4630463946FEF79CFEC7
:10D50000FFF72AFB2146D0BD0000F03D0000F041AE
:10D51000002070477047000070470000704700000F
:10D52000002070470020704700207047012070479E
:10D5300000207047704700000020704700207047AF
:10D5400070470000704700000020704700207047BF
:10D5500070B5154ED6F8380203681B689847042842
:10D560001ADC01281DDC002814BF012441240F4BC4
:10D570001D68E86A0368DB69984701280AD0D6F875
:10D5800038220B4B9A4205D0EB6A93F89C300BB1D2
:10D5900044F08004204670BD0A2814BF01241924D9
:10D5A000E5E71924E3E700BFD0550020CC25002093
:10D5B00010580020044BD3F8380203F51072904243
:10D5C00014BF042002207047D0550020014B93F86F
:10D5D00048017047D04500207047000038B5C57835
:10D5E0000B461C2D044628BF1C251C220021184672
:10D5F00078F0FEF82A4604F10C01BDE8384078F0D6
:10D60000ADB8000038B5C5780B46102D044628BFCC
:10D61000102510220021184678F0EAF82A4604F175
:10D620000C01BDE8384078F099B8000008B53EF02C
:10D63000B5F930B9034A92F8CC3243F0040382F8CA
:10D64000CC3208BDD055002038B591ED000AF7EE78
:10D65000000A0D4618F082FB20B10B4801F0DCFEF9
:10D66000002038BDD5ED007A9FED087AF0EEE77A1C
:10D67000F4EEC77AF1EE10FA03D5034801F0DEFEAE
:10D68000EEE70320EDE700BFD025002000000034C6
:10D6900010B5044608F05CFA204610BD13B58B8B1C
:10D6A000B72B0C4607D0B3F5967F21D002B0BDE86A
:10D6B000104041F0F1BD124912481E2201F0E6FE71
:10D6C000D4ED017A94ED007A0D48FCEEE77ABCEED9
:10D6D000C77A17EE903A8DED017A9DF804109AB250
:10D6E00001F074FB002814BF0020042002B010BD1C
:10D6F00004480549022201F0C9FE0020F6E700BFF8
:10D7000038580020D02500200C58002000B51F4AB2
:10D71000DFED1F6AD2EDB17A92EDB07AD2F8B41291
:10D72000007CA2F580538BB093F96A310491002BF1
:10D7300018BFB0EE677AD2EDAB7A8DED057AFDEECB
:10D74000E77A3E2117EE903AD2EDAC7AF4EEE67A23
:10D75000F1EE10FA58BFF0EE667AFCEEE77A1BB2F3
:10D76000ADF82030ADF8223017EE903A0022039247
:10D7700006920792ADF82430B7221A23CDE9003281
:10D7800003AA3BF08FFB0BB05DF804FBD0550020E3
:10D7900000FF7F4770B5154C94F8D2228AB022B9A9
:10D7A0000AB0BDE870403CF049BE057C56F07EFDF5
:10D7B000D4E98C61D4F82C32A4F50054CDE90513DA
:10D7C000B4F86824ADF826200023CDE90733ADF87E
:10D7D000243068221C23CDE90306CDE90032212143
:10D7E00003AA28463BF05EFB0AB070BDD05500206E
:10D7F000F0B53B4CB4F88C31DE078DB0054637D51B
:10D80000D4F84032089302238DF82430D4F85032F3
:10D81000D4F84402CDF82530D4F84C32D4F838127C
:10D82000D4F83C220590CDF8293062202123D4F889
:10D830003062D4F82C720691CDE90030C221192350
:10D84000287C079203AA049603973BF02BFB287CC5
:10D850003BF0BEFA0646287C3CF0BEF900F12103FD
:10D860009E4205D2287C0DB0BDE8F0403AF02CBDB8
:10D87000B4F88C31990731D5D4F8283308930323B1
:10D880008DF82430D4F83833D4F82423CDF825305B
:10D89000D4F83433D4F82C03D4F820130792CDF8FD
:10D8A000293062222123D4F81863D4F81473059028
:10D8B000CDE90032287C0691192303AAC2210397DF
:10D8C00004963BF0EFFA287C3BF082FA0446287C71
:10D8D0003CF082F900F121039C42C3D30DB0F0BDAE
:10D8E000D045002005207047024BD3F8380203686A
:10D8F0001B681847D055002030B5CD788BB0272D48
:10D9000028BF27250C4627220021684677F070FFA4
:10D910002A4604F10C01684677F020FF1A4BD3F831
:10D92000381203F5127291422BD1DDED057A9FED8D
:10D93000177AF0EEE77AF4EEC77AF1EE10FA20D516
:10D940009DF8262002F0410141291AD1110618D470
:10D9500002F01801182914D00199C3F84C1282F072
:10D9600004020299C3F85012C2F380020399C3F86B
:10D97000541283F85C220499079AC3F85812C3F82A
:10D9800060220BB030BD00BFD05500200000003435
:10D9900030B5194D95F8D13285B00C464BBBCA78DD
:10D9A0008DF80C30092A28BF09220C3101A8CDE9D5
:10D9B000013377F0D3FE9DF808305A1F012A18D999
:10D9C00003F0F703122B14D0A5F58053B3F94A21C5
:10D9D00012B9E279A3F84A21227AE179074800F0E6
:10D9E000B1F9227AE179054800F0E4F9012385F8DC
:10D9F000D13205B030BD00BFD0550020B05000205E
:10DA0000F0B51B4BB3F94A3189B005460E461446B2
:10DA10003BB1D779BB4204D009B0BDE8F0403FF03C
:10DA2000C5BFA27A637A43EA0223E27A43EA024359
:10DA30001D2B13D0212B08D01BB921462846FFF7F8
:10DA4000A7FF224631462846E6E701A92046FFF710
:10DA5000C5FD084801A901F09FFFF2E701A9204692
:10DA6000FFF7D0FD034801A901F0ECFFE9E700BF93
:10DA7000D0450020D025002013B5CA78072A4FF0E2
:10DA80000003044628BF07220C3168460093CDF8F6
:10DA9000033077F063FEBDF900304BB901231C2140
:10DAA000204684F80F3302B0BDE8104041F0ACBB13
:10DAB00002B010BD30B5CD7889B01E2D28BF1E250F
:10DAC0000C461E220021684677F092FE2A4604F199
:10DAD0000C01684677F042FE0248694601F0FEFFFD
:10DAE00009B030BDD025002000B589B0084601A995
:10DAF000FFF774FD034801A901F04EFF09B05DF87E
:10DB000004FB00BFD02500201FB508466946FFF77B
:10DB100079FD0348694601F095FF05B05DF804FB07
:10DB2000D02500202DE9F041CC7894B0262C28BFD8
:10DB3000262488462622002107460AA877F058FEA8
:10DB400002AD224608F10C010AA877F007FE28462C
:10DB500007F05AFD9DF84A30022B06AC03D0032B88
:10DB600044D0002B66D1DFED357ADDED106A9FEDF4
:10DB7000346A9DED0F7A66EEA76ADDED0E7A27EE28
:10DB8000067A67EE867A0023FDEEE66ABDEEC77A76
:10DB9000FDEEE77A17EE102A17EE901A0093204652
:10DBA00016EE903A07F050FD94E80F0085E80F005C
:10DBB00097F80F3363BB012698F8083098F80720D0
:10DBC0008DF8193000238DF818208DF81B3099221C
:10DBD0000423CDE90032387C8DF81A6003232246F5
:10DBE0002F213BF05FF914B0BDE8F081DFED137A2F
:10DBF000DDED106A9FED126A9DED0F7A66EEA76A61
:10DC0000DDED0E7A27EE067A67EE867A0123BBE712
:10DC1000BDF8446086B90B483246294601F0D4FB72
:10DC20000028C8D0084A062138463DF04BFB87F84B
:10DC30000F63C1E70226BFE70026BDE70000C84228
:10DC40008096184BD0250020609A080838B58A7A4B
:10DC50004B7A43EA0223CA7A43EA0243272B05465A
:10DC60000C460CD81C2B10D91D3B0A2B0DD8DFE815
:10DC700003F01E0C0C0C1B0C0C0C0C121500452B8D
:10DC80000FD0522B01D1FFF737FE21462846BDE8C1
:10DC9000384040F099B9FFF7EFFEF6E7FFF742FF93
:10DCA000F3E7FFF707FFF0E7FFF71EFFEDE7FFF7EA
:10DCB0002BFFEAE700207047C8207047012070471B
:10DCC00000207047002070470120704790F8903086
:10DCD0008B4286BF00EB8100D0F894000020704793
:10DCE00090F890308B4286BF00EB8100D0F8940012
:10DCF00000207047014B93F846017047D045002043
:10DD0000036A43F4E0530362436A43F4E05343621B
:10DD1000836A43F4E05383627047000013B54FF405
:10DD20004470CDE9002107F00BFF044628B1DDE97E
:10DD3000002140F0ADFE024B2360204602B010BD32
:10DD4000FC9B08082DE9F04FDFF8649085B006468B
:10DD50000F46904600254FF4837A96F89030ECB247
:10DD6000A34222D920463BF033F8834620463BF0BD
:10DD700033FF031D9B4514D399F96B31ADF808307F
:10DD800094220623CDE90032422102AA20468DF8D2
:10DD90000A708DF80B80ADF80CA03BF083F80135CC
:10DDA000DBE720463AF090FAF9E705B0BDE8F08FDE
:10DDB000D04500202DE9F04FDFF8649085B006468D
:10DDC0000F469046002540F2011A96F89030ECB2CA
:10DDD000A34222D920463AF0FBFF834620463BF07F
:10DDE000FBFE031D9B4514D399F96B31ADF8083048
:10DDF00094220623CDE90032422102AA20468DF862
:10DE00000A708DF80B80ADF80CA03BF04BF8013593
:10DE1000DBE720463AF058FAF9E705B0BDE8F08FA5
:10DE2000D04500201FB500F54053002100F5935068
:10DE3000D3F8B4220191D3F8AC32029201A9083090
:10DE4000039301F0ABFF03F077FB03F041F905B05A
:10DE50005DF804FB70B586B006461322002101A8C8
:10DE600010EE105A10EE904A77F0C2FCA3238DF802
:10DE7000043095238DF8053056F020FA1322CDF8A2
:10DE80000700CDF80B1006F57C6001A9CDF80F5006
:10DE9000CDF8134037F0ECF906B070BD2DE9F04134
:10DEA0008AB00446884617460021232201A8109D07
:10DEB0001E4677F09DFCA3238DF8043095238DF842
:10DEC000053001238DF8063056F0F8F92B68CDF8AF
:10DED0001B306B68CDF80700CDF80B10CDF81F3064
:10DEE0002322AB68CDF80F8001A904F57C60CDF842
:10DEF0001370CDF81760CDF8233037F0B9F90AB0B8
:10DF0000BDE8F0819720704710B500F540530446F6
:10DF1000D3F8380203681B6898471A22C1B204F587
:10DF20007C6037F065FB04F59070BDE810400FF0A1
:10DF3000B9BF000037B500F5055104460122043190
:10DF400035F072FF012504F5FF51104A00950023BA
:10DF50001031DA2033F086FD0D4A0095002304F5D8
:10DF60007C61FD2033F07EFD0A4B1A68D20705D490
:10DF7000094A1D6004F58C540C34146006480121D4
:10DF800003B0BDE8304033F0BFBD00BF64CD090829
:10DF900038520908C82500200022002000207047C0
:10DFA000002070470069C0F3401070470F299DBFE3
:10DFB000302303FB010050300020704700207047E1
:10DFC0000120704770470000036800221B68184753
:10DFD00000207047002070470020704700207047E5
:10DFE00000207047002070470020704700207047D5
:10DFF00000207047002070477047000010207047D5
:10E0000000207047704700000320704701207047D0
:10E0100070470000012070470020704770470000E3
:10E0200000F50650143070470048704730C00808AB
:10E0300008B500F54050D0F8380203681B689847CF
:10E04000C0B208BD034808600F2111704FF0FF32C5
:10E050001A607047C0D7080800207047002070473A
:10E060007047000015F01ABF37F068BA41F0FCBBEA
:10E070003FF0EEBD05F0CCBB06F062BA00F0D4BEB6
:10E0800000F0CEBE00F0ECBE01F024BC00F0BABE41
:10E0900000F0C0BE00F02ABF70B51F4B036000F552
:10E0A00000530446D3F8900C1C4AC3F8E02A08B188
:10E0B00007F052FD1A4B236004F5805393F82C2E81
:10E0C00042B9D3F8285E2DB1284614F0D1FD284678
:10E0D00007F03EFD04F58B50103053F00DFC04F5B5
:10E0E0008350183043F092FC04F6C44504F66446AD
:10E0F000B54204D0183D284614F028FAF8E7094B39
:10E10000C4F8983804F6941039F04AF804F5106011
:10E1100039F046F8204670BDF4D80808446A09086A
:10E120009C4B0908FC21090838B5484B044640F8C7
:10E13000043B43F0E3FD04F1100006F027FB04F17B
:10E14000680035F0E3F804F590700FF08DFA04F5EF
:10E15000866005F0CDF904F2545007F0FFFC04F698
:10E16000980015F03FFD04F5446043F04FFD04F5C1
:10E17000516034F0EDFD04F57C6036F0C1FF04F52C
:10E180008350183043F02AFC04F58550143006F013
:10E19000EFFB04F58B50103053F09AFB04F58C50D4
:10E1A0000C3035F0BFFB04F58F5044F051FF04F5FF
:10E1B00080530025264A83F8045204F5905004F554
:10E1C000905304331430136030F064FF04F593501F
:10E1D0002946083001F0D8FE04F5C55018304CF03F
:10E1E000C5FA04F5E5501C3050F0D0FB04F5EE50B4
:10E1F000143052F0C7FC04F5F150183053F0FCF81D
:10E2000004F5F450103001F01FFD04F5FF501030FC
:10E210004CF0D0FE04F50150083049F0FBFD04F548
:10E22000005304F5045083F804510A4D1C3053F098
:10E230009FFE2B6813B1084856F006F820460749A0
:10E2400033F088FE2C60204638BD00BF9C4B090887
:10E25000CC630020485B0020C0D50808D44A0908D8
:10E2600010B59FED225A9FED224A9FED222ADFED45
:10E27000221A9FED221A9FED220A86B00446F0EE84
:10E28000453AB0EE453AF0EE452AF0EE450AF7EE93
:10E29000004A54308DED054A8DED042ACDED031A68
:10E2A0008DED021A8DED015A8DED000A4BF0FEFF47
:10E2B0009DED015A9DED054A9DED042ADDED031A01
:10E2C0009DED021A9DED000AF7EE004AF0EE453A88
:10E2D000B0EE453AF0EE452AF0EE450A04F59E70A0
:10E2E0004BF0E4FF204606B010BD00BF0000000068
:10E2F000CDCCCC3D00007A450AD7A33CCDCC4C3DDB
:10E30000CDCC4C3EF0B500F50055224BB5F846217A
:10E310001A7087B0044643F0D7F942F08DFF2046CB
:10E3200001F00CFC04F5805393F8E42412F0010290
:10E3300010D102A8019207F067F904F5935002A9E1
:10E34000083002F0DBFE28B12368019ADB6C02A9D9
:10E3500020469847104E3368DB6A93F89C7037B1BB
:10E3600095F806311BB955F0A1FFC5F808013368CF
:10E3700085F80671DB6A93F89C20084B5A7135F0DA
:10E3800037FA34F089FF04F50A5007B0BDE8F040D1
:10E390004BF0DCBF05230020CC250020755A00205F
:10E3A000FFF7B0BF10B50821044601F0ABF918B172
:10E3B00017F0D4F815F0E2FA0121204601F0A2F995
:10E3C00010B12046FFF72EFD0421204601F09AF9F6
:10E3D00018B104F57C6036F009FB1021204601F0ED
:10E3E00091F928B104F57C60BDE8104036F098BB87
:10E3F00010BD0000FFF7D6BF102925D8DFE801F0D7
:10E40000090D11191524242424241D242424242432
:10E41000210000F549500430704700F549502C3078
:10E42000704700F549502430704700F549500830D6
:10E43000704700F549502830704700F548503C308F
:10E44000704700F5495070470020704708B54CF000
:10E45000B5FE044B1B68DB6A93F89C10BDE80840CE
:10E460004CF088BECC250020FFF7F0BF2DE9FF411E
:10E470000446FFF759FE884B236004F5055004F568
:10E4800000550430FFF7ECFE002304F50D50C5F8ED
:10E4900068332C3041F006FCDFF860827F4BC5F812
:10E4A0006C3342F2BC3642F2BC67A01941F088FDE1
:10E4B00044F806803036BE42F7D1A01942F0E4FF9E
:10E4C00004F52B50043039F0ADF804F52B50103022
:10E4D00039F0A8F804F52B570023A5F8DC3A2037CB
:10E4E0006F4BC5F8E03A07F1080055F089F804F5DC
:10E4F0002C5604F52D580C3608F1300830461436E9
:10E500003DF0D8FD4645F9D10723C5F8943C0023DA
:10E51000A5F8983C4FF4CB7007F018FBC5F8900CA9
:10E5200004F532501C3055F06BF804F533502030B0
:10E5300055F066F85B4B1A6802B91F605A4BC5F874
:10E54000E03A0026594B03930294009604AB04F57D
:10E55000335013E90C0040213C3005F077FC04F502
:10E56000485004F54055283007F04EF804F549535B
:10E57000C5F838324E4BC5F83C324E4BC5F84032E8
:10E580004D4BC5F844324D4BC5F848324FF07E53E1
:10E59000C5F84C324A4BC5F8643204F54958494B2A
:10E5A000C5F868320027484BC5F86C3208F13008CE
:10E5B000C5F85872C5F85472C5F8507208F10400D5
:10E5C00007F022F808F1140007F01EF83F4B40480E
:10E5D000C5F89C7204F54B52C5F8A072C5F8A47238
:10E5E0001860103233464FF6FF774FF0140C9EB28E
:10E5F0000CFB06010133097C0029F8D1354B364963
:10E600001E800B6813B1354855F01EFE85F8D132D7
:10E6100004F54B50012385F8D23214300A6053F0D0
:10E6200055FD2F4BC5F8D4322E4BC5F82843C5E90C
:10E63000CB342D4B04F54D50C5E9CD342B4BC5F8EB
:10E640003C33103006F0E0FF04F54D502C3006F05E
:10E65000DBFF04F54E50083006F0D6FF04F54C56AB
:10E66000234BC5F89C33A5F8A07306F1A40006F06F
:10E67000CBFF4FF0FF330C36C5F800341D4B1E495D
:10E680001E60304633F066FC2046A5F84873A5F8B6
:10E69000647304B0BDE8F081F4D80808A4D5080874
:10E6A000446A0908645E0020D09C080895E00008D0
:10E6B00068D908084CD60808B0D908089CD90808B9
:10E6C000C4D9080860D6080874D60808105B002072
:10E6D000DCCF08080C5B0020CC5A0020D4D50808F9
:10E6E0000CD6080859E000085DE0000861E0000869
:10E6F0000000FFFF445A0020302E0908F8D5080812
:10E7000038B5054B1C6823680A461D68034B014653
:10E710002046A847002038BDCC250020D025002069
:10E7200010B555F0E3F9064C064B18602046FFF78C
:10E730009DFE2046044A0549BDE8104074F02ABBFE
:10E74000D0250020CC25002064B8002099E00008E6
:10E7500038B52DED028B0D46F0EE608AB0EE408AA2
:10E76000144602F0E9FE90ED937AD0ED957A67EECB
:10E77000877A90ED927A67EEA87AE7EE087AC5ED8F
:10E78000007AD0ED920AD0ED937A90ED957A67EE0B
:10E79000A07A67EEA80AE7EE480ABDEC028BC4ED4A
:10E7A000000A38BD30B52DED068B83B0F0EE409AEF
:10E7B000B0EE60AA0D46044602F0BEFED0ED7F7AB0
:10E7C000D0F80002B8EEE79A17F094FB07EE900A33
:10E7D000F8EEE78A79EEC9AA3AEE688AFDEEEAAA6F
:10E7E000B0EE480A17F068FBBDEEC00A5DB110EE4E
:10E7F000103ADFED190A002BCCBF38EE608A38EEF4
:10E80000208ABDEEC80AF8EEC00A01AAB8EEEA0AEC
:10E8100069462046FFF79CFFDFED107A104B009A07
:10E82000C3F8B82269EEA79A019AC3F8BC2229EE70
:10E83000279A2AEE27AA68EEA78AA3F58053C3ED8C
:10E840008B9A83ED8C9A83EDC5AAC3EDC68A03B07B
:10E85000BDEC068B30BD00BF00A00C470AD7233C9F
:10E86000D055002038B52DED028B0D46B0EE408A14
:10E87000F0EE608A144602F05FFED0ED937A9FEDD1
:10E88000147AF0EEE77AF4EEC77AF1EE10FA1DD4BE
:10E89000D0ED957A90ED927A67EEE87AE8EE077A15
:10E8A000C5ED007A90ED937AD0ED957A90ED926A6D
:10E8B000C7EE876A0120C6EE077A67EEA80AE6EE81
:10E8C000880AC4ED000ABDEC028B38BD0020FAE7CF
:10E8D0000000003430B55F4C2DED068BB4F9843167
:10E8E000DFED5D8A5B4285B008EE103A054604F61E
:10E8F000C42038F09BFEB8EEC88A90ED00AAB4F9A7
:10E90000843128EE288AF6EE009A98EE29AA04F6B9
:10E91000C42008EE103A38F089FEB8EEC88A90EDAF
:10E92000009AB4F9883128EE288A04F52D6098EE13
:10E93000299A08EE103A38F079FEB4F98A31D0ED10
:10E94000009A04F52D600AEE903A38F06FFEB8EEAA
:10E95000C88AF8EEEAAAD8EE289A6A4602A990ED8B
:10E96000008A8DED00AA9AEEA88A2846F0EE4A0A9F
:10E97000B0EE690A8DED038A8DED019ACDED029A14
:10E98000FFF770FF01AA03A9F0EE490AB0EE480AAA
:10E990002846FFF767FF02F0CFFDD0F8000217F01E
:10E9A000A9FA04F58053D4ED5F7A93EDAB0A30EE0B
:10E9B000270A08EE100A20EE280A17F07DFAB8EEB2
:10E9C000C88A30EE480A17F077FADFED247A9DED19
:10E9D000007AB5EEC00AF1EE10FAACBF70EE676ACD
:10E9E000F0EE406AB4EEE67AB4BF70EE277AF0EE4D
:10E9F000407AF1EE10FA2ADD9DED016AB4EEE76A85
:10EA0000F1EE10FA23D5B5EEC00AF1EE10FA08DDEA
:10EA100077EE665A37EEC65AF4EEC55AF1EE10FAA2
:10EA200013D4B5EEC00AF1EE10FA10D537EE667ABF
:10EA300077EEC67AB4EEE77AF1EE10FACCBF012099
:10EA4000002005B0BDEC068B30BD0120F9E70020A9
:10EA5000F7E700BFD04500200000C84200A00C47E7
:10EA600070B5314C2DED028BA4F58055D5ED5F7A54
:10EA700094EDAB0ADFED2D8A30EE270A84B020EE4C
:10EA8000280A064617F018FAB5F98A31D5ED607AEA
:10EA900001EE103AB5F98831B0EE408A00EE903AB6
:10EAA00094EDAD0AB8EEC11A30EE270AF8EEE00A8E
:10EAB0000C2017F055FA20EE280A30468DED010A99
:10EAC000FFF708FF9DED010A0146F0EE480A3046C7
:10EAD000FFF768FE9DED010A03AA02A9F0EE480ABD
:10EAE0003046FFF735FEB5F98631002B0DDD07EE18
:10EAF000903A94EDAC7AF8EEE77AB4EEE77AF1EE7C
:10EB000010FA02DA94F870324BB99DED020A084807
:10EB100000F00CFB9DED030A054800F0E3FB04B098
:10EB2000BDEC028B70BD00BFD05500200000C84274
:10EB3000D025002038B5484C94F8CC3213F00101B0
:10EB4000054643D1A4F580529FED447AB2F958218D
:10EB500094EDAB0A07EE902AF8EEE77A13F0100F67
:10EB600067EE877AF7EE006ABFEE007A08BFB0EE74
:10EB7000667AA7EE270AC3F30012DFED397A84ED37
:10EB8000AB0AB5EEC00AF1EE10FA0AD51AB161F37C
:10EB9000041384F8CC32B4EEE70AF1EE10FA06DC86
:10EBA0000BE0B4EEE70AF1EE10FA06DD2AB994F8AC
:10EBB000CC3243F0100384F8CC329FED291ADFEDFC
:10EBC000290A2C2017F0CCF984EDAB0A94F8CC324A
:10EBD0009807C3F340012ED4234A9FED207AB2F95F
:10EBE0005A0107EE900AB2F98801B2F98A21F8EECB
:10EBF000E77A01EE102A00EE900A1A0767EE877A8C
:10EC0000F8EEE00A94EDAD7AB8EEC11A18D577EEB9
:10EC1000677AF4EEE07AF1EE10FAC4EDAD7A03D53E
:10EC200061F3C30384F8CC3294EDAD0A3C2017F0B5
:10EC300097F984EDAD0A2846BDE83840FFF710BFCC
:10EC400077EE877AF4EEC17AF1EE10FAC4EDAD7A80
:10EC5000EADD43F00803E5E7D05500200AD7A33CDE
:10EC60000000B44300000000D04500200A20704797
:10EC700001207047094B93F87012024609B1FFF763
:10EC8000EFBE93F8D11229B9A3F5805393F89031D0
:10EC9000DB0702D51046FFF74DBF7047D055002067
:10ECA000042070470120704730B52DED028B8BB0EA
:10ECB000044655F0FBFA07AB054606AA05A9201D38
:10ECC00018F04AFE274A9FED288A136841F28831DE
:10ECD000EB1A8B421CD915603FF0BCFEDDED067AC5
:10ECE00067EE887A054617EE900AFDF705FCDDED24
:10ECF000077A67EE887ACDE9020117EE900AFDF7F0
:10ED0000FBFB1A4ACDE900010621284639F0D2F86A
:10ED1000DDED067ADDED070A9FED150A60EE880A43
:10ED200027EE888A60EE800A204628EE000A00213D
:10ED3000FFF738FDDDED070A9DED060A09AA08A9CF
:10ED40002046FFF705FD9DED080A0A4800F0EEF9A0
:10ED50009DED090A074800F0C5FA0BB0BDEC028B27
:10ED600030BD00BFD8590020E02E654274D9080894
:10ED70000000C842D02500200020704701207047C5
:10ED8000024B014618680268126810476C5E00204A
:10ED900008B50020FFF7F4FFC188472042F000FBD0
:10EDA000472042F0C9F90120FFF7EAFFC188482057
:10EDB00042F0F6FABDE80840482042F0BDB9000034
:10EDC0000220704701207047FFF7B4BE08B50B461C
:10EDD000013BDBB2012B114611D85BB9472042F051
:10EDE000DFFA472042F0A8F942F09EFB42F084F897
:10EDF000012008BD482042F0D3FA4820F2E7002065
:10EE0000F7E7000008B541F0A7F8BDE8084040F07A
:10EE100083BF000000F593500021083002F012BBC0
:10EE200000F2545007F024BB10B5044607F010FC64
:10EE300090F921308BB190F8403373B194F9783563
:10EE40005BB1064B1B68DB6A93F89C302BB904F26C
:10EE50005450BDE8104007F023B910BDCC25002068
:10EE600070B5044600F590700FF074FF94F8E43329
:10EE70001C4904EB0312D2F894010A68824210D0B4
:10EE8000B02202FB034294F8285492F8C12145B9FC
:10EE9000022A06D9144E08603278012A02D9013AB2
:10EEA000327070BDFDD104F54055D5F830222AB935
:10EEB000D5F8342212B905233370F2E7B02202FBF1
:10EEC000034303F5E6730FCB05F50A7585E80F00DC
:10EED000236804F54851DB6C00222831204698470E
:10EEE0000023E9E7DC5900200C22002070470000D5
:10EEF00037B5044642F0E8FB42F09EF904F50055B0
:10EF00004721002042F09AFA4821012042F096FA67
:10EF1000B5F8841101EB810101EB8101490089B24F
:10EF2000472042F0F3F8B5F98831B5F98A110F4D51
:10EF3000C91A01EB810101EB8101490089B2482026
:10EF400042F0E4F842F0F0FA41F0D6FF04F52B501D
:10EF500001A90430019538F0FBFB04F52B5001A901
:10EF60001030019538F0F4FB03B030BDCDCCCC3D72
:10EF7000F0B52DED028B00F5005785B0B7F888216C
:10EF8000B7F88A3104466425482012FB05F613FBC6
:10EF900005F542F0ABF804F5405304F5065018307F
:10EFA000B0EE408ADFED230A93EDAE0A0190002116
:10EFB0004BF036FB07EE906A38EE000AF8EEE77A7F
:10EFC0000198B4EEE70AF1EE10FA25D98DED020AA8
:10EFD00007EE905A9DED027AF8EEE77AF4EEC77AE2
:10EFE000F1EE10FA03D8CDED027A4BF00DFA48207D
:10EFF0009DED020A42F066F897F8DD3A04F52B50D1
:10F00000103083B10C4B039303AA02A938F0A4FB80
:10F0100005B0BDEC028BF0BD0190CDED027A4BF056
:10F02000F3F90198D4E702A938F002FB012387F82D
:10F03000DD3AEDE70AD7A33C0AD7A33C00F54053DD
:10F0400000F50050D0ED5C7A90ED5E6A93EDAE7AFB
:10F0500067EE867AF0EEC76AF4EEE76AF1EE10FA30
:10F0600004D59FED180A482042F02CB8DFED167A3F
:10F07000B5EEC07AF1EE10FA20EE270A10DDB0F8F6
:10F080008831642213FB02F307EE903AF8EEE77A38
:10F09000F4EEC07AF1EE10FA02D59FED0C0AE2E729
:10F0A000B0F88A31642213FB02F307EE903AF8EECF
:10F0B000E77AF4EEC07AF1EE10FA02DD9FED040A71
:10F0C000D1E77047000000000000C84200A00CC655
:10F0D00000A00C4610B5044600F5405304F500545A
:10F0E00000F50650DFED100A93EDAE0A002118304E
:10F0F0004BF096FAB4F98A01B4F988313221C21A78
:10F100001B1A4A434B4301EE102A00EE903A80202E
:10F11000B8EEC11AF8EEE00A16F022FFBDE8104082
:10F12000482041F0CFBF00BF0AD7A33C00F50053F1
:10F1300093F96831012B03D0022B03D0FFF718BFDE
:10F14000FFF77CBFFFF7C6BFF0B52DED028B00F5D2
:10F1500000563223B6F88451DFED310A15FB03F572
:10F1600000F50A5700F5405393EDAF0A83B0002134
:10F17000044638464BF054FA9FED2A1ADFED2A0A6E
:10F18000BF2016F0EDFE4720B0EE408A41F0AEFF02
:10F190009FED241ADFED240A30EE080AC02016F095
:10F1A000DFFE6B4207EE903AF8EEE77AB4EEE70A3C
:10F1B000F1EE10FA26D98DED000A07EE905A9DED7A
:10F1C000007AF8EEE77AF4EEC77AF1EE10FA04D896
:10F1D0003846CDED007A4BF017F947209DED000A37
:10F1E00041F070FF96F8DC3A04F52B5004307BB107
:10F1F0000E4B019301AA694638F0AEFA03B0BDEC9C
:10F20000028BF0BD3846CDED007A4BF0FDF8D4E727
:10F21000694638F00DFA012386F8DC3AEEE700BFC4
:10F220000AD7A33C00A08C4600A08CC60AD7A33CFA
:10F2300000F540539FED117AD3EDAF7A00F5005001
:10F2400067EE877A90ED5D6A90ED5B7A27EE067A3D
:10F25000F0EEE76AF4EEC76AF1EE10FA04D59FED1E
:10F26000080A472041F02EBFF5EEC07AF1EE10FA01
:10F27000CCBF9FED040A9FED040AF2E70AD7233CB6
:10F280000000000000A08C4600A08CC610B504460B
:10F2900000F5405304F50054DFED110A93EDAF0A79
:10F2A000002100F50A504BF0BBF9B4F984314FF658
:10F2B000CE71322213FB02F213FB01F301EE102A8E
:10F2C00000EE903AF120B8EEC11AF8EEE00AB1EE85
:10F2D000400A16F045FEBDE81040472041F0F2BE5E
:10F2E0000AD7A33C00F5005393F96931012B03D0F1
:10F2F000022B03D0FFF728BFFFF79ABFFFF7C6BF67
:10F30000FEF702BE70B500F5005088B090F991018B
:10F310000C46D8B105210E4842F094FA0921064660
:10F320000B4842F08FFA01210390094842F08AFA13
:10F3300004AD00210346039A00912846314606F0A9
:10F3400083F995E80F0084E80F00012008B070BD34
:10F35000E059002037B50C460022054611460F48FB
:10F3600042F07CFA62680D48012142F08FFAA268EF
:10F370000A48052142F08AFAE2680848092142F069
:10F3800085FA05F5065001240DF1070111308DF8BD
:10F39000074033F0D7FB204603B030BDE0590020D2
:10F3A00037B503680191DD6C04460FF011FD90F84C
:10F3B000C412019AB02303FB0101AC3120462B4655
:10F3C00003B0BDE8304018477FB5044604F59356B6
:10F3D000684608360D4606F017F96946304601F0D2
:10F3E000B1FE48B929462046FFF7B4FF064650B99A
:10F3F0000026304604B070BD2946304601F06CFD51
:10F400000028EFD1F4E795E80F0004F548542834BC
:10F4100084E80F00EDE7000010B5074B1B680446B9
:10F42000D86A036801211B68984704F57C600121B4
:10F43000BDE8104035F004BFCC25002010B5074BC7
:10F440001B680446D86A036800211B68984704F5C6
:10F450007C600021BDE8104035F0F2BECC250020D4
:10F4600010B5044654F022FF04F500540021C4F8FE
:10F470006803472041F0B2FF0021482041F0AEFF71
:10F4800042F052F8BDE8104041F036BD70B5044678
:10F4900004F5005304F5405583F80421D5F83832BB
:10F4A0008B420846164627D0C5F838120B685B68B1
:10F4B000984710B32046FFF7AFFFD5F8380203682E
:10F4C0001B6898473246C1B204F57C6036F090F86C
:10F4D00004F52B500021203004F580543FF0B4FE99
:10F4E00004F58D63D3ED007A9FED067AF8EEE77AA6
:10F4F00067EE877AC5EDAB7A70BD2046FFF79EFFB9
:10F50000DBE700BF0AD7233CF7B5044600F590506F
:10F5100014302FF049FF5F4B04F5335001223C308B
:10F520009A71DA7104F5866704F03CFD04F52B55F9
:10F530000823C4F844343846203504F0E9FB284653
:10F540003CF002FE284640F08FF907F081F82023B6
:10F55000036307F07DF808F0F3F804F593560223EF
:10F56000C4F8743104F5907008360EF0F9F830469E
:10F5700000F078FE04F58053002283F87125B4F979
:10F58000A43004F698001BB9B4F8A230A4F8A43053
:10F59000B4F8A41016F054F8304600F05DFF384679
:10F5A000012104F045FA3C4B00933C4B019302AB24
:10F5B00013E9060004F57C6035F036FE40F0CCFC23
:10F5C0009922292141F0D8FB40F0C6FC40F06CFCA8
:10F5D00004F500562046FFF78BFC96ED577ADFEDD9
:10F5E000307AF0EEC76AF4EEE76AF1EE10FA04F54D
:10F5F000405747D8D6ED587ADFED2A6AB0EEE76A71
:10F60000B4EEE66AF1EE10FA3CD8DFED276A27EE99
:10F61000267A67EEA67ABDEEC77AFDEEE77A87ED29
:10F620008C7AC7ED8D7AD7F8303243B9D7F83432B7
:10F630002BB904F5485128312046FFF763FE1B4BD8
:10F640001B68986A03684FF47A715B68984796F96B
:10F650008E112046FEF7D0FE014610B904F549513F
:10F6600004311F222046FFF711FFD6ED597AF5EE3F
:10F67000C07AF1EE10FA0BDD204603B0BDE8F04091
:10F68000FFF7EEBE0A4A0521284638F013FCCAE708
:10F6900003B0F0BD755A0020D025002001F300080A
:10F6A0000000B442000034438096184BCC25002063
:10F6B000D0D9080808B50A2922D8DFE801F00D19C9
:10F6C00011151D2121212121060000F548513C3151
:10F6D000FFF7DCFE012008BD00F549510431F7E7D2
:10F6E00000F549512431F3E700F549512831EFE79E
:10F6F00000F549512C31EBE700F549510831E7E7B6
:10F700000020E8E700F57C6036F01ABC01480321D0
:10F7100041F0FABFE059002070B505462DED028B8F
:10F7200005F5405454F0B6FDD4F89432DFED1D7A5F
:10F73000C31A08EE103AB8EE488A28EE278AF1EE8E
:10F74000047AB4EEE78AF1EE10FA29D504F51D73B8
:10F750000FCB04F5217686E80F00D4EDA80A94EDCE
:10F76000A70A05F54A5068EE200A28EE000A043080
:10F7700006F0DAF9DFED0C7A94EDA97A27EE277A14
:10F78000D4EDA27AF8EEE77A0123E7EE087AFDEEEF
:10F79000E77AC4EDA27A84F87032BDEC028B70BDBA
:10F7A0000023F8E7BD3786350000C84230B585B084
:10F7B0006D460446284605F027FF04F59350294678
:10F7C000083001F09BFC50B104F54054002384F84C
:10F7D000D23295E80F0004F50A7484E80F0005B0F2
:10F7E00030BD0000F8B52DED028B00F54054054604
:10F7F00094F87032002B5ED0D4F8382200F54953CB
:10F80000243300F5485600F54A579A4206F1280677
:10F8100007F1040717D094F8CC32DA0713D439462D
:10F82000304606F06FF89FED277AF6EE007AE0EEAC
:10F83000077A9FED257AFDEEE77AF8EEE77A67EE34
:10F84000877AC4EDAB7A3946304606F0FDF805F507
:10F85000005584EDAC0A95F96A31DFED1C6AD4F8E5
:10F860003802012B05BFD4F88832D4F82C22D4ED0D
:10F87000AA7A9B1A08BF07EE903AF8EEE77A87EE6D
:10F88000A67A84EDB17A03681B689847022812D0E3
:10F8900094F8CC329B070ED495F96A31D4EDAC0ABA
:10F8A0009FED0B8A53B994EDB00A73F0BBFD20EEC7
:10F8B000080A84EDAD0ABDEC028BF8BD94EDB10AE7
:10F8C000F3E700BFA00CB3450AD7233C0000C842B1
:10F8D000E02E654273B50446FFF71EFF2046FFF792
:10F8E00065FF04F500552046FFF77CFFD5ED597AFA
:10F8F000F5EEC07AF1EE10FA09DC244B1E68F06ACE
:10F900000368DB699847012816D102B070BD54F036
:10F91000CDFCD5F8683395ED597ADFED1D6AC01A34
:10F9200007EE900A27EE267AF8EE677AF4EEC77AA9
:10F93000F1EE10FAE1D5E8E7F36A93F89C10E9B923
:10F9400095F98F31012B10D19FED120A472041F01C
:10F95000B9FB9FED100A482041F0B4FB41F0E4FDF3
:10F9600002B0BDE8704041F0C7BA4720019141F0B4
:10F9700017FD0199482041F013FDEFE704F54054CD
:10F98000D4F8380203689B689847E7E7CC25002045
:10F9900000007A440000000037B54B68054613B9F3
:10F9A0008A68002A49D005F540540A20C4F87C3200
:10F9B0008B68C4F88032CA6892FBF0F2C4F87822EF
:10F9C0000B6993FBF0F3C4F8A832B1F91630DFED00
:10F9D0001C7A07EE103AB1F91830B8EEC77A87EE04
:10F9E000276A07EE103AB1F9143084EDA86AB8EE30
:10F9F000C77AC7EE276A07EE103AB8EEC77AC4EDA9
:10FA0000A96AC7EE275AC4EDA75A54F043FCC4F8BC
:10FA1000940254F04BFC0221C4F898022846FFF7E8
:10FA200071FE50B105F54A531C330093D4E99F127F
:10FA3000D4F878322846FEF731FA03B030BD00BF63
:10FA40000000C84210B52DED028B044691ED018AED
:10FA5000DFED207A94F8413428EE278A00F586609D
:10FA6000242202FB0303F0EE480A93ED090A03F097
:10FA700087FCB4EE400AF1EE10FAF0EE400A1FD611
:10FA80009FED157AF0EEC07AF4EE477AF1EE10FAB7
:10FA900016DC04F54053D3EDB27A93F8CC2277EE1E
:10FAA000807A5107C3EDB07A0AD5F1EE407A002191
:10FAB0006FF38202C3EDB27AC3F8C01283F8CC228E
:10FAC000B0EE480ABDEC028B2046BDE81040FEF7C0
:10FAD000C1B900BF0000C842FFFF7F7FB1F900300D
:10FAE00007EE903AF8EEE77A00F5405010B5C0ED19
:10FAF000AB7AB1F9023007EE903AF8EEE77A0023DC
:10FB0000C0F8B032C0EDAD7AB1F9002090F8CC3237
:10FB100047F6FF74121B18BF012262F3000380F83E
:10FB2000CC32B1F9023090F8CC221B1B18BF012354
:10FB300063F3410280F8CC2210BD000010B500F53F
:10FB40004054D4F8980250B154F0B0FBD4F8983235
:10FB5000C01A41F2873398428CBF00200120014B2C
:10FB6000187110BD755A002070B52DED028B00F58F
:10FB700000541646B4F98A2194ED600A01EE102A69
:10FB8000B4F9882100F54053D3EDAD7AD3EDAB8ABB
:10FB900000EE902ADA20B8EEC11AF8EEE00A30EE54
:10FBA000270A0D4616F0DCF9B4F98821B4F98A3138
:10FBB00007EE902AF8EEE77A9B1A30EE670A07EE16
:10FBC000903A30EE000AF8EEE77AB7EE008A80EE5F
:10FBD000277A37EE487A86ED007A94ED5F0A38EEA0
:10FBE000800A16F029F9B4F9843107EE103A30EEA4
:10FBF000000AB8EEC77A0120C0EE077A77EEC87A1D
:10FC0000BDEC028BC5ED007A70BD000070470000AE
:10FC100000207047704700000020704700207047A8
:10FC200000207047002070479FED010A704700BF19
:10FC3000000000009FED010A704700BF00000000B7
:10FC4000002070477047000010B50446143000F0E3
:10FC500019F804F12C0000F015F804F1740054F0C8
:10FC600031FB04F1F40054F02DFB4FF0FF33C4F8E6
:10FC70005031204610BD0000014B1868704700BF8E
:10FC8000E459002070470000F0B52DED048B91B0D1
:10FC900004466D46284605F0B7FC94F8BC33002BAB
:10FCA00072D004F57A730FCB85E80F0094F8F8331F
:10FCB000D4EDEC8A94EDED8A94EDEE9A002B63D0AE
:10FCC00094F8D033002B5FD02D22002104A8D4F863
:10FCD000C073D4F8C463D4F8C853D4F8CC4375F0D7
:10FCE00087FDA3238DF8103095238DF8113046231E
:10FCF0008DF8123054F0E2FA9FED250A9FED257A37
:10FD0000CDF8171068EE807ACDF8130067EE877A89
:10FD1000FDEEE77A17EE903A68EE007A29EE000AD7
:10FD200067EE877AADF81B30FDEEE77A20EE070A22
:10FD300017EE903AADF81D3016F0A8F8DDED017A17
:10FD40009FED157ACDF82D70BCEEC00AF8EEE77A7B
:10FD500010EE103A67EE877AADF81F3017EE903A42
:10FD6000CDF82130029BCDF82530039BCDF829300A
:10FD7000CDF83160CDF83550CDF8394036F016F970
:10FD80002D2204A935F074FA11B0BDEC048BF0BD3E
:10FD9000E02E65420000C8420AD7233C30B52DED65
:10FDA000028B8BB0044624220D4601A8002175F079
:10FDB0001FFDA3238DF8043095238DF805304823CB
:10FDC0009FED1F8A8DF8063054F078FAD4ED817AD1
:10FDD0002B68CDF80F3067EE887A95ED020ACDF8E2
:10FDE0000B1017EE903AD4ED827ACDF8133067EE0F
:10FDF000887A6B68CDF8173017EE903ACDF8070087
:10FE0000CDF81B3016F018F810EE103A94ED830A76
:10FE1000CDF81F3020EE080A16F00EF810EE103A5A
:10FE2000CDF8233094F80C338DF8273036F0BEF837
:10FE3000242201A935F01CFA0BB0BDEC028B30BDB9
:10FE4000E02E654230B587B014460D4618220021D9
:10FE5000684675F0CDFCA3238DF8003095238DF80E
:10FE6000013049238DF8023054F028FAA368039337
:10FE7000E36804936368CDF807100593CDF8030099
:10FE80008DF80B5036F092F81822694635F0F0F9EB
:10FE900007B030BD10B58EB0044602A805F0B4FB23
:10FEA00002A9204601F02AF9002845D001F044FBC0
:10FEB000694600F0BBFF1F22002106A875F098FCE0
:10FEC000A3238DF8183095238DF819304A238DF827
:10FED0001A3054F0F3F9DDED037A9FED1B7A049BA1
:10FEE000CDF82330F8EEE77A059BCDF8273067EEA2
:10FEF000877ACDF81B0017EE903ADDED007ACDF849
:10FF00002B30F1EE677A17EE903ACDF81F102046AD
:10FF100001A9CDF82F3000F0FDFB78B1DDED017ABD
:10FF2000F1EE677A17EE903ACDF8333036F03EF8BE
:10FF30001F2206A935F09CF90EB010BD36F036F838
:10FF4000DFED027AEEE700BF0AD7233C5241C07FC3
:10FF50000023036043608360C36003614361836186
:10FF6000C36103627047000090F8C432B02202FB04
:10FF7000030390F8082393F8A13012B1012B28BF96
:10FF800001231846704700002DE9F04F04468BB05E
:10FF90004FF0000A0D461BF0B9FF84F814A204F5D7
:10FFA00006704FF07E5753F02BFB4FF47A73A4F892
:10FFB000623284F86852C4F84872C4F84C72C4F8CB
:10FFC000507204F51B70002505F01EFB04F52B791B
:10FFD0000323C4F8803204F53476C4F89452C4F88C
:10FFE0009852C4F89C52C4F8A052C4F8A452C4F861
:10FFF000A8524846FFF7ACFF04F5487B3046FFF7B0
:020000040801F1
:10000000A7FFC4F81453C4F81853C4F81C53584637
:10001000FFF79EFFC4F84453C4F84853C4F84C5348
:10002000C4F85053C4F85453C4F85853C4F85C533C
:10003000C4F86053C4F86453C4F86853C4F86C53EC
:10004000C4F87053C4F88C53C4F89053C4F8945354
:10005000C4F8A853C4F8A453C4F8A053C4F8B053C8
:10006000C4F8B453C4F8B853C4F8CC53C4F8C85354
:10007000C4F8C453C4F89C73C4F8C07304F5757015
:1000800005F0C2FA04F57A7005F0BEFA04F5806353
:10009000C4F8FC531D6004F5816304F583601D60A2
:1000A0005D609D6005F0B0FA04F22C4304F26448F0
:1000B0001D605D609D60684BC4F83C3404F50D73B1
:1000C000C4F8403404F50E73C4F8443404F50F73D7
:1000D000C4F8483404F51073C4F84C3404F24523D2
:1000E000C4F8503404F51173C4F8543404F58B6328
:1000F00040461D605D609D60FFF72AFF04F591603A
:10010000FFF726FF04F5976304F23C421D605D6033
:100110009D6004F2C44304F2A4501D605D609D60C4
:1001200004F59A631D605D609D6004F2DC431D6010
:100130005D609D6004F2EC431D605D609D6004F2B3
:10014000FC431D605D609D6004F5A463C2F8D4703B
:10015000C2F8D8701D605D609D6004F22C531D6074
:100160005D609D6004F5A9631F605D6004F26C53DF
:100170001D605D609D6004F5AF631D605D609D6006
:1001800004F5B2631D605D609D6005F03DFA04F208
:10019000B45324221D605D6004F2BC5351461D60BF
:1001A0005D6004F2C45340461D605D6075F020FB45
:1001B00004F2E450C8F82070C8F81070C8F8007055
:1001C000FFF7C6FE04F5C16304F5C7601D605D60FE
:1001D0009D6004F214631D605D609D6004F5C4635E
:1001E0001D605D609D6004F22C631D605D609D601C
:1001F00005F00AFA194B1A491C60204631F0AAFE94
:1002000051462422584675F0F3FAC4F84073C4F8F6
:100210003073C4F8207304F5257207CA04F52873F7
:1002200083E80700484694EDAA1AD4EDA90A94ED94
:10023000A80A16F037FA3546494668466E4616F063
:1002400053F90FCE0FC50FCE0FC533682B60204674
:100250000BB0BDE8F08F00BF10DC0808E8590020A3
:10026000C0DA080810B5044688B001F0EFF994F937
:100270003232012B02D1274804F056FB022B0AD15F
:10028000032384F8323204A9012304F111008DF80C
:10029000103032F019FC94F8323284F8903204F2C3
:1002A0003C4001F089F994F93132642B30D1652357
:1002B00004A904F231208DF8103032F043FC04A977
:1002C000204631F01DF918B304238DF818300023AF
:1002D000CDE9013303930F230593694604A831F058
:1002E000E1FA059B28B108AA02EB8302009942F8C3
:1002F000581C0133112B0593EFD951F0CBFE9DED26
:10030000031ADDED020A9DED010A652151F080FE20
:1003100008B010BD20DA080870B500F5257600F5A4
:1003200028758CB004463146284617F0A7FDE0B981
:1003300096E8070085E8070004F52B7194EDAA1AEA
:10034000D4EDA90A94EDA80A0191084616F0AAF97D
:1003500002AD019902A816F0C7F80FCD04F5347468
:100360000FC40FCD0FC42B6823600CB070BD00000C
:1003700013B540F2411200F50671044601A812F0CF
:1003800031FA04F23C4001F0FFFA20461BF09CFFDA
:1003900001A812F049FA02B010BD0000F8B50B68D0
:1003A000C0F804324B68C0F808328B68C0F80C32D1
:1003B00001F10C0607460C4600F548750FCE0FC537
:1003C0000FCE0FC533682B6004F1300207CA07F562
:1003D000457383E8070004F13C0207CA07F551732F
:1003E00083E8070004F1480207CA07F5547383E85D
:1003F0000700543494E8070007F5577383E80700B3
:10040000384601F037FA3846BDE8F84001F01ABA2C
:1004100013B5044600F23C40019002F0ABFE04F537
:10042000BB610198009102F003FA0099204602B0E6
:10043000BDE81040FFF7B2BF4A78064BC2F3401246
:100440001A754A78C2F380125A750A78C2F30012FC
:100450009A757047755A002013B540F2F52204468C
:1004600000F5067101A812F0BDF9002104F23C402C
:1004700001F0FCFC94F8603223B120461CF0D0F867
:1004800084F8600201A812F0CFF902B010BD00009C
:1004900038B590F80C3305460C462BB1032B0BD026
:1004A00095F86832DB070CD405F5C7630FCB84E8F9
:1004B0000F0095F8480603E01BF05CFF0028EFD022
:1004C00038BD0020FCE7000000F23C4090ED350A0A
:1004D0007047000000F23C4090ED360A7047000083
:1004E00010B490F80C230C462AB1032A0AD000203D
:1004F0005DF8044B704700F5B26007C884E8070058
:100500000120F5E75DF8044B1BF01CBF90F8840355
:10051000431E58425841704738B590F80C330D4689
:100520008BB900F23C4001F0A1FA044610B9002456
:10053000204638BD01F0EEF9D5ED007A27EE800AAD
:1005400085ED000AF4E7D0EDE07AC1ED007A90F88D
:100550007C43002CEBD090EDDE7ADFED086AB4EE40
:10056000E67AF1EE10FAF7EE006AB8BFB0EE667AFE
:1005700067EE877AC1ED007ADAE700BF0000003449
:1005800090F80C33032B01D11BF05CBE00207047A8
:1005900090F80C23032A01D11BF076BF00F23C40F7
:1005A00001F0C6BE30B590F80C3385B004460D4658
:1005B0008BB1032B18D004F5257017F099FC284651
:1005C00001A98DED010ACDED020A8DED031A17F098
:1005D000E9FA012006E000F23C4001F0F1F90028C0
:1005E000E9D1002005B030BD90F86032002BF8D082
:1005F0001BF032FFDFE700007FB590F80C2332B12B
:10060000032A4FF0000309D0039304930CE000F297
:100610003C4007B05DF804EB01F0ACBA03A90393CA
:10062000049305931BF004FE9DED030ADDED040A1F
:1006300007B05DF804FB000007B590F80C3333B148
:1006400000F57F7003B05DF804EB17F0B7BB00F264
:100650003C4001F08FFA68468DED000ACDED010AAD
:1006600017F0ACFB03B05DF804FB000090F80C033E
:10067000003818BF0120704708B590F80C23032AF2
:1006800005D0BDE8084000F23C4001F05DBA1BF027
:10069000CFFD012008BD000010B590F80C230C46DA
:1006A0001AB1032A07D0002010BDBDE8104000F2A7
:1006B0003C4001F0EDB91BF0D1FD012084ED000AB2
:1006C000F2E7000030B590F80C3385B005460C46D3
:1006D00023B1032B09D0002005B030BD00F23C400F
:1006E00005B0BDE8304002F0D3B8002302A9029360
:1006F00003931BF085FD0028EDD001A928461BF0CF
:100700008BFD0028E7D0029B2360039B6360019B65
:10071000A360E1E790F80C231AB1032A05D000206A
:10072000704700F23C4002F0D9B81BF075BD0000E4
:1007300090F932323BB990F8683213F0010F14BFD0
:10074000032000207047032070470000F7B50446DF
:10075000FFF7EEFF0546002862D0032839D194F850
:1007600060326BB394F86832D8072BD501A92046C4
:100770001CF080F8BDF80430002B18BF002594F859
:10078000146206F0FD06012E4AD10023032D0193C9
:1007900007D101A920461CF079F820461BF080FE05
:1007A000064604F23C4002F025F908B994F8090322
:1007B0009DF80430D90703D55A0701D59F0632D4D6
:1007C00000252DE020461BF0F5FC002808BF002581
:1007D000D5E70025D3E713F0020F2EE094F9443259
:1007E00023B99DF80430DB092FD0E9E7002EF8D0BB
:1007F0000EF0EEFAFFF7B8FB022807D99DF8053096
:100800009806DDD59DF80430D906D9D5FB6A93F852
:100810009C30002BE5D118E0DA0601D41B0718D56F
:10082000284603B0F0BD0028FAD094F80923B4F9A3
:100830004C36002ACFD013F0010FF1D1154B1F68B1
:10084000FB6A93F89C30002BC8D19DF804309C07BC
:10085000E2D405F0FDFE05F0F9FD0028B0D10EF060
:10086000B7FAFFF781FB0228AAD90EF0B1FA90F887
:10087000C432B02202FB030090ED2F7AF0EE007A32
:10088000B4EEE77AF1EE10FA9AD59DF80530DB095F
:10089000C6D195E7CC2500202DE9F04790F86032CD
:1008A00092B00446002B00F0948020461CF0EEF835
:1008B0002046FFF74BFF03287BD104F5487800273B
:1008C000414620460097019702971BF0BBFD694601
:1008D00020461BF0ADFD009BC4F80432019BC4F818
:1008E0000832029BC4F80C32204600F0C3FF2046B9
:1008F00000F0A8FF14F032FE054620461BF072FC03
:100900000028A8BFC6B203AA4FF0FF312046BCBFE3
:1009100095F8129395F813630397A8BFB14604970F
:1009200005971BF0A9FC03A817F0E2FA4FF00C0A98
:100930000AFB095084EDD10AC4EDD20A84EDD31A22
:1009400004F5517100F5117017F0E2FA04F55777CC
:100950000AFB065584EDC50AC4EDC60A84EDC71A24
:100960003A464FF0FF31204605F5C4751BF098FC60
:1009700095E8070006AE86E807003946304617F0CE
:100980002DFB04F52B72414609A815F03DFD3146BB
:1009900009A815F0BBFC09A9204684EDD40AC4EDD2
:1009A000D50A84EDD61A1BF071FF09A92046FFF77E
:1009B00043FD94F84E36002B3AD109A804F024FEEA
:1009C00009A920461BF0E2FC90B3012384F84E36BF
:1009D0002EE0D0F864321BB953F068FCC4F864020E
:1009E000154B1B68D86A03685B68984788B153F059
:1009F0005DFCD4F86432C01AB4F86232984204D96B
:100A000020461BF00DFE84F8600294F860327BB142
:100A10004BE753F04BFCD4F86432C01A41F28733F1
:100A20009842E4D835F0C2FA35F0A6FA0028DED1B3
:100A300012B0BDE8F08700BFCC25002090F80C3341
:100A400023B1032B4FF0000007D0704790F93222FA
:100A5000032A04D10A70012070470870FBE718468A
:100A60007047000073B50D460DF107010446FFF70E
:100A7000E5FF064628B19DF807302BB1032B09D0BE
:100A80000026304602B070BD04F5C7630FCB85E881
:100A90000F00F6E7294620461BF06CFC94F86062D4
:100AA000EFE700007FB50E460DF103010446FFF7A6
:100AB000C5FF054618B90025284604B070BD9DF84D
:100AC000033083B1032B16D004F5257017F010FA0C
:100AD00001A930468DED010ACDED020A8DED031A14
:100AE00017F060F8E8E7314604F23C4000F068FF98
:100AF0000028E9D1DFE794F86032002BDBD03146E3
:100B000020461BF0A9FCDFE737B50D460DF10701C4
:100B10000446FFF793FF28B19DF8073023B1032B5C
:100B20000FD0002003B030BD04F5BB631B682B6001
:100B300004F2DC5304F5BC641B686B602368AB6093
:100B4000F0E7204629461BF073FC94F86002E9E7C1
:100B500010B50446FFF7ECFD18B1032807D00020BC
:100B600010BD04F23C40BDE8104000F053BF94F8C3
:100B70006032002BF3D020461BF01CFB0028EED087
:100B800094F8143203F0FD03012BE9D194F80C031F
:100B9000C31E58425841E3E710B50446FFF7C8FDAD
:100BA00080B1032810D194F8600250B153F07EFB5D
:100BB000D4F86432C01A44F62063984294BF0020EF
:100BC000012010BD0120FCE70020FAE708B502462D
:100BD000FFF7AEFD032804D110461BF057FE01209D
:100BE00008BD0020FCE7000030B585B00446019147
:100BF000FFF742F80199054610B9002005B030BD55
:100C00000191FFF70BF801990028F6D02846FFF76D
:100C100009F80028F1D0B4F84C365907EED494F80E
:100C20000933002BEAD00B4A1268D26A92F89C5022
:100C30006DB103A92046FFF7C9FF30B19DF80E3012
:100C40009A07DBD5C3F38000D8E72846D6E71846D5
:100C5000D4E700BFCC2500202DE9F04190F80C33FB
:100C60008CB00027032B06460C46154600970197CB
:100C7000029719D11BF0B6FA6A4680464FF0FF3151
:100C800030461BF00DFBB8F1FF3FA760676027609F
:100C90000DD114F063FC2B4690F81313224613F089
:100CA000EBFC0CB0BDE8F0814FF0FF38EBE714F03F
:100CB00055FC2B4622465FFA88F113F0DDFC95EDDA
:100CC000000A684617F050F903A920468DED051A71
:100CD0008DED030ACDED040A17F080F906F52B72AD
:100CE00006F5487103A815F08FFB214603A815F0FF
:100CF0000DFB84ED021A84ED000AC4ED010A95EDA6
:100D0000007ADFED037AA7EE271A84ED021AC8E70E
:100D10000AE81C4137B5054600F5067140F6033276
:100D200001A811F05FFD2846FFF702FD044640B11F
:100D300003280AD0002401A811F076FD204603B054
:100D400030BD28461BF0DAFAF5E728461BF0D6FA44
:100D50000446F0E708B50246FFF7EAFC10B10328A5
:100D600006D008BDBDE8084002F23C4000F01CBEC1
:100D7000BDE8084010461BF095BD00000B4610B4BE
:100D800011462BB1032B09D000205DF8044B7047AE
:100D90005DF8044B00F23C4000F01CBE5DF8044BD3
:100DA0001BF0F4BA13B50446FFF7C2FC0A4601462D
:100DB00020460192FFF7E2FF70B9084B019A1B68C9
:100DC000DB6A93F89C0038B194F80C13204602B00B
:100DD000BDE81040FFF7D2BF02B010BDCC25002007
:100DE00037B504460D4640F2B25200F5067101A82F
:100DF00011F0F8FC294620461BF0E6FA94F80C3373
:100E0000032B054610D148B104F583612046FFF756
:100E1000C9FF84F82804204600F05CFD01A811F009
:100E200003FD284603B030BD0025F7E770B590F804
:100E30007C32DB0786B004460D460CD402F04EFF30
:100E4000437C242202FB0300D0ED0B7AF1EE677A9B
:100E5000C5ED007A3BE002A804F0D6FB01A92046CC
:100E6000FFF758FCE8B90DF0B3FF94F94432022BB8
:100E70000646E3D1FFF778F80228DFD996F8C402D6
:100E80009FED147AB02303FB0066D4F87032D6F8D5
:100E9000B0209B1A07EE903AF8EEE77A67EE877A71
:100EA000D6E702A92046FFF77DFF0028DBD0D4F863
:100EB0007022039BDFED076A9DED017A9B1A07EE16
:100EC000903AF8EEE77AA7EEE67A85ED007A06B07A
:100ED00070BD00BF0AD7233CF0B50C4687B000F5C3
:100EE0000671064640F6863201A811F07BFCA36825
:100EF00053B9E36843B9636833B9002701A811F017
:100F000093FC384607B0F0BD204604F053FC00289F
:100F1000F3D094E80F0002AD85E80F0000212846C9
:100F200004F00AFC07460028E7D096F87C32DB077D
:100F300004D435F03BF8192134F074FF95E80F0024
:100F400006F51B7C8CE80F0096F87C3243F0010319
:100F500086F87C32304600F0BDFC3DF07BFD46213A
:100F60003EF072F93DF076FD45213EF06DF9054BFE
:100F7000A2681B68DB6A1A61E2685A6162689A615A
:100F8000BCE700BFCC25002038B5144B1B68DD6AD8
:100F90002B6804465B6828469847F0B12B690BB96B
:100FA0006A69D2B1C4F874326B69C4F87832A9693D
:100FB000002204F51B7004F02DFB94F87C3223F022
:100FC000030343F0030384F87C323DF043FDBDE8A6
:100FD0003840034A062136F06DBF38BDCC250020CD
:100FE00048DA080810B588B004460593FFF7A0FB5F
:100FF0000328059B4FF000000AD10690079006A831
:1010000002900B9801900A98009020461BF02EFA4F
:1010100008B010BD38B50446FEF72EFE0546D0B127
:1010200094F80C33032B03D095F84E41204638BD7D
:1010300020461BF093F9FF280446F5D001462846C8
:10104000FEF7F0FD0028EFD021462846FEF7E6FD2A
:101050000028E9D0EAE70446E8E7000008B590F880
:101060000C33032B05D014F079FA90F91203C0B2B7
:1010700008BD1BF0B7F8431CF9D1F4E708B590F8A8
:101080000C3383B1032B03D1BDE808401BF0A2B899
:1010900033F060FB40F6ED424FF4801133F012FB69
:1010A0004FF0FF3008BD1846FCE7000090F80C3305
:1010B000032B01D11BF036BE7047000090F80C33B3
:1010C000032B01D11AF0D4BF704700001BF05AB8AF
:1010D00010B504461DF068FE2046FEF7D5FD2046FB
:1010E000BDE81040FEF7D6BE90F80C330BB1032BD1
:1010F00001D11BF093BE00207047000030B500F511
:10110000757304460D460FCB85E80F0094F8E40391
:1011100030BD0000D0F880330B6090F87C0370473E
:10112000D0F888330B6090F88503704730B500F530
:10113000677304460D460FCB85E80F0094F8AC03A7
:1011400030BD000030B500F5836304460D460FCB7B
:1011500085E80F0094F8280430BD000010B500F2B7
:101160002C4203460C4607CA84E8070093F838046B
:1011700010BD00002DE9F0432DED028B8BB005462C
:101180000E461746FFF746FF014680462846FFF702
:101190002BFD0446002848D0FEF76EFD4146FEF7C1
:1011A00043FD86ED000A95F93032002B3ADD0DF053
:1011B0000FFEFEF7D9FE012834D90DF009FE90F894
:1011C000C432D5EDDE7ADFED5D8A96ED000AB022FD
:1011D00002FB030095F93032D0ED2F0A07EE103AEA
:1011E000F4EEE87AB8EEC77AF1EE10FAB7EE008ABC
:1011F000B8BFF0EE487A37EE201A20EE270A70EEDC
:10120000C70A40F2B63014F0ABFED5EDDE7AF4EE4C
:10121000E87AF1EE10FAB8BFF0EE487A80EE277A5D
:1012200086ED007A01233B7003E095F8083333B96B
:10123000387020460BB0BDEC028BBDE8F08395F80A
:101240000C334FF00009CDF80490CDF80890CDF89C
:101250000C9043B1032B10D0CDF81090CDF8149022
:10126000CDF818907CB902233B703246414605F216
:101270003C4001F083FB0446DBE701A928461BF054
:1012800061F80446E8E795F80C33002BEBD004A98D
:101290002846FFF763FF04460028E4D001A904A80C
:1012A00016F04CFE07A8CDED080A8DED091A8DED5C
:1012B000070A17F057FA04A8B0EE408A17F052FA5E
:1012C00095F93032002B30DD07EE903AF8EEE77AF0
:1012D0004FF47F7070EE670A37EE801AF5EEC00AA1
:1012E000F1EE10FA48BFDFED160AF4EE410AF1EE16
:1012F00010FAB0EE480AC8BFB0EE601A14F030FE23
:10130000B0EE408AD5EDDE7A9FED0C7AF4EEC77A26
:10131000F1EE10FAB7EE007AB8BFF0EE477A88EE39
:10132000277A032386ED007A7DE7B5EEC08AF1EED9
:1013300010FA48BF9FED028AE4E700BF00000034C6
:101340000000000010B50446FFF788FE84F80D0386
:101350002046FFF783FE84F80E032046FFF77EFE4B
:1013600084F80F032046FFF789FE04F55A7184F8CC
:1013700010032046FFF7B4F884F8740300F0CAFAAB
:1013800004F5617284EDDE0A04F560712046FFF712
:10139000F1FE04F5627184F87C032046FFF7BCF887
:1013A00004F5637184F885032046FFF7E9F804F536
:1013B000677184F898032046FFF7F4F804F56C7120
:1013C00084F8AC032046FFF79FFB04F5707184F8A6
:1013D000BC032046FFF766FB04F5757184F8D00363
:1013E0002046FFF755F804F57A7184F8E4032046A7
:1013F000FFF738FB84F8F8032046FFF7FDF804F503
:10140000806384EDFF0A2046C3ED000AFFF714F95C
:1014100004F2044383ED000A04F2144204F58161EE
:101420002046FFF719FC04F583612046FFF7BAFC5C
:1014300004F22C4184F828042046FFF71DF984F8B3
:10144000380410BD37B50D46044600F0FFF81DB94D
:1014500014F084F813F040F84FF4BE7204F50671EE
:1014600001A811F0BFF994F869322BB92046FFF7B3
:101470008BFD012384F86932224B1D68A86A03683A
:101480009B6998472046FEF747FF2046FEF7C0FFBE
:10149000204600F051FA2046FFF7FEF9286B30B1E4
:1014A0000368D4EDD20ADB6894EDD10A9847D4F8EA
:1014B000100208B153F068FE204600F07DF8204687
:1014C000FFF744F994F8903284F80C0383420ED06D
:1014D00084F8900298B10C4D0C4B032808BF1D46B0
:1014E0003DF0B8FA0A4A2B46062136F0E3FC2046C6
:1014F000FFF728FF01A811F097F903B030BD054DA3
:10150000EEE700BFCC2500208BAD08083FDA0808C5
:1015100060DA080844DA0808D0EDDE7A9FED057A33
:10152000F4EEC77AF1EE10FAB7EE000AA8BFB0EEFB
:10153000670A704700000034014B1868704700BF0D
:10154000E85900204FF0FF3070470000012070473D
:10155000704700000020704700207047704700006F
:10156000704700000020704700207047002070473F
:10157000002070470020704700207047002070470F
:10158000012070470368D3F8943018470020704753
:1015900000207047002070470020704700207047EF
:1015A00000207047002070470020704700207047DF
:1015B00000207047704700007047000008B513F026
:1015C000CDFF90F8130308BD08B513F0C7FF90F8DE
:1015D000120308BD30B52DED028B9FED1A1ADFED19
:1015E0001A0A91ED000A87B005462D200C468DEDB4
:1015F000011ACDED000A14F0B3FC9DED011ADDEDEA
:10160000000AF0EE408A2E2094ED010A14F0A8FCA6
:101610009DED011ADDED000AB0EE408A2F2094ED19
:10162000020A14F09DFC03A905F52570CDED038A8F
:101630008DED048A8DED050A31F068FB07B0BDEC35
:10164000028B30BDC2B8323EC2B832BE10B50446BD
:1016500052F02CFED4F8F4321BB1C21AB2F57A7FE4
:1016600012D30A4A1268D26A92F89C2002B15BB97E
:10167000C4F8F40294F8314213F070FF80F80D437F
:1016800004F0E6FF80F8254010BD00BFCC25002007
:101690002DE9F0432DED028B91ED007AD1ED037A27
:1016A00087B08DED047AB0EEC77AB5EEC07AF1EE70
:1016B00010FADDE91087DDF84C90CDED057A0C4687
:1016C00015461E4606DCF0EEE77AF5EEC07AF1EE3E
:1016D00010FA02DD04A816F0C3FB6B20B7EE001A67
:1016E000FFEE000A9DED050A14F03AFC6C2089ED2E
:1016F000000AB7EE001AFFEE000A9DED040A14F08E
:101700002FFC04A888ED000A16F032FBB7EE008A21
:10171000002852D00023C9F8003088ED008AD4EDAB
:10172000067A67EEA77AF4EEC87AF1EE10FA4ADB91
:101730000023336085ED008ADFED3F0A96ED000A55
:101740007C20B7EE001A14F00BFC86ED000A95ED34
:10175000000A7D20B7EE001AFFEE000A14F000FC2C
:1017600085ED000AD4ED067A129BDFED346AF1EEC6
:10177000677AC3ED007A96ED007AF0EEC77AF4EE60
:10178000E67AF1EE10FA2BD503AB02AA01A92046A6
:1017900014F0E8FF9DED018AB0EE480A71F020FCDC
:1017A00085ED000AB0EE480A71F070FD87ED000A81
:1017B00007B0BDEC028BBDE8F08304A816F0C4FAB4
:1017C0000028A7D1ABE738EE670A14F0FBFA86EDE4
:1017D000000A94ED087AC7EE007AC5ED007AABE70F
:1017E00094ED076AC6EE077AC7ED007A96ED007AA7
:1017F000B0EEC77AB4EEE67AF1EE10FAC4D495ED05
:10180000007ADFED0F6AB0EEC76AB4EE666AF1EEF9
:1018100010FAB9DCB4EE477AF1EE10FAB4D6B0EEB5
:10182000E77AB4EE667AF1EE10FAADDCF4EE677AA0
:10183000F1EE10FABCD7A7E700000000000000346A
:10184000FFFF7F7F1FB500F51773039300F5167335
:10185000029300F51573019300F51473009300F5DE
:10186000127200F5137300F54871FFF711FF05B010
:101870005DF804FB9FED156A90ED817ADFED146A47
:10188000D0ED837A27EE067A67EE867A27EE267AFF
:1018900067EEA67ABDEEC77AFDEEE77A80ED7E7A36
:1018A00090ED827A27EE067A17EE903A27EE267AA6
:1018B000002BB8BF03F50C43BDEEC77AB8BFA03309
:1018C00080ED7F7AC0F80032704700BFE02E65429D
:1018D0000000C8421FB50E4B1B680446B3B16846F2
:1018E00003F092FE69462046FFF72CFC20B16A46C1
:1018F00000212046FEF7A6FA94F87C32DB0705D5D6
:1019000004F51B7201212046FEF79CFA04B010BDBD
:10191000945C002008B502F0E1F9BDE8084001F050
:101920006FBD000010B580F8F812044652F0BEFCFE
:10193000C4F8FC0210BD000010B590F8F83204465F
:1019400053B152F0B3FCD4F8FC32C01AB0F57A7F30
:1019500084BF002384F8F83294F8003353B152F076
:10196000A5FCD4F80433C01AB0F57A7F84BF0023F5
:1019700084F8003310BD000000F5AA700B4607C8BC
:1019800083E80700012070470023C0F89C30C0F8AE
:101990009830C0F89430C0F8A830C0F8A430C0F82F
:1019A000A030C0F8AC30704770470000024B0B60AD
:1019B0004FF07C53136070470000484270470000AE
:1019C00008B50B4600F12801184615F035FD012039
:1019D00008BD000010B500F5B4700C460FC884E8CF
:1019E0000F00204603F000FE30B1FFF7A5FD00F523
:1019F0001B700FC884E80F00204603F0F5FD80F04F
:101A00000100C0B210BD000010B5044604F0A0F8FB
:101A1000204610BD10B5D0F8603104465BB152F0DD
:101A200045FCD4F86031C01A41F28833984294BF23
:101A30000020012010BD0120FCE7000013B5009339
:101A400003680192D3F890309847DDE900210446FD
:101A500028B90448044B0068C06A11F0A3F8204676
:101A600002B010BDCC25002080DB080813B5044669
:101A70000191FEF701F92368019A1B6D014608B137
:101A800090F84E11204602B0BDE810401847000003
:101A900030B585B0002301930293039303680D468C
:101AA000DB6D01A99847044620B1039B2B602046BB
:101AB00005B030BD02F012F9417C01F0DDFD0446B5
:101AC0000028F4D002F00AF901F03CFDB1EE400A22
:101AD00085ED000AEBE7000090ED007ADFED0F7A6C
:101AE000B0EEC77AB4EEE77AF1EE10FA14D590EDC5
:101AF000017AB0EEC77AB4EEE77AF1EE10FA0BD5C0
:101B000090ED027AB0EEC77AB4EEE77AF1EE10FA11
:101B10004CBF0120002070470020704700000034B7
:101B200010B5FEF7A9F8044658B190F84E11FEF72B
:101B300075F830B194F84E112046BDE81040FEF71C
:101B400071B8002010BD000038B50D460DF040F909
:101B50000446FEF709FA022881BF94F8C402B023B4
:101B600003FB0040D43089BF07C8002085E8070088
:101B7000012038BD2DE9F0432DED028B8FB00368B5
:101B80000025DB6C0395049505950695029502A941
:101B900004469847064638B1FFF7BCFEDDED027AF1
:101BA00027EE800A8DED020A0DF012F9FEF7DCF93E
:101BB0000746002E50D0DDED027AD4ED646A94ED34
:101BC000657A23680B9527EE877A67EEA67A8DED06
:101BD000097ACDED0A7A0C950D959B6C0BA92046E0
:101BE00009AD98470BA9284616F038F8012F8DED5E
:101BF000030ACDED040A40F2B3800DF0E9F890F845
:101C0000C432DFED5B7AB02505FB030090ED308A2E
:101C100028EE278AB0EE480A71F0E2F9F0EE408A29
:101C2000B0EE480A71F032FBCDED0B8A8DED0C0A57
:101C30000DF0CEF890F8C43205FB030090ED2F0AAA
:101C40000BA816F02BF809AD8DED050ACDED060AAF
:101C500005A896BB03C885E00128CED89DED020AF1
:101C6000B5EEC00AF1EE10FA7FDD07AED4F894218C
:101C7000D4F8903107923046089316F02DF8236877
:101C80000B950C950D959B6C0BA920469847DDEDA7
:101C9000077A9DED0B7A77EE877A9DED0C7ACDED84
:101CA000077ADDED087A77EE877A09ABCDED087A11
:101CB00096E8030083E8030049E0236993ED000AF6
:101CC000B7EE008A38EE408A15F0E8FF04F5BC79DB
:101CD0008DED090A4846B0EE480ACDED0A0A15F026
:101CE000DDFF0BA92846CDED0C0A8DED0B0A15F092
:101CF000B5FF04F5C47603AFC4ED5F0A314684ED49
:101D00005E0A384615F0BAFF04F5C0788DED090A71
:101D10004046B0EE480ACDED0A0A15F0BFFF0BA908
:101D200028468DED0B0ACDED0C0A15F097FF97E8CC
:101D3000030084ED600AC4ED610A86E803004946A9
:101D4000404615F08BFF8DED090ACDED0A0A9DED99
:101D5000090ADDED0A0A0FB0BDEC028BBDE8F08385
:101D6000DDE9030185E80300F1E709950A95EEE74F
:101D700035FA8E3C10B590F84213044604F082F810
:101D80007C23C0B203FB0044D4F8A00010BD0000C7
:101D9000044B026F1B68DB6A5A60426F9A60826F65
:101DA000DA607047CC250020F0B58FB0044613F000
:101DB000D5FB002302930393049390F8121301AB15
:101DC00002AA054612F0FEFB04F19407D8B39DED7C
:101DD000010AB5EEC00AF1EE10FA34DD02A816F0E1
:101DE000D3F804F1B00684ED2C0AC4ED2D0A84ED7D
:101DF0002E1A3946304616F0D7F804F17C013046E9
:101E000016F086F804F1880105A88DED050ACDEDE0
:101E1000060A8DED071A16F07BF808A88DED080A62
:101E20009DED010ACDED090A8DED0A1A16F09CF818
:101E30000BA904F128008DED0B0ACDED0C0A8DEDF8
:101E40000D1A14F03BFD95F812030C2303FB005010
:101E5000394600F5117016F05BF884ED2C0AC4EDDC
:101E60002D0A84ED2E1A0FB0F0BD00002DE9F047C9
:101E7000824B00251F682DED028BC0F89C50C0F8E6
:101E80009850C0F89450C0F88450C0F88050C5678E
:101E9000C0F89050C0F88C50C0F88850C0F8B850C6
:101EA000C0F8B450C0F8B0500446F86A03688AB06D
:101EB0005B680E46984704F12809002854D052F078
:101EC000F5F942F20F7398424ED8FB6A9FED6C8A87
:101ED00093ED010A84ED1C0AD3ED020AC4ED1D0A3C
:101EE00093ED031A484684ED1E1A14F0DBFB3CF018
:101EF000B1FDD4ED1E7A67EE887A054617EE900A9A
:101F0000FAF7FAFAD4ED1D7A67EE887ACDE9040182
:101F100017EE900AFAF7F0FAD4ED1C7A67EE887A99
:101F2000CDE9020117EE900AFAF7E6FA554ACDE933
:101F300000010621284635F0BDFF94ED1E8AB0EE63
:101F4000480A71F04DF884ED650AB0EE480A71F068
:101F50009DF984ED640A52F0A9F9C4F864010AB04D
:101F6000BDEC028BBDE8F087A6B194ED1C0AB4EE7F
:101F7000400AF1EE10FA0DD6D4ED1D0AF4EE600A17
:101F8000F1EE10FA06D694ED1E1AB4EE411AF1EEF7
:101F900010FA52D713F0E2FA90F813334FF00C0A0C
:101FA0000AFB030303F5C473074693E8070007AE73
:101FB00086E807004FF01508B2EE028AF2EE068AB4
:101FC000304616F0CFFBB4EEC80AF1EE10FA38D561
:101FD00008F1FF3818F0FF083CD1304616F0C2FB7C
:101FE000F1EE047AB4EEE70AF1EE10FA43DD9DED6E
:101FF000090ADDED087A9DED078A20EE000AA7EEBA
:10200000A70A71F059FBF0EE400AB0EE480A71F0F1
:1020100009FADDED090A84ED1D0A9DED080AF1EECD
:10202000600AB1EE400A71F0FDF984ED1C0A9FEDE3
:10203000161AD4ED1D0A94ED1C0A484614F032FB22
:102040007BE7304616F08EFBB4EEE80AF1EE10FAAC
:10205000BEDCC2E7384612F077F9384612F03CFA97
:1020600097F813330AFB037303F5C47393E807006F
:1020700086E80700A4E725676567D8E7CC25002038
:10208000E02E65428CDB0808000000000021FFF70D
:10209000EDBE000037B5044608461546019116F01E
:1020A00061FBB7EE007AC7EE007AB4F8D030019841
:1020B0000133A4F8D03094ED337A37EE277A84EDEB
:1020C000337AB0EE007AF4EEC77AF1EE10FA06D564
:1020D000B6EE007AF4EEC77AF1EE10FA0DDC9FED61
:1020E0000E7AF4EEC77AF1EE10FA13D59FED0B7A63
:1020F000F4EEC77AF1EE10FA0CDDB0EE670A15F0D7
:1021000033FF012085ED000AC5ED010A85ED021AB5
:1021100003B030BD0020FBE700247449BD3786358D
:1021200070B52DED028B00F1280600F134058AB060
:1021300029460446304615F093FFB6EE008A20EE9D
:10214000088A2846B0EE480A15F00EFF07A9304667
:10215000CDED080A8DED091A8DED070A15F0EEFE9A
:1021600030468DED010AB0EE480ACDED020A8DED44
:10217000031A15F0F9FE07A928468DED070ACDEDE3
:10218000080A8DED091A15F0D9FE04A901A88DEDF4
:10219000040ACDED050A8DED061A15F075FF3246DD
:1021A00001A920468DED070ACDED080A8DED091A2B
:1021B000FFF770FF58B952F079F80121C4F86001B7
:1021C0002046FFF753FE0AB0BDEC028B70BD2A46D5
:1021D00004A92046FFF75EFF0028ECD004F140027E
:1021E00007A92046FFF756FF0028E4D0EBE70000E0
:1021F00030B52DED028B0D4683B091F842130446A5
:10220000284603F03FFEC1B27C2000FB0151903113
:1022100004F1280014F0D6F868468DED000ACDEDE3
:10222000010A15F0CBFDDFED1C7AB4EEE70AF1EE02
:1022300010FA05D59FED190A03B0BDEC028B30BD35
:10224000684615F00DFE684615F092FD0028F1D1A4
:10225000284694ED428A03F089FFF0EE400AB0EE82
:10226000480A13F07BFD80B9284603F07FFF84ED18
:10227000420AB0EE408A70F0B3FE84ED430AB0EE3D
:10228000480A71F003F884ED440A04F58671684643
:1022900015F04CFDD0E700BF000000340000000046
:1022A0009FED0C7AB4EEC70AF1EE10FA0BD4DFED15
:1022B0000A7AB4EEE70AF1EE10FA07DCC0EE077A0C
:1022C000B0EE670A7047F7EE007AF9E7F2EE047AAB
:1022D000F6E700BFF3665F3F58A00B4108B51C301E
:1022E00015F06CFDF1EE007AB4EEE70AF1EE10FAAB
:1022F0009DBFF1EE027A37EEC00ADFED047A9FED62
:10230000040A98BF20EE270A08BD00BFCDCC4C3E82
:10231000CDCCCC3D08B5836993F9000038B10CF001
:1023200057FDFDF721FE012894BF0020012008BDC4
:10233000F8B52DED028B054604F08AF904F086F815
:102340000446B8B3FFF7F8F890F8093393B328467A
:10235000FFF7E0FF064668B30CF03AFD90F8C43290
:10236000B02707FB030090ED2F7AF0EE087AB4EE69
:10237000E77AF1EE10FA1DD495ED1E8A0CF028FDD7
:1023800090F8C432DFED1E7A07FB030090ED300AAF
:1023900098EE270A13F066FDDFED1A7AB0EEC00A58
:1023A000B4EEE70AF1EE10FA08DC51F07FFF344694
:1023B000C5F85001BDEC028B2046F8BD05F5AA70AA
:1023C00016F0D0F9B0EE408A0CF002FD90F8C4325D
:1023D0009FED0D7A07FB0303D3ED2F7A67EE877A23
:1023E000B4EEE78AF1EE10FADFD551F05FFFD5F8D1
:1023F0005041001BB0F5FA6F8CBF00240124D9E7CF
:10240000E02E654200003442CDCC4C3F10B50A4B63
:102410001B68DB6A93F89C3004465BB951F046FFB9
:10242000D4F86431C01A44F61F6398428CBF002070
:10243000012010BD0020FCE7CC250020F8B52DEDD3
:10244000068B04460CF0C4FC054604F001F9064670
:1024500006F0EAFD002840F0AA802046FFF768FF5A
:10246000002800F0A7803046FFF784FCD4F8DC3069
:10247000984200F018813046FFF77CFCD4F8DC303D
:10248000DFED8E7AC31A08EE903AF8EE688A30468D
:1024900068EEA78AFFF76EFC94F8BC30C4F8DC0045
:1024A000F3B9304603F0E4FFD0B104F1280796F801
:1024B00042233946304603F05DFED4ED1D0AB0EEEE
:1024C000401A384694ED1C0A14F0ECF80023C4F8C6
:1024D0009030C4F88C30C4F88830012384F8BC30C4
:1024E00020463146FFF784FE95F8C40205EB00153F
:1024F000B0EE408A2B6FC4F8E03004F1B000D4EDA8
:10250000129A16F02FF96368DFED6D7A93ED007A79
:10251000B4EEE77AF1EE10FA68EE299AB0EE40AA2E
:1025200001D5C3ED007A2046B0EE4A0AFFF7B8FEA7
:10253000636820EE299A93ED000A29EE009AFFF7CE
:10254000CDFE29EE009A204684ED249AFFF75EFF27
:1025500038B1D4ED247AB2EE007A67EE877AC4ED12
:10256000247AF0EE007AF4EEE78AF1EE10FA10D554
:10257000DFED547AB4EEE7AAF1EE10FA09D5DFEDFB
:10258000527A69EEA79AD4ED2A7AE9EEA87AC4EDD8
:102590002A7A9FED4E0A94ED367ADFED4D7AB0EE51
:1025A000C88A28EE008AA7EE278A84ED368ABDEC19
:1025B000068BF8BDFEF7C0FF90F80933002B72D0F0
:1025C0002046FFF7A7FE00286DD095F8C42205EB42
:1025D0000213196FD4F8E0308B4264D0B02606FBAA
:1025E000025292ED2F7AF0EE087AB4EEE77AF1EE2D
:1025F00010FA58DBCB1AC4F8E01008EE903A95F8C0
:10260000C4329FED341A94ED1E0ADFED337A06FBD7
:102610000353D3ED309A69EE819AF8EE688A39EE69
:10262000C00A68EEA78A13F087FCB0EE409A70F0FB
:102630002DFE94F8BC30B0EE408AF3B1F3EE047A8C
:10264000F4EEE78AF1EE10FA17DC95F8C40206FB07
:10265000005595ED2F7AF2EE027AB4EEE77AF1EEBC
:1026600010FAFFF64AAFDFED1D7AB0EEC99AB4EE6C
:10267000E79AF1EE10FAFFF640AF9FED198AD4ED1C
:102680001D0A94ED1C0AB0EE691A04F1280014F03A
:1026900009F8012384ED248A84ED238A84ED228ABB
:1026A00084F8BC3029E7BDEC068B04F188009FED6F
:1026B0000D0ABDE8F84015F0ABBC00BFBD3786354C
:1026C000CDCC4C3DC2B8B23E0AD7233CCDCC4C3E1B
:1026D000CDCC4C3F35FA8E3C6F12833A1904863FBD
:1026E00000000000EC51783F30B50C2303FB0101E2
:1026F00001F1C003144693E807008BB004AD85E8F0
:10270000070094E8070083E807002846FFF7E4F98C
:1027100007AB58B194E8070083E807009DED070A6E
:10272000DDED080A9DED091A0BB030BD95E80700F4
:10273000F2E70000F0B52DED028BD0F818318B6078
:10274000D0F81C31CB6085B004460D4601F0C6FAC6
:1027500006460CF03DFBA36993F90030022B0746B7
:102760004BD1FDF701FC022847D997F8C432B022BB
:1027700002FB0373D3F8B0100022284602F04AFF90
:10278000D4ED4A0A94ED490A284603F0CDF994F8AD
:102790002C3163B351F08AFD9FED228A97F8C41261
:1027A0008DED018A01AA064638460BF095FBD4F858
:1027B00020019FED1D0A361A07EE906AF8EE677A3F
:1027C0004FF4876027EE800AB6EE001AF0EE480A52
:1027D00013F0C6FBDDED017A30EE270A04F1F000BC
:1027E0008DED010A15F05AFA284603F09DF994F888
:1027F0002C0105B0BDEC028BF0BD707C242303FBE3
:10280000006696ED0B8AFEF797FED0ED9C7A9FED61
:10281000077AF8EEE77AE8EE077AFDEEE77A17EE48
:10282000901AA9E7000000006F12833A0000C84226
:10283000F8B5036F0B60436F4B60836F8B6000F1E3
:102840004C050E46074601F10C040FCD0FC40FCD09
:102850000FC42B68236007F1B00207CA06F13003EA
:1028600083E8070007F1940207CA06F13C0383E8F6
:10287000070007F11C0207CA06F1480383E80700B6
:1028800006F160013846FFF755FF86F87000F8BD85
:1028900030B589B0044668460D4602F0B5FE69467B
:1028A0002046FFF797F818B90024204609B030BD3C
:1028B00004A802F0A9FE204604A9FFF73BFF044646
:1028C0000028F1D004A9684603F086F885ED000AD7
:1028D000C5ED010A85ED021AE7E700001FB50023E8
:1028E0000C4601A9019302930393FFF7D1FF08B1AE
:1028F000039B236004B010BD30B585B001AD00234B
:102900000C462946019302930393FFF7C1FF034648
:1029100018B195E8030084E80300184605B030BDFF
:10292000F8B506460F461546FDF7A6F9044690B1E0
:102930003946FDF773F970B120463946FDF772F953
:10294000044640B1FDF798F93946FDF76DF985ED7C
:10295000000A2046F8BDFEF7EFFD90F8083343B1BA
:102960003046FFF7D7FC044618B1D6F84C312B603F
:10297000EFE7D6F84C312B600024EAE770B52DED77
:10298000048B1646FFF7CCFF054670B3FEF7D4FD67
:1029900090F930424CB30CF01BFAFDF7E5FA012830
:1029A00023D9E4B207EE904AB8EE678A0CF010FA29
:1029B00090F8C43296ED009AB02202FB0300D0EDED
:1029C0002F8AFEF7A7FF38EE281A78EEC80A40F2E1
:1029D000614029EE000A13F0C3FAB0EE408AFEF718
:1029E00099FFC8EE007AC6ED007ABDEC048B28464C
:1029F00070BD000008B503F02BFEBDE8084003F0F1
:102A000025BD000010B5044615F05AFB50B904F17D
:102A10000C0015F055FB28B904F11800BDE8104072
:102A200015F04EBB012010BD38B500F12805044655
:102A30002846FFF7E7FF28B120460121BDE83840CE
:102A4000FFF714BAD4ED107AB7EE007AF4EEC77A35
:102A5000F1EE10FA06D5BFEE007AF4EEC77AF1EE89
:102A600010FA12DC2046FFF75BFB2846FFF7CAFF8F
:102A70000028E1D1D4ED107AB2EE047AF0EEE77AD4
:102A8000F4EEC77AF1EE10FAD6DC38BD10B5044684
:102A900015F068FE2046BDE8104015F0CDBA0000E4
:102AA0002DE9F04F2DED048B9FEDC48A95B00446BF
:102AB000F0EE408A8DED028A8DED038A8DED048A59
:102AC000FFF7BCFC12F04AFD0023054695F879217A
:102AD000012AA8BF012293423FD20021284611F0CB
:102AE0009FFB01230028F1D008AB0BAA0021284648
:102AF0008DED0B8A8DED0C8A8DED0D8A11F0BCFDEC
:102B00009DED080AB5EEC00AF1EE10FA23DD0BA820
:102B100015F03AFA11A904F128008DED110ACDED56
:102B2000120A8DED131A13F0F1FB0EA88DED0E0AAB
:102B3000B0EE680ACDED0F0A8DED101A15F014FAFB
:102B400011A904F1E4008DED110ACDED120A8DED0D
:102B5000131A15F029FA0123B8E795F813130C237B
:102B600003FB015104F1280B01F5C471584613F021
:102B7000CDFB84ED070A94ED3F0AC4ED080A70EE20
:102B8000288A84ED091AC4ED3F8A0CF021F9064623
:102B9000FEF7D2FC90F8093300932046FFF7BAFB0A
:102BA00080B13046FDF7E0F902280BD996F8C4222F
:102BB0006169B02303FB026391F9001093F8D2001E
:102BC00088425FDA94ED3F7ADFED7D7AB4EEE77A02
:102BD000F1EE10FA5DD4D4ED538AFEF7A1FF38B1BF
:102BE000FDF74AF890F84E11FDF71EF8F0EE408A16
:102BF000236C626BA16A1393B0EE680A11A812925B
:102C0000119115F0B1F904F5AA7102A88DED020A2F
:102C1000CDED030A8DED041A15F0C6F951F046FB0F
:102C20000023074684F814312046FFF773FB002881
:102C300065D096F8C422B02302FB033232445268B6
:102C4000C4F8182196F8C42202FB033333449B686E
:102C5000C4F81C3151F02AFB0123C4F8200184ED93
:102C6000498A84ED4A8A84F82C31D4F80031002B4B
:102C700058D102AB93E80700C4F80071F03484E83F
:102C8000070006E006EB0212176FD4F80021BA42E3
:102C900004D115B0BDEC048BBDE8F08FD43393E8BC
:102CA000070094F814310DF1080C8CE807001BB9EB
:102CB00004F1F00383E807000123604684F814312F
:102CC00004F5AA7115F03AF911A904F14C008DED43
:102CD000110ACDED120A8DED131A13F045FBB5EE76
:102CE000C00AF1EE10FA8DED110AD8BF9FED330A3C
:102CF000CDED120A8DED131A84ED530A94E794ED8D
:102D00003F7AD4ED497ADDED026AE6EE877ADDEDB1
:102D1000036AC4ED497AD4ED4A7AE7EE267AC4ED27
:102D20004A7AA2E7D4ED3F7A224B8DED058AF5EE83
:102D3000C07AF1EE10FA8DED068A0793A9D99FEDBE
:102D40001E7A94F8143167EE877AB7EE007AC7EEF0
:102D5000279A1BB9009B002B00F0AA80E36804F1BE
:102D6000F00102A8D3ED008A15F0E8F869EEA88A10
:102D70008DED110A11A8B0EE680ACDED120A8DEDA5
:102D8000131A15F0F1F80EA905A88DED0E0ACDED78
:102D90000F0A8DED101A15F007F905A8FFF776FE5A
:102DA00005A815F0A7F9D8B151F080FAC4F8600170
:102DB0006FE700BF000080BF0AE81C410000000070
:102DC000CDCC4C3ECDCC4C3FCDCC4C3D920A06BF39
:102DD000920A063FC2B8B23E728A0E3C5B82183934
:102DE000012301930023CDE90833CDE90A33CDE96E
:102DF0000C335FED0E8A4FF0FF3A04F1E40895F8CA
:102E00007921012A1046A8BF0120834257D201230D
:102E1000002AFAD095F835130029F6D0B0EE690AE9
:102E2000404615F0F5F8019B0DF12C09002B41D01F
:102E3000424600212046FFF757FC8DED0B0ACDEDF1
:102E40000C0A8DED0D1A4846FEF746FE70BB48464B
:102E5000FFF71CFE484615F04DF938BB05A948465A
:102E600015F012F9484605A98DED080ACDED090ABD
:102E70008DED0A1A15F0F4F808A8B0EE409A15F096
:102E800071FCBAF1000F06D1F4EEC08AF1EE10FA2F
:102E9000D8BFB0EE680AB5EEC09AF1EE10FAF7EEC0
:102EA000008A58BFF0EE408A4FF0000A0123A6E7DF
:102EB000009B96E798E8070089E80700C3E7BAF1A6
:102EC000000F7FF471AF002384F804312046FFF730
:102ED0002FFA38B12046FFF71DFA002840F025816F
:102EE0008DED0A8A95F8123395F878219A4240F2CE
:102EF00033812B4493F83433002B00F02D8195F867
:102F0000133395F879219A4240F226812B4493F8A5
:102F10003533002B00F0208108A9584613F024FA1D
:102F20008DED080ACDED090A8DED0A1A08A815F0F5
:102F3000C7F8002840F0178108A815F0DBF8002832
:102F400040F011815FED627A94ED357A68EEA78AE0
:102F50005FED647AE7EE278A04F1B000C4ED358AAC
:102F600015F000FCA3685FED687A93ED007AB4EE8B
:102F7000E77AF1EE10FAF0EE408A00F1F880204690
:102F8000B0EE680AFFF78CF908A814F0EDFFA3680B
:102F90008DED110ACDED120A8DED131A93ED000A95
:102FA00011A814F0E1FF204684ED1F0AC4ED200AA9
:102FB00084ED211AFFF72AFA28B1B2EE000A04F1D3
:102FC0007C0015F025F8009BB3B33046FCF7CCFF2E
:102FD000012831D996F8C402B02303FB006696EDB0
:102FE0002F7AF0EE087AB4EEE77AF1EE10FA23D5F4
:102FF00095F813030C2303FB005595ED627AF1EE6F
:103000000C7AB4EEE77AF1EE10FA15DBD4ED1D7A06
:103010001FED927AF4EEC77AF1EE10FA0CDD1FED97
:10302000947AF4EEC77AF1EE10FA05D5B6EE000AFE
:1030300004F17C0014F0ECFF5FED9A7AF4EEE78A7D
:10304000F1EE10FA22D51FED9C0A08A814F08CFFAF
:103050000EA88DED0E0A94ED3F0ACDED0F0A8DED11
:10306000101A14F081FF11A904F1A0008DED110ACE
:10307000CDED120A8DED131A14F096FFD4ED2B7AD4
:1030800094ED3F7A77EE877AC4ED2B7A94ED2B7A24
:10309000F1EE047AB4EEE77AF1EE10FA3BDB12F0CF
:1030A0005DFA5FEDB27A94ED2B1A94ED280A21EEC9
:1030B000271A40F2C530F1EE410A8DED011ACDED2F
:1030C000000A12F04DFF9DED011ADDED000A84EDBE
:1030D000280A40F2C63094ED290A12F041FF9DED16
:1030E000011ADDED000A84ED290A40F2C73094EDA3
:1030F0002A0A12F035FF04F1A00184ED2A0A04F136
:10310000940014F051FF84ED2A8A84ED298A84ED1D
:10311000288A84ED2B8A0023C4F8E430C4F8E83010
:10312000C4F8EC3084ED3F8AA3E5E368F7EE000ACB
:1031300093ED000A12F012FE00283FF4D1AE94ED98
:103140001C0AB0EEC00A70F0A1F8DDED0A7A27EE95
:10315000800A8DED0A0AC5E68DED0A8A8DED098A91
:103160008DED088AE2E62046FFF75EFC1CE6C3ED23
:10317000007A04E72DE9F04D2DED048B9EB0044656
:1031800012F0ECF9D0EDC87A90ED618AF4EE487A4D
:10319000F1EE10FA48BFB0EE678ADFED5C7AB4EE6C
:1031A000E78AF1EE10FA0EDD0023C4F8E430C4F82B
:1031B000E830C4F8EC300023C4F8FC301EB0BDEC9D
:1031C000048BBDE8F08D2046FEF7EEFD2046FEF7AD
:1031D000A7FFB0EE480A2046FFF762FC2046FFF743
:1031E00023FCFEF7A9F914AD00F5347204F12801AF
:1031F00014A813F009F90FCD04F14C060FC60FCD3A
:103200000FC62B68336004F1740204F1780304F1F3
:10321000700104F14C0013F0A5FA94ED1E8AB0EE93
:10322000480A6FF0DDFE84ED650AB0EE480A70F0E2
:103230002DF8204684ED640AFEF7AAFDFEF77CF91E
:1032400004F5B471FDF77EFF51F030F8D4F89831F1
:10325000C31A632BB2D9C4F8980132F0A7FE9FEDD0
:103260002C9A054651F02AF8D4ED1C7A67EE897A3B
:10327000074617EE900A0E46F9F73EF9D4ED1D7A8F
:1032800067EE897A824617EE900A8B46F9F734F991
:1032900094ED1E0A20EE090A41EC180B12F0CCFD49
:1032A000D4F85C0110EE108AF9F726F9CDE9120185
:1032B000D4F85801F9F720F9CDE91001D4F85401F8
:1032C000F9F71AF9CDE90E01D4F8D800F9F714F995
:1032D000CDE90C01D4F8D400F9F70EF9CDE90A01D3
:1032E0004046F9F709F90B4B01930B4B0093CDE9DD
:1032F00008018DED068BCDE904ABCDE90276074BD5
:10330000074A0849284632F0DDFB57E7CDCC4C3E52
:10331000E02E6542F1DB0808FBDB0808B8DB080893
:10332000C2DB080844DA080808B52DED048BB0EEBE
:10333000609AF0EE408A00F011F9B0EE408A89EE12
:10334000280A70F0D9F8DFED0B7A20EE270A70F02A
:103350006BF8DFED097A38EE278ADFED087A28EE80
:10336000278AF7EE007A37EEC00A28EE000ABDEC95
:10337000048B08BD41D3423E33938843A1D81943FF
:10338000FFF7D2BF08B52DED048B9FED189AF0EE34
:10339000E07AF4EEC97AF1EE10FAF0EE408AB0EE7F
:1033A000608A1ED400F0DAF8DFED117A9FED117A11
:1033B00070EE277A9FED100AE8EEC77A9FED0F7A3C
:1033C00027EE800AC8EE007A87EE270AB4EEC90A13
:1033D000F1EE10FA05DBBDEC048BBDE8084070F09F
:1033E0006BB9BDEC048BB7EE000A08BD00000034D9
:1033F00033938843F4FDD43B48A18F43CDCC9C3F0D
:10340000427CD0ED257A242101FB020292ED0B0AC9
:10341000D2ED090A30EE270AFFF7B4BF38B52DED1B
:10342000088BDFED21AA9FED21AA9FED21BA054669
:10343000B0EE409AF0EE609AB0EE408A1524013C5E
:10344000A4B25CB3F0EE490A2846B0EE480AFFF792
:103450006BFFF0EE490A70EE698A284638EE2A0AB8
:10346000FFF762FFB0EEE87A70EE697AB4EECA7ADE
:10347000F1EE10FA77EEE87A10D468EEAA8A40F2FC
:10348000631088EEA70AB0EE4B1A38EE400AF0EE51
:103490004A0A12F065FDB0EE408AD0E7B0EE480A65
:1034A000BDEC088B38BD00BFCDCCCC3D0AD7233C4A
:1034B00000247449002343608360C3600361436157
:1034C0008361C361002380F82030704790F820208A
:1034D000531CDBB2062B80F8203000EB820288BF41
:1034E000002382ED010A88BF80F820307047000079
:1034F0004FF0FF3310B543610E4BC0F8A8300023E6
:10350000044680F8C830A830FFF7D4FF0A4BC4F84F
:10351000A83004F5867050F073F8084B08491C6019
:1035200020462EF017FDD4F89030C4F89430204691
:1035300010BD00BF18DE080828DE0808EC5900207E
:10354000C0DE080808B5A83033F062FDDFED027A6E
:1035500020EE270A08BD00BF00007A4490ED3C0A27
:10356000DFED057AB0EEC07AB4EEE77AF1EE10FA4C
:1035700048BF90ED3D0A70470000003473B5D0F8A5
:10358000A43004460E4663B150F090FED4F8A43047
:10359000C01A42F20F73984203D894ED280A02B081
:1035A00070BD114B1D687DB195F84E112846FCF792
:1035B00039FB48B195F84E1101AA2846FCF728FBC3
:1035C00010B19DED010AEAE7242101FB064494EDC8
:1035D0000A0ADFED067AB4EEE70AF1EE10FA58BFF8
:1035E000B0EE670ADBE700BFE459002000000C42A0
:1035F00008B561B10378022B02D9064850F024FEC9
:103600005A1C027000EB83004160012008BD08468F
:10361000FCE700BFE0DC08082DE9F84305460E464C
:103620009146002400F13C082B78A34211DD0023D1
:103630004A46314601200EF049FF242363430746E2
:10364000002158F803000EF051FF874204D00134E6
:10365000EAE70020BDE8F8830120FBE7054B1B6883
:103660002BB141694A1C02D0184632F069BC0020D7
:10367000704700BF945C002002290BD8242303FB71
:10368000010191F8390030B191F83A0018B191F880
:103690003B007047002070472DE9F047044650F08A
:1036A00005FED4F8F86042F21073861B9E4288BF74
:1036B000C4F8F80000274FF0240942F2107A237C66
:1036C000FDB2AB421CD929462046FFF7D5FF70B1A9
:1036D00009FB054898ED0D0AD8ED097AD4ED250AC5
:1036E00030EE270A2046FFF799FE88ED0C0A564572
:1036F00004D909FB054030302EF004FE0137DEE727
:10370000617C2046FFF73AFF84ED3D0ABDE8F08773
:1037100070B5044686B050F0C9FDD4F89830C31A8D
:10372000B3F57A7F05464FD3344B94ED257A1B6869
:10373000DFED336ADB6AD4ED247A93F89C60B0EE57
:10374000C76AB4EEE66AF1EE10FA32D5B0EEE76A77
:10375000B4EEE66AF1EE10FA2BD502A801F054FFA0
:1037600096BBFDF7E9FE02A9FDF7ECFC60B3DDEDC9
:10377000037A9FED247AF8EEE77A67EE877AC4ED54
:10378000257AC4F89850FDF7D7FEFDF7C3FA204616
:10379000FFF782FF3BF05EF90546D4F89400F8F796
:1037A000ABFE194ACDE900010621284634F082FB20
:1037B0000AE037EE676AF7EE005AB0EEC66AB4EE7A
:1037C000E56AF1EE10FA01DC06B070BDB0EEE76A12
:1037D000B4EEE66AF1EE10FAF6D4002ECFD0204611
:1037E000903080ED007A2EF08DFD3BF033F9074AE2
:1037F000012106B0BDE8704034F05CBBCC25002050
:10380000000000340AD7233C21DD0808FCDC08084E
:10381000F0B52DED048B85B004464FF4537200F5DE
:10382000867103A80EF0DEFFD4ED227AD4ED236A70
:103830009FED796A637C37EEE67A2422B0EEC77A90
:10384000B4EEC67AF1EE10FAC1BF9FED747A67EE5E
:10385000877A9FED737AE6EE877A02FB03430025B1
:10386000C4ED237A93F839602378E9B28B4206D904
:1038700004EB81030135586851F0BEFFF4E7DFED3A
:10388000698A9FED698A9FED699A0027237CFDB2C2
:10389000AB4264D9242303FB054393F83920002A63
:1038A0005BD0D3ED0C7AF4EEE87AF1EE10FA0BDB94
:1038B000F4EE677AF1EE10FA06D6F0EEE77AF4EE5F
:1038C000487AF1EE10FA04DD242303FB05435A6A1B
:1038D0001A63242303FB0543D3ED090AD3ED0D7AC4
:1038E00093F8382070EEA70AA2B993ED0C0A20468F
:1038F000FFF746FDD4ED257A30EE670AB4EE400AB4
:10390000F1EE10FA16D7242303FB0545002385F8B2
:103910003A3022E0012A09BFD3ED0C7A93ED0B0A6D
:1039200077EEE00AD4ED3B7A04BF80EE897A87EE29
:10393000270AE3E7F0EEC07AF4EE487A2423F1EEAA
:1039400010FA03FB0545E1DC012385F83A30D4ED9C
:10395000237A37EE800A85ED0B0A013796E7627C01
:1039600020461146FFF788FE48B1242101FB0242A0
:1039700092ED0B0AD16904F1A80033F029FB94F908
:103980009C10277C002907DBB94205DACAB2114630
:103990002046FFF771FE68B900226274D5B2AF42CB
:1039A00009D929462046FFF767FE01320028F5D0E5
:1039B000657400E062742046FFF7AAFE2046FFF718
:1039C0004DFE10B1204652F01DF8637C242505FB06
:1039D000034393F83930B34216D032F0E7FA4FF68A
:1039E000FF7132F0ADFA78B1607C05FB004494F8C9
:1039F0003930002B14BF00220422019232F0D6FA93
:103A0000019A122132F02EFA03A80EF00DFF05B034
:103A1000BDEC048BF0BD00BF0AD7233C0AD7A33C02
:103A200048E17A3F00000034FFFF7F7F0020194605
:103A30002DE9F04F0446007C0F4687B004F13A03AD
:103A400000220121D5B2A84203F1240305D903F8CD
:103A5000231C03F8241C0132F4E76F4B1E68F06A44
:103A600003685B68984740B13AF0F4FF6B4A06215F
:103A700007B0BDE8F04F34F01DBA3AF0EBFF684AEA
:103A8000062134F017FA002303A904F188000393F8
:103A90002EF0EEFF0A2550F009FC80462046FFF785
:103AA000B7FE50F003FCA0EB0800B0F5FA7F02D996
:103AB0005C4800F039FFB06A03680A215B689847E8
:103AC000617C2046FFF7D8FD0028E7D0B06A036884
:103AD00064215B68013D984715F0FF05DBD1524B2F
:103AE00005951B888DF80650CDE90355ADF80430D7
:103AF000052550F0DBFB80462046FFF789FE50F09D
:103B0000D5FBA0EB0800B0F5FA7FD1D8617C204648
:103B1000FFF7B2FD0028EFD094F810B00DF10C08BB
:103B2000A14601AA4FF0000A5FFA8AF18B4516D927
:103B30002046FFF7A1FD50B1D8ED007A99ED097A42
:103B4000137877EE877A0133C8ED007A13700AF1A3
:103B5000010A08F1040809F124090132E4E7B06A16
:103B6000036864215B68013D984715F0FF05C0D1EB
:103B7000A9464FF02408237C5FFA89F6B34226D980
:103B800006AB334413F8143C33B908FB064686F8F9
:103B90003B3009F10109EEE7002FFAD007EE903A29
:103BA00006AA02EB8602F8EEE77A12ED030AD4EDDC
:103BB000250A204680EE270AFFF730FC08FB064066
:103BC00002A930308DED020A2EF052FFE1E7617C50
:103BD000DFF85C902046FFF7D1FC002684ED3D0A1B
:103BE0004FF02408237CF7B2BB420FD908FB0743F0
:103BF00093F83B3043B13AF02DFF7B1C4A46062137
:103C000034F058F90135EDB20136EBE70DB907484C
:103C10004FE707B0BDE8F08FCC2500203CDD080859
:103C200067DD08087DDD0808F4980808B9DD080894
:103C300097DD080808B5037C022B02D9034850F031
:103C400003FB5A1C0274184608BD00BFD8DD0808E3
:103C500038B5057C02460024E1B28D4206D91046F3
:103C6000FFF70AFD01340028F6D138BD281E18BF21
:103C70000120FAE770B50D4609780729044606D8F1
:103C8000027E437E22B901228A401343437670BDEF
:103C9000002BFCD000262278F3B29A42F7D904EB2D
:103CA0008303294658680368DB6898470136F2E7C2
:103CB00037B50D460192FFF7CBFF0199044630B9A5
:103CC0000448054B00682A46C06A0EF06BFF204688
:103CD00003B030BDCC250020F3D80908014B18688B
:103CE000704700BFEC59002010B50446006810B1C1
:103CF00003685B689847204610BD000010B5044675
:103D0000006810B103685B689847204610BD00004A
:103D100070B5D0ED247A9FED427AF0EEE77AF4EEBA
:103D2000C77A0123F1EE10FA8AB00446037609D46B
:103D30009030002309A9059009932EF099FE05986B
:103D40002EF0E0FA0026E6632666C4F88460762248
:103D500031462046FFF760FC054600283BD0CDE900
:103D60000666079A0992002309A92046CDE9073380
:103D700051F0A6FC01462046FFF73AFC09A8FFF7E0
:103D8000BDFF08A8FFF7BAFF07A8FFF7ADFF15B101
:103D900006A8FFF7A9FF2378032B3FD0237C032B32
:103DA0003CD0D4F80031DA0403D5637E0BB901238B
:103DB00063760025637EEB40DB07EAB21AD4013557
:103DC000082DF7D123781BB1237C0BB163682BBB83
:103DD000144800F0A9FD144B1B68596804220B68B5
:103DE000CDE90102114A00921E680246762307A817
:103DF000B047B6E73820059201F0A2FE064618B19A
:103E0000059A214651F072FE31462046FFF7F0FB3D
:103E10002378032B02D0237C032BD0D10AB070BDB2
:103E200000000034ECDD0808CC250020801A0600D4
:103E300090F81835934207D902F59E7250F8220087
:103E400010B103689B6A1847002070472DE9F341C1
:103E500005466E4686E80C00134B45F8043B0446C5
:103E60000F4600F5C87828462C3500F085FCA8459B
:103E7000F9D196E8030004F21C53C4F8147583E8E2
:103E80000300089BC4F82435084920462EF062F848
:103E9000074B1A6812B1074850F0D6F920461C604B
:103EA00002B0BDE8F08100BFE0E10808A8E0080822
:103EB000F0590020ECDF08082DE9F041A2B00C46D3
:103EC00007A92DF01DFB002855D000210D220CA8BC
:103ED0000591ADF818100B9171F08AFC2B4B611C09
:103EE0001F68C9B20BAD0129F86A0A9546D1284B63
:103EF000062205A90EF056FE264B019305AB009352
:103F0000002411222946244BF86A8DF819400EF03E
:103F100049FE04AA0DF10F0128468DF83C40049497
:103F20002EF084FC38B31D49DFF86C80482210A8BD
:103F300071F014FC062610AC2268531E049AC2F3DA
:103F4000513202EB831223798DF82430A368019358
:103F500005AB00930892434611222946F86A0EF0F9
:103F600021FE0021B7EE000A07A82DF0CBFC013E90
:103F700004F10C04E0D122B0BDE8F0810091084BBF
:103F8000062205A90EF00EFEB6E700BFCC250020E4
:103F90007DCF08081DE0080817E00808F898080811
:103FA00010E008082DE9F74F90F818650446002E38
:103FB00051D17F2380F8283500F5C87500F59E683B
:103FC000071D5FFA86FA1822FF21284671F010FCBF
:103FD00085F857A097F92490B9F10A0F59D03DDC24
:103FE000B9F1040F0FDCB9F1020F0FDD442001F02D
:103FF000A7FD834620B13B462A46214651F002FEEA
:10400000C8F800B002E0B9F1090F36D0D8F80000C6
:1040100050B1E96DC5F8589031B1254B43F82610E1
:104020002EF0A6F92EF09CF958F8040B0AF10109BC
:104030005FFA89F940B103689B68984784F818953E
:1040400051462046FFF738FF0136092E05F160057D
:1040500007F12C07B5D103B0BDE8F08FB9F1190F06
:10406000D4D1482001F06CFD83460028C8D03B46DF
:104070002A46214652F03EFCC2E7382001F060FD9E
:1040800083460028BCD03B462A46214652F012FA0D
:10409000B6E7302001F054FD83460028B0D0CDF8BB
:1040A00000A03B462A46214652F0A6FBA8E700BFE7
:1040B000F459002090F818358B4283BF602303FB2E
:1040C000010090F8D50100207047000090F81835E5
:1040D0008B4283BF602303FB010090ED6A0A9FEDD2
:1040E000010A70470000000090F818358B4206D98D
:1040F00001F59E7150F8210008B151F017BF9FEDF6
:10410000010A70470000000010B490F818458C4276
:104110000A4614D901F59E7450F824407CB1E46835
:10412000246A640603D55DF8044BFFF7DDBF602108
:1041300001FB020393ED6A0A5DF8044B70479FEDA3
:10414000010AF9E70000000090F818358B420BD9FE
:1041500001F59E7150F8210038B1C3681B6A1A42FC
:1041600014BF0120002070470020704770B590F800
:104170001835934204460E46154601D8002070BDFE
:1041800002F59E7350F823000028F7D003689B695E
:1041900098470028F2D0602202FB0544D4F8AC31E5
:1041A0003360ECE770B590F81835934204460E463C
:1041B000154601D8002070BD02F59E7350F823000B
:1041C0000028F7D003689B6998470028F2D0602246
:1041D00002FB0544D4ED6C7AF4EE677AF1EE10FA46
:1041E000E8D6C6ED007AE6E770B590F81835934248
:1041F00004460E46154601D8002070BD02F59E7398
:1042000050F823000028F7D003685B69984700281E
:10421000F2D0602202FB0544D4F8B4313360ECE7FD
:1042200090F8183593420ED902F59E7350F823305A
:104230005BB1602303FB020292F8E40130B1D2F8D3
:10424000E0310B607047002070471846704700004F
:1042500008299DBF2C2303FB010040680020704704
:104260002DE9F04F4B4B2DED028B1B68DB6A93F869
:104270009C3089B00446002B00F08680DFF82CB11A
:104280009FED458A4FF0000994F818355FFA89F5DB
:10429000AB4279D905F59E7354F8230000285DD010
:1042A00003685B6B9847602303FB0543074693F85D
:1042B000D431834252D2032861D8DFE800F04F02A4
:1042C0005259364E4FF000083AF0C4FB94F81825C6
:1042D000AA4284BF602202FB05424FF0600105F153
:1042E000010301FB05458CBFD2F8A82118EE102A66
:1042F0008246D5F8B001CDE90632F8F7FDF8079A05
:10430000CDE904011046F8F7F7F8069B0096CDE9D1
:1043100002015A460421504633F0CCFD0123204AC5
:1043200084F8293585F8D471D372D4F824354BB389
:10433000002255B25957481C03D0414502F10102F1
:10434000F7D194F92835AB4208DBD4F82035D4F8FE
:104350001C0542463146984784F8285509F1010961
:1043600092E72C2303FB05430E4E93F92B80ABE71A
:104370002C2303FB05430C4E93F92C80A4E7002665
:10438000B046A1E71D46DCE709B0BDEC028BBDE8F5
:10439000F08F00BFCC2500200000000031E00808AD
:1043A000755A0020CEE2090828E0080840E0080815
:1043B00090F818358B4207D901F59E7150F821000D
:1043C00010B10368DB6918470020704708299CBFBB
:1043D000602303FB010000F5C870704790F81835A2
:1043E000934207D902F59E7250F8220010B103687B
:1043F0005B6A1847002070472DE9F04F002493B006
:1044000005460E46174621462F2206A8059405F5B7
:104410009E6971F0EDF905F1280A4FF02C0B05F5B6
:10442000F4730BFB04F259F8040B1AF90210E5B20D
:1044300030B951B90134092CF3D14FF0010813E020
:10444000602262439A58914212D01548154B006879
:1044500001930135EDB20095134BC06A32463946DF
:104460000EF0A0FB4FF00008404613B0BDE8F08FFF
:1044700005A93322039351F03BFE039B804605A917
:104480000028D7D1064801910135EDB200680095AA
:10449000054BC06A324639460EF084FBE4E700BFA4
:1044A000CC25002076E0080868E008082DE9F04FE8
:1044B000DFF88090DFF880A0DFF880B08DB006468E
:1044C000002796F81835FCB2A3422ED9602505FBCB
:1044D000046595F8DC3133B395F8DD1119BB4FF065
:1044E00001082022444404A889F8198071F080F959
:1044F00007EE904A4AF21043F8EEE77A03AA4C21FD
:10450000ADF8283050462423CDED037A35F0D2FBA8
:104510003AF0A0FA9BF80030054A0094042133F0E9
:10452000C9FC85F8DD810137CBE70DB0BDE8F08F20
:1045300080E00808755A0020215D00200523002036
:104540002DE9F04F2F4B1E6885B0044646B1D0F8D8
:104550001415304631F0F4FC10B1304630F052FC06
:104560004FF0A4FE4FF0000801904FF02C0A4FF0DE
:10457000600B94F818355FFA88F5AB4239D904EB33
:104580008507D7F8F00488B30AFB05430BFB054900
:1045900093F92820D9F8E8118A4227D132B302686A
:1045A000D2689047D7F8F0040268126B904799F8E8
:1045B000D52112B1019BC9F8D831BEB1D4F8141578
:1045C000304631F0BDFC88B14FF078FECDE90210E5
:1045D00002460B46D7F8F004294651F07FFFDDE98B
:1045E0000232D7F8F004294651F0F6FF08F101082D
:1045F000BFE72046FFF734FE204605B0BDE8F04F88
:10460000FFF754BF945C00202DE9F0474FF00008FD
:104610002DED028B04468946B0EE408A47460126BE
:104620004FF0600A94F818355FFA88F5AB421AD952
:1046300029FA05F3DB070AD505F59E7354F8230024
:1046400078B10368B0EE480A9B6B984706400AFBB6
:10465000054508F1010895F8D4319F4238BF1F463F
:10466000E0E70646F3E727B97F23A4F82835034B94
:10467000DF72BDEC028B3046BDE8F087755A002032
:1046800090F818358B4207D901F59E7150F821003A
:1046900010B10368DB6B1847002070470B461146CA
:1046A00090F818259A4207D903F59E7350F8230015
:1046B00010B103681B6C18477047000070B50446C2
:1046C0000E46002594F81835E9B28B4205D93246DA
:1046D0002046FFF7E3FF0135F4E770BD2DE9F8430D
:1046E00090F818550246002400F128062C2700F502
:1046F000F4784FF06009E1B28D420FD907FB04F363
:1047000009FB04F0F35658F80000834209D11BB1AD
:104710001046FFF7CFFC10B10134ECE70120BDE8F3
:10472000F8830020FBE7000010B590F818258A42B6
:10473000044617D9602202FB010393F8D431022BFF
:1047400003D004D9032B18BF0023184610BDFFF770
:1047500097FF48B92046FFF7C1FF00280CBF06238A
:104760000123F2E70023F0E70623EEE7014B186888
:10477000704700BFF059002010B5034904462DF0E2
:10478000E9FB204610BD00BF58E2080810B50446FA
:10479000203043F005FA044B04491C6020462DF0FC
:1047A000D9FB204610BD00BF185A0020D4E30808EA
:1047B000F7B5B7EE000A0022022104462DF0BAF93F
:1047C000204652F0E7F843F0CFFA144B1D68064636
:1047D000E86A03685B6A98470B460221024600912B
:1047E000304643F0F3F9B4F94A60002E14DDEF6A65
:1047F0003B6838465B68B4B2984728B197F84D30AB
:1048000013B1C92EA8BFC824A86A03685B682146F3
:1048100003B0BDE8F040184703B0F0BDCC25002040
:1048200010B5044652F084F82046BDE8104052F01E
:10483000AFB800002DE98048284BDFF8A490DFF8DE
:10484000A4A0DFF8A4B01446012293B005460E469A
:104850001A704FF000084FF029FDD9F8003003938B
:10486000A0EB080241F287339A4207461FD9CDE9EF
:10487000005603985346342205A9C06A0EF092F9F7
:10488000214605A804944EF039FFCDE9005603985F
:104890005B46342205A9C06A0EF084F904943AF00C
:1048A000D9F8049B05AA022133F0EAFAB8463AF097
:1048B000D1F839F0CDF93AF0CDF83AF0D5FF0A2128
:1048C00005A80DF075FF039B986A036805215B68D6
:1048D000984705A80DF078FFBDE700BF1C5A0020DF
:1048E000CC25002048E3080871F709080FB400B58B
:1048F00095B016AA002152F8043B039205A83C2269
:104900000193049170F074FF054A019B402104A8B3
:104910004EF09CFE039A034804A9FFF78BFF00BFEB
:1049200050E3080866E308080FB407B504AA034873
:1049300052F8041B0192FFF77DFF00BF78E30808DF
:10494000014B1868704700BF185A00200146D0E993
:10495000070300B11847002BFCD17047B0F90230B3
:1049600002889A4314BFC3F3C000002070470000C0
:1049700038B507230380022200230525C0E905324C
:10498000C0E90D33C0E91033C0E92C330C49036290
:10499000C0F89C5004462DF0DDFA0A4B196811B19D
:1049A00009484FF051FC94F910001C602A4611F0A0
:1049B00015FB637C207403F010036361204638BD4F
:1049C00034E50808205A002074E4080801234361F4
:1049D0000423C36470470000002343610423C364BD
:1049E000704700000123C364704700000223C364C2
:1049F000704700000323C3647047000010B5C3690B
:104A000093B190F9514090F950309C4207DA074B2E
:104A100007480068C06A0EF0C5F8002010BD036AA0
:104A2000012B01D8034BF3E70120F7E790E40808D6
:104A3000CC2500209CE40808F8B504463BF08CFA2D
:104A40003BF076FA3CF034F907463BF085FA3BF050
:104A500079FA3CF02DF906463BF07EFA3BF054FA29
:104A60003CF026F905463BF077FA3BF057FA3CF06C
:104A70001FF90246606C50B101285FD1012E5DD153
:104A8000012A5BD1012D14BF00200820F8BD012FA1
:104A900028D176B9012A61D1012D63D1627CD70773
:104AA00005D494F9511094F95020914210DA022063
:104AB000ECE7022E16D1012A50D1012D52D1627C91
:104AC000D60741D494F9511094F9502091423BDB20
:104AD0006269216C8A421AD0002A33D0012A08BFA9
:104AE0000A20D3E7002D3BD0012E0BD1012A09D19A
:104AF000022DEDD12046FFF731FF002814BF04201E
:104B00000320C3E7E2B1022AE2D10620BEE7E26C4D
:104B1000A16B8A42BAD0012A1DD1617C0D0715D440
:104B2000617C490710D4022A12D1617C0B070DD495
:104B3000627C12F0040F18BF0220A7E70020A5E74F
:104B40000520A3E70920A1E701209FE710469DE784
:104B5000042A9BD1ECE7032AE5D1E1E7002DD1D16E
:104B6000072093E7002DB3D1FAE700004B6A022B30
:104B70004FF0000303D080F84830436470478A68E0
:104B8000032A05D0042A05D0002380F84830704756
:104B90004364F9E70B680A7B5B78012A03F00F0393
:104BA00005D0022AF0D1002BEED00262ECE7002BF8
:104BB000EAD005230362E7E7FFF7D8BF037C033B96
:104BC000022B94BF0120032070470000037C033BAD
:104BD000022B94BF0120042070470000C06910B16F
:104BE00003681B6A1847704770B50446C0690368BC
:104BF00000215B6C9847E069036801219B6C984732
:104C0000E06903680021DB6B9847E5692B6828465B
:104C1000D3E90D63984740F4407081B22846B0470D
:104C20000A23E0691A464FF4E1310DF087FEE0698E
:104C30000368BDE870401B6A184700000339042967
:104C40009ABF024B58560020704700BF2CE5080859
:104C5000F7B5C36904466BB3E2B9012915BF002358
:104C6000012303270427CC208DF804008DF80510BC
:104C70000BB18DF80620002630467D1EF3B2AB4204
:104C800006F1010609DA02AA134413F8041C11F014
:104C900047FAF3E701230427E5E702AB1D443A4650
:104CA00005F8040CE069036801A9DB689847E0692E
:104CB0000DF0A0FE03B0F0BD10B5C4693CB184692D
:104CC000012C06D1C262CAB22146FFF7C1FF2046BD
:104CD00010BD0020FCE70000042910B5044604DCE8
:104CE00002290DDC01290ED010BD0A29FCD1FFF7E5
:104CF00065FFE26801462046FFF7DEFF032306E07A
:104D0000437C9B07F0D5FF23A4F852300423236291
:104D1000EAE7000010B590F8513080F850300446B2
:104D200043F074F920B100F58050002380F88434FA
:104D30006369012B0DD163885B060AD52046FFF716
:104D40003DFFE26801462046FFF7B6FF03232362DA
:104D500010BD0223FBE70000013938B504460629DF
:104D600069D8DFE801F0042031688B8BB60090F938
:104D70005030002B5FDC013380F85030C2680221D4
:104D8000FFF79AFF94F95030002B0ADD43F03EF90B
:104D900020B100F58050012380F88434052323627C
:104DA00049E00423FBE790F95030002B08DD013B7C
:104DB000C26880F850300221FFF77EFF0623EEE73D
:104DC000BDE83840FFF7A6BF90F9503090F9521077
:104DD000012B20DD90F91000484D421EC2EBC202AB
:104DE000AB18AA5C2AB353FA81F394F853205B788A
:104DF000013B9A421DD105281BD0A2680021204604
:104E0000FFF75AFF002384F8533094F85030013BE9
:104E100084F850300FE00CD190F910203748531E21
:104E2000C3EBC303C35C23B1013B994201D1052A03
:104E300002D100290BDA38BDE26800212046FFF7D5
:104E40003BFF94F85030013B84F85030B6E794F9BA
:104E500010302A4A013BC3EBC30313440B445B7875
:104E6000002BE8D0A26800212046FFF725FF94F927
:104E700050300133022BA8BF0223C9E70121826809
:104E8000FFF71AFF94F950301C49012B94F91030A8
:104E900011DD013B94F8520094F85320C3EBC30397
:104EA0000B44034401325B78B2FBF3F103FB1122A4
:104EB00084F85320BFE7013BC3EBC30394F95220AE
:104EC000CB5C013292FBF3F103FB112284F85220F8
:104ED000B1E790F95030002B09DD013B80F85030EC
:104EE0000023C26880F853300221FFF7E5FE94F9F1
:104EF0005030002B9FD194F85130A5E70D220020AF
:104F000010B54369012B044610D143885B060ED5CA
:104F1000437CD90607D4FFF751FEE26801465200F0
:104F20002046FFF7C9FE0323236210BD0BB1022305
:104F3000FAE743885A06FAD5437CDB06F7D5FFF734
:104F400045FEE268014652002046FFF7B5FEEEE757
:104F5000042910B5044604DC02290DDC01290ED019
:104F600010BD0929FCD1FFF731FEE2680146204659
:104F7000FFF7A2FE02230EE0437C9B07F0D52046FC
:104F8000FFF724FEE26801462046FFF795FEFF2367
:104F9000A4F8523004232362E2E7000010B504466F
:104FA0004FF084F9A36AE26AC31A934207D3226AD4
:104FB000A0620023022AE36202D0032A10D010BDAF
:104FC0006269012A0AD1638813F0400F0CBF0021E7
:104FD0000A212046BDE81040FFF77EBE1946F8E7DB
:104FE000616949B9638813F0400F18BF0921204651
:104FF000BDE81040FFF7ACBF1946F8E773B50B6882
:105000005B78836143885B045EBF0B685B88438089
:10501000B0F90230002B04461ADD0123036239F097
:1050200019FD05462046B4F90260FFF797FC68B900
:105030002388B3430CBF022300230093094A33465D
:105040000621284632F036FF02B070BD0523F4E792
:1050500039F000FD044A042102B0BDE8704032F08E
:1050600029BF00BFB0E40808E1E40808FFF7C6BFA5
:1050700070B50446D0F8B8000E46E8B1D4F8A830B0
:1050800023B1D4F8A420CB1A934221D3B4F8AC5066
:105090009DB12046FFF7A8FDD4E9260194F8A02091
:1050A000FFF7D6FDB4F8AC30C4F8A8600020013B8F
:1050B00084F8A100A4F8AC3070BD042304F194007E
:1050C000C4F8B830FFF742FCC4F8B8502846F3E7FC
:1050D0000120F1E738B50024054620466B7BA3424A
:1050E00005DD2B68195D11F01BF80134F6E738BDBA
:1050F0002DE9F041C3690446002B43D04FF0D6F8A8
:1051000001462046FFF7B4FF00283BD0E069036862
:105110005B699847402828BF40200025064604F1D7
:105120009407A846AE422DD04FF0C0F80146204665
:10513000FFF79EFF30B3E06903689B69984794F8D6
:10514000A130C0B20BB9CC281AD1D4F89420D054D5
:1051500094F8A13094F8A2200133DBB29A4284F88B
:10516000A1300DD13846FFF7B5FF00280CBF022350
:105170000323C4F8B8303846FFF7E8FBC4F8B8801A
:105180000135CFE7BDE8F081074A002352F833002C
:10519000884203D102EBC303187970470133042B13
:1051A000F4D10020704700BF3022002038B50373CF
:1051B00000234373049B03611546BDF814308560DA
:1051C00001F154020446C0E90021038300F11C03ED
:1051D000DDE9060183E80300012363624FF066F80E
:1051E000294660612046FFF7CFFFA073204638BDF7
:1051F0002DE9F0438FB016AC064634F8049B0F46F9
:1052000090461D46FFF7EAFC94E8030002AB83E8F2
:1052100003003A46CDE900594346314604A804ACA0
:10522000FFF7C4FF0FCC06F194050FC50FCC0FC5D7
:1052300094E80300424685E80300394630460FB043
:10524000BDE8F043FFF704BD10B586B0094B0593E8
:10525000049006AA12E9030001AB83E803000022D0
:105260004FF6FF73009311464FF47A63FFF7C0FFC8
:1052700006B010BD6D50010813B51A4B04461868EE
:1052800020B100221A212EF02DFCE061E36953B118
:1052900001230DF1070104F110008DF807302DF006
:1052A00023FC2DF05DF894F9103013B9E36102B0DE
:1052B00010BDE269002AFAD0022B01D0052B03D1E0
:1052C0004FF6FF73A4F850302046FFF78DFC4EF0E8
:1052D000EDFF6368A0622046E36202B0BDE81040C3
:1052E000FFF7B2BF445B002030B587B004AB83E862
:1052F0000600054693E8030001AC022384E805009C
:105300000421009301224FF4C8732846FFF770FF71
:1053100007B030BD30B587B004AB83E80600054662
:1053200093E8030001AC84E80500022200924FF4E8
:10533000C87304212846FFF75BFF07B030BD0000AB
:1053400010B586B006AC04E90C0061B101244464D8
:1053500001AC84E80C000224CAB200944FF4C87374
:105360002146FFF745FF06B010BD000070B586B0BE
:1053700004AB83E8060002254564044693E8030075
:1053800001AE86E805004FF4C873009500220321A2
:105390002046FFF72DFF06B070BD000010B50123B9
:1053A00080F848304B1E88B00446C262072B31D8C3
:1053B000DFE803F0040E181818181825164B009093
:1053C0001A460146019308B0BDE81040FFF78CBFB4
:1053D000114B02901A460146039308B0BDE81040F5
:1053E000FFF798BFFFF72AFC0B4B049401462246B7
:1053F0002046059308B0BDE81040FFF7A1BF064B5B
:105400000793069008AB13E9060008B0BDE810400A
:10541000FFF7ACBF08B010BDB94B01084B1E10B56B
:105420000446092B20D8DFE803F00C233636363645
:1054300036053636642208212046BDE81040FFF7C5
:10544000ADBF90F9503083B942F0E0FD20B100F5D6
:105450008050012380F88434642201212046FFF724
:105460009DFF012384F8503010BD64220321E3E73F
:1054700090F95030002BF7DD42F0C8FD20B100F567
:105480008050002380F88434642202212046FFF7F4
:1054900085FF0023E6E76422CEE7000013B504464B
:1054A0000191FFF75BFA019928B1204602B0BDE8EF
:1054B0001040FFF7B3BF2388B4F90220934305D10E
:1054C000204602B0BDE81040FFF746BC02B010BD58
:1054D00070B504464EF0EAFE94F8482022B9A36A5B
:1054E000E16AC31A8B4202D20023236370BDC4E970
:1054F0000A022046FFF7A0FA236B62698342014645
:10550000236AE06C0ED1656BAB420BD1A56B854273
:1055100008D194F93C6094F95050AE4202D1256C08
:105520009542E3D0C4E90C13A063013B94F850000A
:1055300084F83C002264052BD8D8DFE803F0030888
:105540000D1213182046BDE87040FFF7D9BC204665
:10555000BDE87040FFF7C0BB2046BDE87040FFF7D4
:10556000F7BC01212046BDE87040FFF797BF02213C
:10557000F8E7000010B50D4B1B68DB6A93F89C3010
:10558000044623B12046BDE81040FFF707BD42F0B6
:105590003DFD28B100F5805393F86434032BF1D816
:1055A0002046BDE81040FFF793BF00BFCC25002088
:1055B00038B5C36904467BB190F9103063B1FFF789
:1055C00097FD4EF073FE636AC31A642B054603D938
:1055D0002046FFF7CFFF656238BD0000014B186819
:1055E000704700BF205A002008B50449102270F00F
:1055F000A5F8B0FA80F0400908BD00BF245A002089
:105600001022002170F0F4B810B50446FFF7F8FF3F
:10561000204610BD0378416023F00D03022A037079
:1056200008D0032A0AD0012A03D1DBB243F00103D8
:1056300003707047037843F00803F9E7037823F019
:10564000050343F00503F3E773B504460E4615461C
:105650000193FFF7D5FF2046C4E90265069A019938
:10566000FFF7D8FF02B070BD0078420704D40307EB
:1056700004D400F0010070470320704702207047F7
:10568000F0B585B005461646FFF7EEFF88420F4697
:1056900005D16B6833600124204605B0F0BD0328B6
:1056A00001D10024F8E70329FBD001280BD0022800
:1056B00016D018BB6D68012F22D0022F2ED0002FDC
:1056C000EFD13560E7E7FBF737FF90F87C32DB0777
:1056D000E7D56D68FBF730FFD0F870321D44EAE77C
:1056E0006846FFF78DFFFBF727FF6946FBF72AFDAA
:1056F00004460028D0D06D68019BEFE70025DAE76B
:10570000FBF71AFF90F87C4214F00104C9D0FBF7B4
:1057100013FFD0F87032ED1A3560BDE76846FFF729
:105720006FFFFBF709FF6946FBF70CFD04460028F5
:10573000B2D0019BEFE7000073B501AA05460E4603
:10574000FFF79EFF044620B1019932462846FFF735
:1057500061FF204602B070BD13B5144601AAFFF7E1
:105760008FFF48B1DDED017A9FED047AF8EEE77A1C
:1057700067EE877AC4ED007A02B010BD0AD7233CE9
:1057800007EE900A9FED090AF8EEE77A08B527EED2
:10579000800A6DF025FCDFED067AB4EEE70AF1EE43
:1057A00010FAD8BFB0EE670A08BD00BF50E0EF3076
:1057B0000AD7233C10B50446806810F059FD20B18B
:1057C000E068BDE8104010F067BD10BD0D4B83428E
:1057D0004FF000038B4106DA00F1255000F531103F
:1057E00000F5E0507047084B98424FF0FF3371EBE3
:1057F0000303BEBF00F1564000F5130000F524403E
:10580000704700BF00D2496B002EB69490EA010F9A
:1058100001D4401A7047C317401A63EBE1710D4B76
:1058200083424FF000038B4106DA00F1255000F56A
:10583000311000F5E0507047074B98424FF0FF33AE
:1058400071EB0303BEBF00F1564000F5130000F5F5
:105850002440704700D2496B002EB69470B52DEDF0
:10586000028B84B0044668460D46FFF7C9FEFBF77D
:1058700063FE6946FBF766FC064608B3A368029A16
:10588000DFED128A03999B1A07EE903AF8EEE77A59
:1058900067EEA87AC5ED007AE068FFF7B7FF08EE7B
:1058A000100AA068024402EBD272B8EEC88A501007
:1058B000FFF766FF28EE288A28EE000A85ED010A28
:1058C000304604B0BDEC028B70BD00BFF67C8E3F4D
:1058D00037B500230C4601AA022105460193FFF7C4
:1058E000CFFE10B9002003B030BD21462846FFF797
:1058F000B5FF0028F6D0DDED017AF8EEE77AC4EDC9
:10590000027AF0E738B52DED028B0C460246C168ED
:10591000E068FFF77BFF9568A46808EE100A60193D
:1059200000EBD0704010641BFFF72AFF07EE904A8F
:10593000F8EEE77AF8EEC80A87EE807ABDEEC70A7D
:1059400010EE103A5B4200EE103AB8EEC00A6DF06D
:1059500069FDDFED087A30EE270ABDEC028BB5EE6B
:10596000C00AF1EE10FA44BFDFED037A30EE270AE9
:1059700038BD00BFDB0FC93FDB0FC94030B52DED8F
:10598000028B0B4685B08C68D0E90251D868FFF7CE
:105990003DFF08EE100A601900EBD0704010FFF7D1
:1059A000EFFE641B07EE904AF0EE400AB8EEC88A9C
:1059B0009FED060AF8EEE77A28EE008A27EE800AC5
:1059C00068EE200A05B0BDEC028B30BD8262363C29
:1059D00082B002B0FFF7D2BFF0B52DED028B0D46BD
:1059E00089B08C680646D0E90271E868FFF70EFFBF
:1059F00008EE100AE01900EBD0704010FFF7C0FE6F
:105A000073686A689FED0E1A9B1A07EE903AE41BC2
:105A1000B8EEE77AF0EE400A07EE904A9FED090AE9
:105A2000B8EEC88AF8EEE77A28EE008A27EE011A67
:105A300027EE800A68EE200A09B0BDEC028BF0BDAB
:105A40000AD7233C8262363C10B52DED028B846868
:105A50008A680B46111B08EE901AC168D868FFF7D8
:105A6000D5FE224402EBD27208EE100A5010FFF766
:105A700087FEB8EEC88AF8EEE88A28EE000A20EE23
:105A8000000AA8EEA80A6DF017FEBDEC028BDFED50
:105A9000027A20EE270A10BD8262363C094B9842FA
:105AA00006DDC0F1D64000F5930000F5A440704734
:105AB000054B9842BEBFC0F1144000F5360000F51A
:105AC0003850704700E9A43500175BCAF8B52DEDD2
:105AD000028BDFED148A076820EE280A0646FDEEE9
:105AE000C07A0D4617EE904A04EBD47007EB6000C5
:105AF000B0EE608AFFF744FE28EE288A3819C8EE17
:105B0000007AFFF7CBFF306017EE900AF7F71EFA26
:105B10002B68C01841EBE371FFF758FEBDEC028B18
:105B20002860F8BD02AAB34200F10C010830FFF76B
:105B3000CDBF00000148FFF763BD00BF245A00201D
:105B40000121884238BF08466BF072BBFFF7F8BFEF
:105B500008B16BF071BB7047FFF7FABF00214FF03F
:105B6000FF3310B500220363044601600171C0F8E1
:105B70000510417280F8251000F13C0300F50B7010
:105B8000D9709A60DA601A615A619A61DA611A62B0
:105B90005A629A62DA631A645A649A64DA641A6519
:105BA0005A659A65DA65DA661A675A677C339842ED
:105BB000E6D1214604F5167007F0AAFA044B1A68DC
:105BC00022B904491C6020462CF0C4F9204610BDBF
:105BD000345A00206CE7080873B5D0F83C320191C4
:105BE0009942044613D0D0F84032994218D0D0F8E8
:105BF00044328B4216D102200AE0D4F8343253B337
:105C0000D4F838324BB34FF0030002B070BD00201F
:105C100094F822308342F8D8431C84F82230F4E709
:105C20000120F5E7D0F83062002EE6D194F8412348
:105C30003546B6009AB1A319C3F83012A319019AD8
:105C4000C3F83C2294F82230AB429CBF6B1C84F812
:105C500022302846D9E70126E8E70226E6E704F5E0
:105C60000C7001A930442DF011F8E7E738B504466F
:105C70000D462CF081FF291D201D2CF07DFF05F124
:105C8000080104F108002DF051F805F1140104F1A8
:105C900014002DF04BF805F1200104F120002DF047
:105CA00045F805F12C0104F12C002CF0F9FE05F16A
:105CB000300104F130002DF001F805F13C0104F150
:105CC0003C002DF033F8AB6BA3636B6B636338BDA3
:105CD0002DE9F043A1B00023002500F13C07064662
:105CE0008DF8075003930493059306930793089345
:105CF00009930A930B931093119312931393149394
:105D000015931693179318931C931D931E9300F5E8
:105D10000F78B94658F8043BF3B1F26E934223D0A2
:105D2000D6F8E820934221D0D6F86421934213D1CB
:105D30000221EBB299420FD0C1EB411109EB810472
:105D4000214601A8FFF792FF39462046FFF78EFF54
:105D500001A93846FFF78AFF0135032D07F17C07BB
:105D6000D8D121B0BDE8F0830021E2E70121E0E7CE
:105D70002DE9F04706460F461546804604464FF08B
:105D8000000A39463046FFF727FF626FBA425FFAD2
:105D90008AF90ED1C3B2022B0BD87C2202FB0A6611
:105DA000012086F83E0086F83F3085F80090BDE877
:105DB000F0870AF1010ABAF1030F04F17C04E0D183
:105DC000002439463046FFF707FFD8F86C205FFA09
:105DD00084F912B9C3B2022B22D90134032C08F181
:105DE0007C08EED100244FF07C0906F13E0A3946CA
:105DF0003046FFF7F1FE034609FB04F05FFA84F832
:105E00001AF8002012B9DBB2022B12D90134032C8C
:105E1000EDD196F82300042814D919484EF014FA4D
:105E20007C2000FB0464012084F83E0084F83F30AD
:105E3000BBE70644012086F83E0086F83F3085F82F
:105E40000080B4E706F54371002251F8043BBB42E1
:105E5000D4B208D1A04202D8631C86F823300334A0
:105E60002C700020A3E73BB9421C06EB800086F8AB
:105E70002320C0F80C73F2E70132052AE5D1F0E7E0
:105E8000A4E50808C9B200EB8101D1F83C3253B156
:105E9000026F93420AD0D0F8EC20934208D0D0F899
:105EA0006821934206D04FF00300704700207047EE
:105EB000012070470220704759B190F82030032B21
:105EC00007D05A1C80F8202000EB8300416101209C
:105ED00070470020704700002DE9F8430F469146B7
:105EE000044600F5BA7894F83E5035B97C34444500
:105EF000F9D100252846BDE8F88300234A463946F3
:105F000001200CF0E3FA00210646E06E0CF0EEFAF8
:105F10008642EBD1EEE700002DE9F043DFF87C800C
:105F200085B0044600F50F7600257C27B14656F86B
:105F30000C3CD9F800209342E9B206F1040619D1CD
:105F4000C3B12046FFF79EFFC0B207FB004090F8A8
:105F50003E307BB903A9A9F10C0003932CF096FE07
:105F600038F078FD56F8043C009342462B46012158
:105F700031F0A0FF0135032DD8D104F16C0504F5F3
:105F8000F074296821B9AB6813B128462BF0D4FA14
:105F90007C35A542F5D105B0BDE8F083C0E5080821
:105FA00038B504461546FFF76DFFC0B2022808D881
:105FB0007C2303FB004029465030BDE838402CF0DC
:105FC000A5BE38BD38B504461546FFF75BFFC0B225
:105FD000022808D87C2303FB004029465C30BDE83A
:105FE00038402CF093BE38BD37B50D4604468DEDD4
:105FF000010AFFF747FF022D07D8C0B27C2303FB3D
:10600000004001A968302CF033FD03B030BD000022
:1060100038B50546FFF736FFC4B2022C13D8C4EBDF
:106020004414A4003C3504F10800284400212BF05E
:1060300083FA04F1340104F1300029442844BDE816
:1060400038402CF023BE38BD70B505460E461446C8
:10605000FFF718FFC3B2022B0DD87C2000FB0353BF
:1060600094E80700443383E8070031462846BDE83A
:106070007040FFF7CDBF70BD37B504461546FFF73A
:1060800001FFC0B2022809D87C2303FB00400DF1B8
:10609000070140308DF807502CF06EFD03B030BD85
:1060A00010B500210446FFF7B3FF20460121FFF79A
:1060B000AFFF20460221BDE81040FFF7A9BF000056
:1060C0001FB590F92C30044623B390F921300BB35F
:1060D0006846FFF799FAFBF72FFA6946FBF70EF8C7
:1060E000C0B1DDED037A9FED0C0AF8EEE70ADDEDB5
:1060F000027AF8EEE77A0123C0EE800A84F83D3395
:1061000087EE800A07F046FADFED047A20EE270AD0
:1061100084ED0A0A04B010BD8096184B35FA8E3C07
:10612000024690F9210058B192F8400340B1114461
:1061300091F92C0220B192F92400033818BF0120F4
:106140007047000038B590F8223005465BB1002456
:106150002346E1B22846FFF7E3FF08B10133DBB283
:106160000134032CF5D1184638BD000090ED0A0A21
:106170007047000038B50C46D1ED066A1146054659
:10618000FFF780FEC3B27C2000FB0353D4ED087AF6
:10619000D3ED260A94ED076AD3ED255A93ED245AE0
:1061A00026EE600A67EEA00AA5EEA70AF0EE607A76
:1061B000E5EE867AB7EE007AA6EEE67A67EEE60AB4
:1061C000B1EE400AE5EE070A6DF02CF99FED071AD3
:1061D000DFED070A40F61C000FF0C2FED5ED0A7A8B
:1061E000BDE8384030EE270A0FF0A6BEDB0F49406D
:1061F000DB0F49C02DE9F04190F822308B42044674
:106200000D4602D20020BDE8F081FFF73BFEC0B290
:1062100004F13C06C0EB401006EB8000083012F0A1
:10622000A1FADFED157AB0EEC00AB4EEE70AF1EE9E
:1062300010FAE7D429462046FFF724FEC5B27C2099
:1062400000FB05473B6F002BDCD0032DDAD000FBB1
:1062500005603030D7F86C802BF052FFD7E91B3245
:10626000934201D1984505D07C2000FB0544C4F839
:106270006C80C7E70120C6E7000000342DE9F74F26
:1062800004460E46174600F50F7A4FF0000B5AF8F9
:10629000049B5FFA8BF8B9F1000F26D041462046E7
:1062A000FFF73EFF08B341462046FFF7EBFD7C2396
:1062B000C0B203FB004090F83E505DB908F1010305
:1062C0001B4ADBB2394630464DF0C0F9284603B0D0
:1062D000BDE8F08F5AF8102C914506D0154A394682
:1062E00030464DF0B3F90025F0E70BF1010BBBF19F
:1062F000030FCCD14FF0000894F822305FFA88F1F8
:106300008B420DD920460191FFF774FF054620B955
:1063100001992046FFF704FF20B908F10108EBE7D7
:106320000125D3E7044A394630464DF08FF9CDE7D1
:10633000E8E50808FDE5080822E608082DE9F0412F
:106340002DED048B90F842139FED348ADFED348AF3
:106350009FED349A82B00646FFF794FD06F13C07A4
:10636000C5B27C2000FB057554354FF0000896F847
:1063700022205FFA88F39A424ED919463046FFF739
:10638000CFFE10B908F10108F1E719463046FFF7D2
:1063900079FDC4B27C2000FB0474D4ED157AF0EED4
:1063A000E77AF4EEC87AF1EE10FA04F154040ED54F
:1063B000D4ED017AF0EEE77AF4EEC87AF1EE10FA55
:1063C00005D5002002B0BDEC048BBDE8F081294664
:1063D000204612F0DFF9B4EEE80AF1EE10FAF0DC34
:1063E0002946204611F0FEFCB4EEC90AF1EE10FA7F
:1063F000E7DC2146284611F041FC68468DED000A95
:10640000CDED010A11F0DAFCDFED077AB4EEE70A10
:10641000F1EE10FAB6DDD4E70120D3E70000003436
:10642000DB0FC93F920A863F00004843022910B59E
:10643000044608D8FFF726FD7C23C0B203FB0044C6
:1064400094F83D0010BD0020FCE7000013B590F863
:10645000421301910446FFF7E9FF30B1019920464C
:1064600002B0BDE81040FFF75BBE02B010BD0000F7
:10647000F7B590F921500446002D73D090F84053A1
:10648000002D6FD090F84213FFF7D0FF94F83D3302
:10649000064613B92046FFF713FE002594F8202086
:1064A000EBB29A4207D904EB8303013558690368BC
:1064B0009B689847F2E74DF0F9FE0027224604F565
:1064C000BA7140F2F315D2F89C30C31AAB428CBFBC
:1064D0000023012382F83D307C32914247EA0307D2
:1064E000F1D194F92430032B07D194F83C33002BDD
:1064F0003BD0D4F83803002849D167B1236B01336E
:1065000009D02FF053FD216B2FF01AFD18B12FF099
:106510004DFD2EF08BFD94F92C32002B3AD194F9DD
:106520002D32CBBB94F92E3213B1022384F84233BF
:1065300094F842132046FFF779FF8642054611D0B2
:106540002FF034FD4FF6FF712FF0FAFC50B1002D03
:1065500014BF0022042201922FF028FD019A03218A
:106560002FF080FC284603B0F0BD012384F83C33B3
:106570000420FFF7E5FA054610B1214606F05EFE5D
:1065800094F92430C4F83853032BB2D0B5E706F0A1
:1065900063FEB2E70023C9E70123C7E738B590F9E6
:1065A00021300446D3B190F84053BDB1FFF76AFCE7
:1065B000C0B2022812D87C2303FB0044D4ED1A7A1F
:1065C0009FED087AF4EEC77AF1EE10FA06D4B7EE32
:1065D000087AF4EEC77AF1EE10FA00DD00252846BD
:1065E00038BD00BFABAA2A3F70B5D0F8085315F4E8
:1065F000003504460E460DD190F840335BB90A7859
:10660000072A07D8012303FA02F290F83F33134315
:1066100080F83F3370BD94F82020EBB29A42F9D94C
:1066200004EB8303314658690368DB6898470135FA
:10663000F1E7000038B505466C242B591BB1002149
:1066400028192AF079FF7C34B4F5F07FF5D138BDF4
:10665000014B1868704700BF345A00202DE9F04FF5
:10666000AA4BD3F800800446D8F8040003688DB024
:106670009B689847002507464FF0010909FA05F382
:106680003B4240F082820135202DF7D1D8F804003A
:106690000368DB689847002507464FF0010909FAAF
:1066A00005F33B4240F0B3820135202DF7D1D8F8F5
:1066B000040003689B689847002507464FF00109CE
:1066C00009FA05F33B4240F0E1820135202DF7D174
:1066D000D8F80400DFF840B203689B6898470025AB
:1066E0000490049A0123AB40134240F00B83013520
:1066F000202DF6D1D8F80400DFF81CB20368DB685F
:10670000984700250490049A0123AB40134240F0BF
:10671000C9830135202DF6D1D8F804000368DB6861
:106720009847002507464FF0010909FA05F33B4257
:1067300040F083840135202DF7D1D8F80400036898
:10674000DB689847002507464FF0010909FA05F371
:106750003B4240F0B1840135202DF7D1D8F8040038
:1067600003689B689847002507464FF0010909FA1E
:1067700005F33B4240F0DF840135202DF7D1D8F8F6
:10678000040003689B689847002507464FF00109FD
:1067900009FA05F33B4240F00E850135202DF7D173
:1067A000D8F8040003689B689847002507464FF017
:1067B000010909FA05F33B4240F03D850135202DE2
:1067C000F7D1D8F804000368DB689847002507462E
:1067D0004FF0010909FA05F33B4240F068850135A5
:1067E000202DF7D14A4B089308AF0425D8F80400B0
:1067F00003689B689847002683460123B34013EA49
:106800000B0F40F08F850136202EF6D1D8F804000A
:106810000368DB689847002683460123B34013EAE8
:106820000B0F40F0C4850136202EF6D1013D15F046
:10683000FF0507F10107D9D1D8F8040003689B6868
:1068400098474FF00109074609FA05F33B4240F02B
:10685000F2850135202DF7D1D8F804000368DB68F4
:106860009847002507464FF0010909FA05F33B4216
:1068700040F01D860135202DF7D1D8F804000368BB
:106880009B689847002507464FF0010909FA05F370
:106890003B4240F048860135202DF7D1D8F804005E
:1068A0000368DB689847002507464FF0010909FA9D
:1068B00005F33B4240F073860135202DF7D1154B8F
:1068C0000793D8F8040003689B689847002583461F
:1068D0000123AB4013EA0B0F42D000275FFA85F982
:1068E000D4F8083313F4803A32D107AB4946DB5D64
:1068F00004931A462046FFF7EFFA049B0646002849
:1069000000F08986CDE908AA08E000BFCC25002068
:106910000C0D0E0F20212223801A0600099B0B93D9
:10692000002201210BA8CDE9092204F003FE014653
:106930002046FFF7C1FA0BA8FDF7E0F90AA8FDF71A
:10694000DDF909A8FDF7D0F916B108A8FDF7CCF9D3
:1069500094F82330052B00F048810137042FBFD174
:106960000135202DB4D1D8F804000368DB689847BE
:10697000002583460123AB4013EA0B0F38D00027D4
:106980005FFA85F9D4F8083313F4803A28D107ABBD
:106990004946DB5D04931A462046FFF79DFA049BA7
:1069A0000646002800F04686CDE908AA0022099B89
:1069B0000B9311460BA8CDE9092204F0BBFD01465B
:1069C0002046FFF779FA0BA8FDF798F90AA8FDF71A
:1069D00095F909A8FDF788F916B108A8FDF784F91B
:1069E00094F82330052B00F000810137042FC9D122
:1069F0000135202DBED1D8F8040003689B68984764
:106A0000002682460123B34013EA0A0F31D0102535
:106A10005FFA86F9D4F8083313F0080B20D12A4620
:106A200049462046FFF758FA0746002800F011862D
:106A3000CDE909BB0A9B002201210BA8CDE90A235D
:106A400001F00AFC01462046FFF736FA0BA8FDF7D5
:106A50004BF90AA8FDF748F917B109A8FDF744F961
:106A600094F82330052B00F0C0800135EDB2142DD1
:106A7000D0D10136202EC5D1D8F8040003689B6818
:106A80009847002682460123B34013EA0A0F34D008
:106A900014255FFA86F9D4F8083313F4001B24D1C7
:106AA0002A4649462046FFF717FA0746002800F015
:106AB000E385CDE908BB099B0B93002201210BA8BC
:106AC000CDE9092201F0DAFF01462046FFF7F4F98B
:106AD0000BA8FDF713F90AA8FDF710F909A8FDF7AF
:106AE00003F917B108A8FDF7FFF894F82330052B38
:106AF0007BD00135EDB2182DCDD10136202EC2D17B
:106B0000D8F804000368DB68984700268246012312
:106B1000B34013EA0A0F34D014255FFA86F9D4F88B
:106B2000083313F4001B24D12A4649462046FFF7B8
:106B3000D3F90746002800F0AF85CDE908BB002255
:106B4000099B0B9311460BA8CDE9092201F096FF92
:106B500001462046FFF7B0F90BA8FDF7CFF80AA8C9
:106B6000FDF7CCF809A8FDF7BFF817B108A8FDF7A5
:106B7000BBF894F82330052B37D00135EDB2182D32
:106B8000CDD10136202EC2D12FE0D4F8083313F036
:106B9000010A25D15FFA85FB1E2259462046FFF7E0
:106BA0009BF9064620B3CDE908AA099A0B92002367
:106BB000082201210BA8CDE9093303F089FA014627
:106BC0002046FFF779F90BA8FDF798F80AA8FDF71A
:106BD00095F809A8FDF788F816B108A8FDF784F81C
:106BE00094F82330052B7FF44EAD0DB0BDE8F08F47
:106BF000D8F8041004220B68CDE90102A84A0092DB
:106C0000D3F800A05A461E2309A8D047CDE7D4F8F0
:106C1000083313F0010A24D15FFA85FB1E2259467E
:106C20002046FFF759F9064608B3CDE908AA099BA3
:106C30000B93062200210BA8CDE9091103F048FAB5
:106C400001462046FFF738F90BA8FDF757F80AA8C8
:106C5000FDF754F809A8FDF747F816B108A8FDF7A5
:106C600043F894F82330052B7FF41EADBDE7D8F828
:106C7000041004220B68CDE90102894A0092D3F87E
:106C800000A05A461E2309A8D047D0E7D4F80833FD
:106C900013F4805A21D15FFA85FB0D225946204614
:106CA000FFF71AF90646F0B1CDE909AA0A9B0022BE
:106CB000CDE90A23012108220BA804F077FA014646
:106CC0002046FFF7F9F80BA8FDF70EF80AA8FDF724
:106CD0000BF816B109A8FDF707F894F82330052B37
:106CE0007FF4F3AC81E7D8F8041004220B68CDE9F7
:106CF00001026B4A0092D3F800A05A460D230AA85D
:106D0000D047D3E7D4F8083313F480773FD15FFA44
:106D100085F90C2249462046FFF7DEF80646002892
:106D200000F08480CDE90677079B0A934FF0000AB4
:106D3000692249462046CDF81CA0FFF7CDF807464A
:106D4000002800F08180CDE908AA099B0B9300225E
:106D50001A2309920BA901220AA801F005F801469D
:106D60002046FFF7A9F80BA8FCF7BEFF09A8FCF71F
:106D7000BBFF17B108A8FCF7B7FF0AA8FCF7B4FFE0
:106D800007A8FCF7B1FF16B106A8FCF7ADFF94F811
:106D90002330052B3FF429AFD4F8083313F4807760
:106DA0007FF4A5AC5FFA85F90C2249462046FFF72F
:106DB00093F80646002856D0CDE90677079B0A933C
:106DC0004FF0000A682249462046CDF81CA0FFF784
:106DD00083F80746002854D0CDE908AA099B0B93F5
:106DE00000221A2309920BA901220AA800F0BCFF75
:106DF00001462046FFF760F80BA8FCF775FF09A8CD
:106E0000FCF772FF17B108A8FCF76EFF0AA8FCF7A1
:106E10006BFF07A8FCF768FF16B106A8FCF764FF34
:106E200094F82330052B7FF462ACDEE6D8F804102A
:106E300004220B68CDF800B0CDE901024A461F6874
:106E400007A80C23B8476FE7D8F8041004220B6892
:106E5000CDF800B0CDE901024A46D3F800A009A858
:106E60006923D04771E7D8F8041004220B68CDF8E5
:106E700000B0CDE901024A461F6807A80C23B847B5
:106E80009CE7D8F8041004220B68CDF800B0CDE9D7
:106E900001024A46D3F800A009A86823D0479DE71D
:106EA000801A0600D4F8083313F480773DD15FFAD6
:106EB00085F90C2249462046FFF70EF806460028C1
:106EC00000F08180CDE90677079B0A934FF0000A16
:106ED000692249462046CDF81CA0FEF7FDFF074673
:106EE00000287ED0CDE908AA099B0B9300221A2323
:106EF0000BA90AA8099200F037FF01462046FEF7C9
:106F0000DBFF0BA8FCF7F0FE09A8FCF7EDFE17B1BC
:106F100008A8FCF7E9FE0AA8FCF7E6FE07A8FCF7BC
:106F2000E3FE16B106A8FCF7DFFE94F82330052B2C
:106F30003FF45BAED4F8083313F480777FF4E9AB09
:106F40005FFA85F90C2249462046FEF7C5FF064642
:106F5000002855D0CDE90677079B0A934FF0000A29
:106F6000682249462046CDF81CA0FEF7B5FF07462B
:106F7000002853D0CDE908AA099B0B9300221A23BD
:106F80000BA90AA8099200F0EFFE01462046FEF781
:106F900093FF0BA8FCF7A8FE09A8FCF7A5FE17B104
:106FA00008A8FCF7A1FE0AA8FCF79EFE07A8FCF7BC
:106FB0009BFE16B106A8FCF797FE94F82330052B2C
:106FC0007FF4A7AB11E6D8F8041004220B68CDF8C3
:106FD00000B0CDE901024A461F6807A80C23B84754
:106FE00072E7D8F8041004220B68CDF800B0CDE9A0
:106FF00001024A46D3F800A009A86923D04773E7E5
:10700000D8F8041004220B68CDF800B0CDE90102D5
:107010004A461F6807A80C23B8479DE7D8F8041014
:1070200004220B68CDF800B0CDE901024A46D3F83E
:1070300000A009A86823D0479EE7D4F8083313F0CE
:10704000200A24D15FFA85FB1C2259462046FEF710
:1070500043FF064608B3CDE908AA0022099B0B931B
:1070600011460BA8CDE9092203F030FC0146204669
:10707000FEF722FF0BA8FCF741FE0AA8FCF73EFE34
:1070800009A8FCF731FE16B108A8FCF72DFE94F80C
:107090002330052B7FF44EABA7E5D8F8041004226B
:1070A0000B68CDE90102B84A0092D3F800A05A4615
:1070B0001C2309A8D047D0E7D4F8083313F0200ADE
:1070C00024D15FFA85FB1E2259462046FEF704FFB5
:1070D000064608B3CDE908AA0022099B0B93114686
:1070E0000BA8CDE9092203F0F1FB01462046FEF78B
:1070F000E3FE0BA8FCF702FE0AA8FCF7FFFD09A8B7
:10710000FCF7F2FD16B108A8FCF7EEFD94F8233069
:10711000052B7FF420AB68E5D8F8041004220B6837
:10712000CDE90102984A0092D3F800A05A461E23E6
:1071300009A8D047D0E7D4F8083313F0200A25D1A6
:107140005FFA85FB1C2259462046FEF7C5FE06461F
:1071500010B3CDE908AA099A0B920023022201215B
:107160000BA8CDE9093303F0B1FB01462046FEF739
:10717000A3FE0BA8FCF7C2FD0AA8FCF7BFFD09A8F7
:10718000FCF7B2FD16B108A8FCF7AEFD94F8233069
:10719000052B7FF4F1AA28E5D8F8041004220B6827
:1071A000CDE90102784A0092D3F800A05A461C2388
:1071B00009A8D047CFE7D4F8083313F0200A25D127
:1071C0005FFA85FB1E2259462046FEF785FE0646DD
:1071D00010B3CDE908AA099A0B92002302220121DB
:1071E0000BA8CDE9093303F071FB01462046FEF7F9
:1071F00063FE0BA8FCF782FD0AA8FCF77FFD09A837
:10720000FCF772FD16B108A8FCF76EFD94F8233068
:10721000052B7FF4C2AAE8E4D8F8041004220B6816
:10722000CDE90102584A0092D3F800A05A461E2325
:1072300009A8D047CFE7D4F8083313F0400A21D18A
:107240005FFA85FB0C2259462046FEF745FE0646AE
:10725000F0B1CDE909AA0A9B0022CDE90A23012158
:1072600006220BA800F046FD01462046FEF724FE4C
:107270000BA8FCF739FD0AA8FCF736FD16B109A8E2
:10728000FCF732FD94F82330052B7FF497AAACE489
:10729000D8F8041004220B68CDE901023A4A0092A2
:1072A000D3F800A05A460C230AA8D047D3E7D4F855
:1072B000083313F0400A20D15FFA85FB0C225946AF
:1072C0002046FEF709FE0646E8B1CDE909AA0022EC
:1072D0000A9B11460BA8CDE90A2300F00BFD0146DD
:1072E0002046FEF7E9FD0BA8FCF7FEFC0AA8FCF718
:1072F000FBFC16B109A8FCF7F7FC94F82330052B2A
:107300007FF46DAA71E4D8F8041004220B68CDE96B
:1073100001021D4A0092D3F800A05A460C230AA885
:10732000D047D4E7D4F8083313F0800A26D13B784D
:10733000F1B21A462046CDE90413FEF7CDFDDDE992
:107340000413814610B3CDE909AA0A9B0022CDE9B6
:107350000A2301210C220BA803F086F901462046DE
:10736000FEF7AAFD0BA8FCF7BFFC0AA8FCF7BCFCC3
:10737000B9F1000F02D009A8FCF7B6FC94F823304D
:10738000052B7FF440AA30E4801A0600D8F80400E8
:10739000B84AD0F800E000924FF0040CCDE9019C0F
:1073A0000A46DEF800A001460AA8D047CDE7D4F887
:1073B000083313F0800A26D13B78F1B21A462046F2
:1073C000CDE90413FEF788FDDDE90413814608B317
:1073D000CDE909AA0A9B0022CDE90A2300210C224B
:1073E0000BA803F041F901462046FEF765FD0BA806
:1073F000FCF77AFC0AA8FCF777FCB9F1000F02D081
:1074000009A8FCF771FC94F82330052B7FF40BAA34
:10741000FFF7EBBBD8F80400964AD0F800E00092E2
:107420004FF0040CCDE9019C0A46DEF800A00146AD
:107430000AA8D047CEE7D4F8083313F4004A20D185
:107440005FFA85FB0C2259462046FEF745FD0646AD
:10745000F0B1CDE909AA0A9B002201210BA8CDE9D0
:107460000A2302F077FF01462046FEF725FD0BA810
:10747000FCF73AFC0AA8FCF737FC16B109A8FCF7A0
:1074800033FC94F82330052B7FF4E3A9FFF7ADBB61
:10749000D8F8041004220B68CDE90102754A009265
:1074A000D3F800A05A460C230AA8D047D3E7D4F853
:1074B000083313F4004A20D15FFA85FB0C225946A9
:1074C0002046FEF709FD0646F0B1CDE909AA0022E3
:1074D0000A9B11460BA8CDE90A2302F03BFF0146A7
:1074E0002046FEF7E9FC0BA8FCF7FEFB0AA8FCF718
:1074F000FBFB16B109A8FCF7F7FB94F82330052B2A
:107500007FF4B8A9FFF771BBD8F8041004220B6808
:10751000CDE90102574A0092D3F800A05A460C2345
:107520000AA8D047D3E7D4F8083313F4007A20D15F
:107530005FFA85FB302259462046FEF7CDFC064611
:10754000F0B1CDE909AA0A9B002201210BA8CDE9DF
:107550000A2303F087FC01462046FEF7ADFC0BA88A
:10756000FCF7C2FB0AA8FCF7BFFB16B109A8FCF7A1
:10757000BBFB94F82330052B7FF48DA9FFF735BBB7
:10758000D8F8041004220B68CDE90102394A0092B0
:10759000D3F800A05A4630230AA8D047D3E7D4F83E
:1075A000083313F4007A20D15FFA85FB3022594664
:1075B0002046FEF791FC0646F0B1CDE909AA00226B
:1075C0000A9B11460BA8CDE90A2303F04BFC0146A8
:1075D0002046FEF771FC0BA8FCF786FB0AA8FCF717
:1075E00083FB16B109A8FCF77FFB94F82330052B29
:1075F0007FF462A9FFF7F9BAD8F8041004220B68E7
:10760000CDE901021B4A0092D3F800A05A4630236C
:107610000AA8D047D3E7D8F8041004200A68CDE9B7
:10762000016014480090D2F800A009A84A46D0474B
:10763000FFF774B9D8F8041004200A68CDE9016096
:107640000C480090D2F800A009A84A46D047FFF79E
:10765000ADB9D8F8041004220B68CDE90102054A3F
:107660000092D3F800B04A462B460AA8D847FFF745
:10767000E1B900BF801A0600D8F8041004220B6894
:10768000CDE901020C4A0092D3F800B04A462B46DD
:1076900009A8D847FFF70FBAD8F8041004220B68DE
:1076A000CDE90102044A0092D3F800B04A462B46C5
:1076B00009A8D847FFF743BA801A060073B50446F5
:1076C000FEF7CCFF94F82330052B32D0002594F838
:1076D0003F33EB40DA07E9B216D40135082DF6D175
:1076E00094F82330052B24D094F8203013B194F86B
:1076F0002230F3B9104B11491B68986903681B6865
:1077000002B0BDE870401847D4F808339B030CD48E
:107710002C200191FEF714FA064610B1019903F0EE
:1077200019FC31462046FEF7C7FB94F82330052BA1
:10773000D3D102B070BD00BFCC2500203CE60808C4
:107740002DE9F04F90F9213089B00446002B00F06C
:107750000481012300F50C7580F84133024600F5E1
:107760000F712B462E46D06E002859D0002384F886
:10777000413394F94030642B5BD094F9BC30642BD6
:1077800000F08D8094F93831642B00F08A80D4F8B1
:1077900030722FBB01A9204629F0B2FE00B30C23A2
:1077A0000593012306978DF81830714B07936946AE
:1077B000BDF80430049704A8ADF810308DF80070BF
:1077C0002AF070F89DF9001051B1022908DC38B197
:1077D000C9B27C2303FB01416C3128462BF06EFAC1
:1077E00094F841B3BBF1000F5DD0E36E6367D4F84A
:1077F000E830C4F8F030D4F86431C4F86C3194F84F
:10780000233003F1C30204EB82020021042B7CD855
:1078100052F8040B1061013342F8041CDBB2F5E7A7
:1078200053F8040B0028A1D18B4202F17C029AD1BB
:107830009FE7002066238DF810307C2303FB004077
:1078400004A940302BF07EF904A9204629F058FE07
:1078500000289CD004238DF818300023CDE9013393
:10786000039331230593694604A82AF01BF8059B6E
:1078700028B108AA02EB8302009942F8E01C013308
:10788000332B0593EFD94AF005FC9DED031ADDED8E
:10789000020A9DED010A66214AF0BAFB77E7012052
:1078A000C8E70220C6E70127A94655F8043B23B1E3
:1078B000AB600137042FF7D197E7AA46B8465FFAC5
:1078C00088F3022BF5D8DAF8002055F8043C9A42E8
:1078D00005D104A95046CDF810B02BF0EFF95AF8B5
:1078E000043B08F101020BB99046E8E704A906EB56
:1078F00088000193CDF810B02BF0E0F9019BAB604C
:1079000001A948462BF0DAF9D3E794F8413313B9CB
:107910002046FEF7DDF994F822300BB3154B1B68B7
:10792000986A036864215B6898472046FEF7A0FDCB
:1079300094F83E3003B9E36694F8BA300BB9C4F852
:10794000E83094F836310BB9C4F86431F9F7F4FD36
:10795000F9F77CFE0123A4F8403309B0BDE8F08FAD
:107960002046FFF7ABFE94F82230002BE0D0D5E79D
:10797000887B0908CC250020704700000120704753
:1079800001207047436898687047000010B5054BA8
:1079900003600446806A10B103685B68984720461C
:1079A00010BD00BF00EB0808406803685B6A184719
:1079B00033B46C46406884E80C0003689D6A94E820
:1079C0000C00AC4602B030BC6047000010B5044665
:1079D000FFF7DCFF2046FEF7BBF8204610BD000095
:1079E00040680AF0A5BC0000406801230AF0A0BC72
:1079F00040680AF079BC000040680A220AF01EBC08
:107A000040680AF033BC000040680AF0B5BC0000D2
:107A100090F82E2022B190F82D10002201F06EB9BE
:107A20007047000073B5044605250026A06A8DF84E
:107A3000076003680DF10702DB680121984778B100
:107A40009DF807300C2B09D0102B05D0092B07D13E
:107A500084F8303002B070BD1523F9E71423F7E73E
:107A6000013DE3D12846F5E710B4806A03681C693C
:107A70000822A44601235DF8044B31216047000031
:107A800010B4806A03681C690122A44600235DF8D3
:107A9000044B322160470000F0B50446806A036859
:107AA00085B05B6998470546002800F08480A06A8D
:107AB00003685B69984703689B689847A06A0368F6
:107AC0009B69984760B93D4B3D491B6898690368BD
:107AD0001B6898472B682846DB689847002667E0B4
:107AE0002046FFF7CDFF0028F4D02046FFF79AFF8D
:107AF0000028EFD0A06A03680121DB6A984720467E
:107B0000FFF7B2FF30B92D4B2E491B689869036807
:107B10001B68DEE7A06A0368DB69984730B9274B2A
:107B200029491B68986903681B68D2E7A06A94F822
:107B30003010012784F82E7003685B6A9847A06AAA
:107B400003689B6A984704F12D020146204601F024
:107B500023F906460028BDD0A06A94F82D100368CA
:107B600001919B6A984701990246204601F018F955
:107B700094F82C302BB194F82D103A46204601F0A1
:107B800023F994F82F2094F82D10204601F03EF9A7
:107B90002B682846DB689847A06A029403681D6A30
:107BA0000A4B039304AB13E90C0042F21071A8478F
:107BB000304605B0F0BD0646FAE700BFCC250020F0
:107BC0006CEA080892EA0808B1EA0808C57C0108CE
:107BD00070B5002586B0CDE9005500230446806AC3
:107BE0008DF8085005930393049303686A469E68D2
:107BF00010210923B047A0B19DF8003013F0010611
:107C000015D194F831300133DBB2052B84F83130D3
:107C100007D12046FFF734FF2046FFF725FF84F801
:107C20003160A06A03681B6B984706B070BD9DF871
:107C3000083084F831501B07F3D4BDF901309FEDB3
:107C40001F6A06EE903ABDF9033007EE103ABDF90F
:107C50000530F8EEE66A07EE903ACDED036AF0EEF5
:107C6000E66AB8EEC77AF8EEE77AF4EEC66AF1EEA5
:107C700010FA8DED047ACDED057A0DD5B0EEC77A08
:107C8000B4EEC67AF1EE10FA06D5F0EEE77AF4EE2D
:107C9000C67AF1EE10FAC4D49FED090A03A810F0D9
:107CA000B7F9B2EE040A03A810F0B2F994F82D2047
:107CB0000A2303A9204601F00FF9B2E700000034BF
:107CC0009A99193EFFF784BF10B5044B044640F85B
:107CD000043BFCF709F8204610BD00BF18EB08086C
:107CE00010B50446FFF7F0FF2046FDF731FF2046B0
:107CF00010BD0000F7B503680F4616461BB90024F7
:107D0000204603B0F0BD0024046008200193FDF775
:107D100017FF054620B1124B0360019B436001949D
:107D200001A8FBF7E1FF002DE9D03420FDF708FFA3
:107D300004460028E3D000F0E1FE0A4BA562236070
:107D400084F82C7084F82F602046FFF7A5FE0546C6
:107D50000028D5D1236820465B6898472C46CFE79A
:107D600018EB080800EB08082DE9F74F04680646F1
:107D70000D4690469946002C6CD00B68002B49D0DC
:107D8000236820465B6A984703689B6898470123ED
:107D900028680DEB030200210AF0CAFA98B39DF897
:107DA0000130EA2B2FD1DFF8F0B04FF0060A286837
:107DB0000023802206210AF097FA20B3DBF8007036
:107DC000B86A03680A215B689847002328681A4646
:107DD00006210AF089FAB0B1B86A03680A215B6823
:107DE0009847012328680DEB030206210AF0A0FA48
:107DF00048B19DF8014014F040042FD00AF1FF3A39
:107E00001AF0FF0AD3D1306803685B6A98470368A9
:107E1000DB68984700241DE0022223460F212868D2
:107E20000AF062FAB86A036801215B689847306813
:107E300003685B6A98470368DB6898473368346077
:107E40004A46414601A80193FFF754FF044601A8A2
:107E5000FBF74AFF204603B0BDE8F08F22462346D9
:107E60000F2128680AF040FAB86A036801215B68AC
:107E700098470223214630680DEB03020AF058FAB6
:107E800004460028C8D0B869024903681B689847AF
:107E9000B9E700BFD8EA0808CC25002090F82C10DC
:107EA000002200F02BBF000070B504468CB0042601
:107EB000013E76B2731C4AD0A06A15236A465D2142
:107EC0000AF036FA0028F3D0A06A152306AA5D212D
:107ED0000AF02EFA05460028EAD0152206A96846BF
:107EE0006DF02CFC0028E3D19DF8003084F82E3092
:107EF0009DF8073084F830309DF8143084F83A301B
:107F00009DF813309DF8102084F83B309DF80F3019
:107F100043EA0223A3879DF8013084F82F309DF8AF
:107F2000083084F83130039B9DF80C20C3F30F23F5
:107F300063869DF80B3043EA0223A386049BC3F3B8
:107F40000F23E386019BC3F30F23238707E0054B31
:107F500005491B68986903681B68984700252846EF
:107F60000CB070BDCC2500204CEB08082DE9FF417A
:107F700004460023806A8DF807300368DFF86881C3
:107F80005B6A984703689B689847A06A03680A2160
:107F90009B6C9847A06A0A2204210AF04FF9042535
:107FA000013D6DB26B1C32D000234B21A06A8222AE
:107FB0000AF09AF9D8F800600746B06A036802210F
:107FC0005B689847002FEBD001231A464B21A06A2B
:107FD0000AF08AF90746B06A036802215B6898478D
:107FE000002FDDD0A06A01230DF1070240210AF025
:107FF0009FF90028D4D09DF80720322A10D0002DF8
:10800000CED1B069364903681D683223A847A06AFB
:1080100003685B6A98470368DB68984700255BE064
:108020002046FFF741FF0028F1D0A06A0123172264
:1080300051210AF059F90028E9D05222A06A0123FF
:1080400011460AF051F90028E1D0A06A0123382234
:108050004C210AF049F90028D9D0A06A03685B6A6C
:1080600098470368DB689847A06A05210AF0FEF884
:10807000A36A04F12C029968204600F08DFE0546A3
:1080800050B3A36A94F82C109A68204600F088FE3A
:1080900094F8442094F82C10204600F0B7FE94F891
:1080A00045302BB194F82C100122204600F08CFEB4
:1080B000A06A036802219B6C9847A06A0294036837
:1080C0009E6A084B039304AB13E90C0044F21B11A6
:1080D000B0474CF0EBF82064284604B0BDE8F081CE
:1080E00074EB080855820108CC25002070B5858FF7
:1080F00090F93B60AD03B5FBF2F2A2F5804404FBBE
:1081000004F2D51190F83A200498D201624306FB9C
:1081100005225212A03002F58012424312134A4344
:10812000DB0003EB623000B270BD000010B5448E7E
:1081300053005C43B0F93830C91A838FD31AB0F9B1
:108140003620B0F93400534304F500449B10C3EBD0
:10815000C13300EB2440044993FBF0F04FF400429C
:108160000DF02CFF00B210BD0080FFFF10B52DED0B
:10817000028B8AB004460823806A05AA42210AF0CD
:10818000D7F818B1BDF81A20D30719D4A06A0AF09D
:10819000F3F84CF08BF8236CC31AFA2B0CD920643B
:1081A000002382224B21A06A0AF09EF80123A06AD4
:1081B0001A464B210AF098F80AB0BDEC028B10BDAC
:1081C000BDF9141094F930300093920894F92E30D0
:1081D0000392C9102046FFF789FFBDF9161094F9E4
:1081E0003130039A009308EE900A94F92F30C910A9
:1081F0002046FFF77BFFBDF91810039A491008EEDF
:10820000100A2046FFF792FF07EE900AF8EEE88A80
:10821000F8EEE77AB8EEC88AB3EE000A07A8CDED0B
:10822000097ACDED078A8DED088A0FF005FFB2EED1
:10823000040A07A80FF0ECFE4CF038F894F82C2054
:1082400020640A23204607A900F046FEA06A0AF02F
:1082500093F8B1E7FFF78ABFF7B503680D461646F6
:108260001BB90024204603B0F0BD0027076048205A
:10827000CDE90073FDF764FC044650B100F03EFC0C
:108280000E4B2360019BA362019784F8446084F83D
:10829000455001A8FBF732FD6846FBF72FFD002C87
:1082A000DFD02046FFF762FE05460028DAD12368BA
:1082B00020465B6898472C46D4E700BFACEB080823
:1082C00010B5044B044640F8283BFBF717FD204649
:1082D00010BD00BFACEB080810B50446FFF7F0FF77
:1082E0002046FDF735FC204610BD000090F82C100C
:1082F000002200F003BD0000F8B504460D46174605
:108300001E4600F0FBFB094B23602B68A362002292
:1083100000232A6084F82D7084F82E60236563653D
:10832000A365E365236663662046F8BDC4EB0808D1
:10833000F8B51C4609331646DB086A46A2EBC303B0
:1083400000AF9D46806AA31C6A4609F0F1FF05460E
:1083500028B122460DF1020130466DF0FFF92846A2
:10836000BD46F8BD2DE9F34106460F4614464BF0D5
:108370009DFF114BD3F800800546D8F8280003680C
:1083800001215B68984701230DF107020721304660
:10839000FFF7CEFF60B19DF80730DA0702D4B7EBE4
:1083A000531F05D04BF082FF431BA342E5D30020AF
:1083B00002B0BDE8F08100BFCC2500202DE9F041DE
:1083C000DFF8608292B0044602AF002646F0200239
:1083D000A06A0023D2B2502109F086FF002800F0E5
:1083E0000C810325013D6DB26A1C00F00681D8F8AE
:1083F0000030986A03684FF496719B689847012390
:108400000DF1060255212046FFF792FF002800F0EB
:10841000F4809DF8063013F0E00F40F0EE80DB07AB
:10842000E0D502230DF1060252212046FFF780FF1E
:10843000002800F0E280BDF8063001365BBA202E3D
:1084400027F8023BC2D1BDF824309DF826109FEDDD
:108450006D7ADFED6D6A9FED6D6A43F30B0207EEF7
:10846000902A1B0903F47063BDF82620F8EEE77A22
:108470000B4343F30B03C4ED0C7A07EE903A02F47E
:1084800070639DF82820F8EEE77A134343F30B035B
:10849000C4ED0D7A07EE903A9DF92230F8EEE77AB6
:1084A000C4ED0E7A07EE903A9DF92930F8EEE77A9E
:1084B00067EE877A07EE103AB8EEC77A9DF92A3050
:1084C000C4ED0F7A27EE267ADFED517A84ED107A2B
:1084D00007EE103AB8EEC77A9DF92B30E7EE267A10
:1084E000C4ED117A07EE903AF8EEE77A9DF9233061
:1084F00067EEA67ADFED476AC4ED127A07EE903A8E
:108500009DF92C3007EE103AB8EEC77A9DF92E305F
:1085100027EE267AF8EEE77A84ED147A67EE867A0B
:1085200007EE103A9DF93030C4ED137A07EE903A19
:10853000F8EEE77A9DF92D3067EEA67AB8EEC77AA5
:10854000C4ED167A27EE267A07EE903A84ED157A76
:10855000F8EEE77A9FED307A9DF92F3067EE877A53
:10856000C4ED177A07EE903A9DF93130F8EEE77ACC
:1085700006EE903A67EE877AF8EEE66AC4ED187A6E
:10858000DFED267ABDF93830E6EE877A07EE103A4D
:108590009DF93230C4ED197AB8EEC77AF3EE077A56
:1085A000E7EE067A07EE103ADFED1D6AC4ED1A7A9F
:1085B000B8EEC77A27EE267A84ED1B7A9DF9333020
:1085C00007EE103AB8EEC77A9DF9343027EE267AD6
:1085D00084ED1C7A07EE103A9DF9353007EE903A9B
:1085E000B8EEC77AF8EEE77A27EE267A67EEA67A33
:1085F00084ED1D7AC4ED1E7A00E0002012B0BDE8C3
:10860000F08100BFCDCC4C3E0000803B0000003B21
:108610000AD7233C0000003D0000803817B7D1B8CE
:108620000AD7A33ACC25002073B501230E460DF1DD
:10863000070206210446FFF77BFE18B900252846ED
:1086400002B070BD9DF80730013B012B0CD8002310
:10865000A06A1A46062109F047FE0028EED006223D
:1086600000212046FFF77EFEA06A00233246062145
:1086700009F03AFE05460028E0D026223146204681
:10868000FFF770FEDBE7000013B501230DF10702D1
:1086900007210446FFF74CFE10B9002002B010BDC0
:1086A0009DF807301B070CD50023A06A1A46062147
:1086B00009F01AFE0028F0D0062200212046FFF71C
:1086C00051FEA06A00230722062109F00DFE0028B2
:1086D000E3D0132207212046FFF744FE0028DCD018
:1086E000A06A00230522062109F0FEFD0028D4D04F
:1086F000172205212046FFF735FE0028CDD00121A5
:108700002046FFF791FFC9E7F7B50446806A5B4F43
:1087100003685B6A984703689B689847A06A036888
:108720000A219B6C9847A06A0A22042109F086FD61
:108730000525013D6DB26B1C00F09680A06A0023F8
:10874000B6227E2109F0D0FD0028F2D03B68986A5D
:10875000036818215B686E46984701233246002162
:108760002046FFF7E5FD0028E3D09DF80030332BCD
:10877000DFD12046FFF722FE002875D0A06A002333
:108780008022502109F0B0FD00286DD02046FFF76F
:108790007BFF002868D0A06A002386222E2109F0E2
:1087A000A3FD002860D0A06A00232422042109F040
:1087B0009BFD002858D0A06A00230222062109F060
:1087C00093FD002850D0142202212046FFF7CAFD55
:1087D000A06A00230722052109F086FD002843D066
:1087E00001212046FFF720FF00283DD0A06A036842
:1087F00003219B6C9847A06A03685B6A98470368EB
:10880000DB689847A06A172109F030FDA36A04F1DC
:108810002C029968204600F0BFFA054608B3A36A07
:1088200094F82C109A68204600F0BAFA94F82E209A
:1088300094F82C10204600F0E9FA94F82D302BB172
:1088400094F82C100122204600F0BEFAA06A0368BA
:108850009F6A0B4B0094019396E80C0042F2107152
:10886000B847284603B0F0BDA06A03685B6A984722
:108870000368DB6898470025F3E700BFCC2500209C
:10888000798A010810B586B00C236A463121044666
:10889000FFF74EFD002800F0DF809DF801309DF8C5
:1088A0000020DFED717ADFED715A1B0403EB022328
:1088B0009DF8022003EB02631B1206EE903A9DF82E
:1088C00004309DF803201B0403EB02239DF80520D0
:1088D00003EB02631B1207EE103A9DF807309DF878
:1088E00006201B0403EB02239DF8082003EB026320
:1088F0001B1206EE103A9DF80A309DF809201B0461
:1089000003EB0223F8EEE66AB8EEC77A9DF80B2077
:1089100066EEA76A27EE277AB8EEC66ADFED547ACC
:1089200003EB02631B1226EE276A07EE903AF8EE7D
:10893000E77A67EEA57AF5EEC07AF1EE10FA40F329
:108940008D80DFED4C5A77EEE57AD4ED134A94ED45
:108950000F5A94ED1C4AD4ED1D3A94F82C20F7EEF2
:10896000005A74EEA54AF0EE632AA4EEA75A0A2331
:1089700003A9D4ED107AD4ED0C4A77EEA57A2046FF
:10898000E7EEA64AD4ED1A7A75EE677A94ED145A9A
:10899000F0EE646AD4ED174AE5EE276AB0EE655A48
:1089A000A7EEA45AC6EE854A94ED115AD4ED0D6A8D
:1089B00035EE255AE5EE076A94ED157AE7EE876AFB
:1089C00094ED187AB0EE655AA7EE875A86EE857A4E
:1089D00094ED125AD4ED0E6A35EE255AE5EE066A8C
:1089E00094ED166A94ED195AE7EE866AB0EE656A60
:1089F000A7EE856AF0EE657A86EE863A94ED1B6AFC
:108A0000F0EE646AE6EE447AE6EE476A86EEA75A2E
:108A1000F0EE476AE4EE646AC6EEA75AD4ED1E6A29
:108A2000D4EE262AE6EE636AB2EE046A27EE667A90
:108A300065EE066AA2EEA47ACDED036A65EE866A5B
:108A4000CDED046AC7EE276A76EE837A67EE867A02
:108A5000CDED057A00F040FA06B010BD44BFDFED61
:108A6000055A77EEA57A70E747ABE73B5B9E803A05
:108A7000F61BEB3B85EBCB41FFF704BF30B513464C
:108A8000026885B00D461AB90024204605B030BDF5
:108A9000002101607C2001930392FDF751F8044608
:108AA00020B1019B2A4603A9FFF726FC03A8FBF788
:108AB00025F9002CE8D02046FFF726FE05460028C1
:108AC000E3D1236820465B6898472C46DDE7000029
:108AD00010B5044B044640F8283BFBF70FF920463D
:108AE00010BD00BFC4EB080810B50446FFF7F0FF47
:108AF0002046FDF72DF8204610BD0000064B10B5AE
:108B000003600446FDF7A4FD606004F108004AF02C
:108B100077FD204610BD00BFDCEB080873B50646A4
:108B2000144675687C2303FB0253C4EB441405EB25
:108B30008404084693F8A41001900FF0FFFA94F90A
:108B40003C3001983BB9736893F8251002B0BDE83A
:108B500070400FF0F3BA94F84010F7E737B5446867
:108B600001917C2505FB024595F83F3004EB830419
:108B7000D4F84C325BB14BF099FBC5F89C000199DD
:108B8000D4F84C0203B0BDE8304003F079BE03B026
:108B900030BD00002DE9F04FC2EB421447684FEAA8
:108BA000840881460E4607F13C0B08F108018BB0A2
:108BB0001546594430460FF0F7F9D9F80400294614
:108BC0000BEB8404FDF7EAFC38B17C2303FB05734F
:108BD00093ED1A0A30460FF01BFA7C2303FB057352
:108BE00093ED146ADFED3A7AD3ED156AB0EEC67AEA
:108BF000B4EEE77AF1EE10FA0FD5B0EEE67AB4EE05
:108C0000E77AF1EE10FA08D594ED077AB0EEC77A5C
:108C1000B4EEE77AF1EE10FA1BD47C2303FB057364
:108C2000D86D196E5A6E9B6D029003910490079156
:108C300001A831468DED016ACDED056A06920892D4
:108C400009930DF063FB86ED000AC6ED010A86ED7F
:108C5000021A7C2303FB05770023C7F88C30C7F882
:108C60008830C7F88430D9F8040090F95C3208F1F4
:108C70003C0A08F14808DA44D84463B15DB941467A
:108C800000F5167004F0B4FA414630460BB0BDE86A
:108C9000F04F0FF089B990F93430012B0BD190EDE2
:108CA0000E0A50460FF060F984ED120AC4ED130A63
:108CB00084ED141AE8E7022BE6D1FBF757FD0022FA
:108CC00001A9FBF753FA0028DED09DED010AE8E781
:108CD0000000003410B543687C2404FB023407C94B
:108CE00004F1900383E807004BF0E0FAC4F89C001D
:108CF0004BF0D0FAC4F8A00010BD0000F0B5074654
:108D000085B00D46164600F10801A92203A809F016
:108D100069FD7C687C2303FB0543D3F8B42022B9AA
:108D200003A809F081FD05B0F0BDBEB196ED007A53
:108D3000D3ED2A7A67EE877AC3ED2A7A96ED017A27
:108D4000D3ED2B7A67EE877AC3ED2B7A96ED027A14
:108D5000D3ED2C7A67EE877AC3ED2C7A7C2607EE6A
:108D6000902A06FB0541A831B8EE670A0846019132
:108D70000FF062F901992A463846FFF7ABFF06FB70
:108D800005410023C1F8B030C1F8AC30C1F8A830BB
:108D90000023C1F8B430C3E74068FCF7E9BF000026
:108DA000F7B50646406801927C2707FB01000D4697
:108DB0006C3001A9144629F061FF716807FB0515A5
:108DC0002C6703B0F0BD000007B540687C2303FBAF
:108DD000010393F93C30022B0BD000F13C03C1EBB3
:108DE000411003EB80000DF107018DF8072029F0F9
:108DF0009FFE03B05DF804FB43687C2202FB013157
:108E000091F93C00003818BF0120704743687C206E
:108E100000FB013181F8A42070470000F8B5054639
:108E200008460F460FF066F910B100242046F8BD41
:108E300038460FF045F904460028F6D16B6893F9DF
:108E400034637EB138460FF08DFC95ED087ADFED86
:108E50001F7AF0EEC76AF4EEE76AF1EE10FA03D576
:108E600085ED080A0124E1E777EE407A30EE076AE3
:108E7000F0EEE77AC7EE866AF6B207EE906A9FEDEB
:108E8000146AF8EE677A26EE866AF4EEC67AF1EE98
:108E900010FA48BFB2EE046ADFED0E7A45BF6B6A86
:108EA00066EE866AB0EE676A87EEA66A46BF013351
:108EB0006B620124F7EE007A77EEC67A20EE060A9E
:108EC000A7EE270A85ED080AB0E700BF00000034CE
:108ED00000004843CDCCCC3D2DE9F74304460E4677
:108EE00015461F46FFF71AFE2A4631462046FFF771
:108EF00035FE314620462A46FFF74CFE31462046D5
:108F0000FFF78CFF28B39B2204F1080101A809F0A8
:108F100069FC64684FF07C0909FB054808F1A80862
:108F2000314640460FF040F809FB0542D2F8B41034
:108F30000131C2F8B4104FB1B94207D34908C2F8A1
:108F4000B410B0EE000A40460FF076F801A809F020
:108F50006BFC03B0BDE8F08310B50446FCF792FF4C
:108F6000C0B23C34C0EB401004EB800010BD0000E8
:108F7000F8B50A4E044600F5167704F5137555F852
:108F8000040B08B103F0B0FFBD42F8D13368986A12
:108F9000036801215B689847EFE700BFCC250020FC
:108FA00008B5FFF7E5FF0000F0B5144E00EB8107B0
:108FB00073780446D7F84C026FF3410387B00D462F
:108FC0007370C8B102F07EFB68B1737843F0100390
:108FD00073702C440023A372D7F84C0207B0BDE88D
:108FE000F04002F0F3BAD7F84C12684602F09AFB50
:108FF000009B012BEDD1E8E707B0F0BD945A0020AB
:1090000070B506460D46002445FA04F3DB07E1B2CD
:1090100002D53046FFF7C8FF0134032CF4D170BDF0
:10902000FF21FFF7EDBF000030B500F5137587B0E5
:1090300000F5167455F8041B21B9A542FAD1002099
:1090400007B030BD684602F06DFB009B013B022B70
:10905000F3D80120F4E700002DE9F0472DED028B55
:1090600088B004460D469046B0EE408AFDF7DEF922
:1090700030B90026304608B0BDEC028BBDE8F08761
:1090800029462046FDF74CF806460028F1D004EBAF
:109090008507D7F83C22D7F830329A4206D035F00F
:1090A000D9FC5C4A03212EF005FFE2E7D7F84C32E9
:1090B00083B94FF49870FCF743FD814608B103F083
:1090C00017F8C7F84C92B9F1000F03D135F0C2FC84
:1090D000514AE7E7B4F84A32D90711D505F078FECE
:1090E00090F8082390F8C43232B9B02202FB030092
:1090F00090F8A130012B03D835F0ACFC474AD1E7FA
:109100002046FFF791FF20B9454A537843F0020308
:10911000537094F9353053B329462046FFF71CFFAE
:1091200090F90030002B53D029462046FFF714FF5A
:1091300090F80490B9F12B0F19D829462046D7F89A
:109140004CA2FFF709FF94F9353090F90020022B6B
:10915000D4BF00210121012BD4BF00230123003AF9
:10916000009118BF01224946504602F043FA6319A4
:1091700000229A7275B3D4EDC10AB4F84822D7F828
:109180004C0270EEA00A2B46B0EE480A414602F0AF
:1091900051FA94F83E33002B31D1224A06941268DA
:1091A0000127E773906A0268156D1F4A07920293C0
:1091B00009224FF40063CDE9003208AA12E9060043
:1091C0001A4BA847C8B935F045FC194A02216AE78D
:1091D0009946B2E729462046FFF7BEFE90F90030D7
:1091E000002BC8D0D4EDC10AB4F84822D4F84C0200
:1091F0002B46B0EE480A4146C9E784F83E73002387
:109200000DF1170104F124008DF8173029F09AFCB4
:1092100030E700BFECEB08081EEC080841EC08083A
:10922000945A0020CC250020A18F01085FEC08088B
:109230006AEC08082DE9F0412DED028B0024437300
:109240009DF82030837305460F469046B0EE408A65
:10925000264647FA04F3DB07E1B210D5B0EE480A20
:1092600042462846FFF7F8FE064640B939462846EA
:10927000FFF7C6FEBDEC028B3046BDE8F08101343D
:10928000032CE6D1F6E70000F8B500242DED028BA3
:1092900005460F46B0EE408A427383732646E1B21C
:1092A000B0EE480A3A462846FFF7D6FE01340028B9
:1092B00018BF0646032CF2D1BDEC028B3046F8BD38
:1092C000F0B500EB81030D46D3F84C129BB0044679
:1092D00011B900201BB0F0BD0BA802F007FA63190A
:1092E000987A0028F6D10B9A002A48D0042AF0D1A7
:1092F00001229A720DAA07CA02AB83E8070010AADE
:1093000007CA05AF87E8070013AA07CA9DED180A28
:1093100008AE86E807001A46294620468DED010A68
:10932000FCF792FE3A4629462046FCF739FE3246C3
:1093300029462046FCF746FE9DED010A29462046B7
:10934000FCF752FE9DF8643083B129462046FFF7B2
:1093500003FE90F900304BB194F93530012B05DD57
:109360009DF85D2029462046FCF786FE2046FFF743
:109370005BFE20B9034A537843F004035370012085
:10938000A8E700BF945A00202DE9F0410546884621
:1093900000F513770024012657F8043BE1B26BB1C6
:1093A00048FA04F3DB0709D52846FFF789FF0028B0
:1093B00057F8040C08BF002602F008F90134032C0A
:1093C000EAD13046BDE8F0812E4B2DE9F04F1F6801
:1093D000FB6A93F89C8087B00446B8F1000F38D13F
:1093E000DFF8A8A000F5137600F1030B054656F848
:1093F000040BA5EB04095FFA89F9E8B102F04EF914
:1094000028B19AF8013043F008038AF8013056F881
:10941000040C02F057F9F8B9637B6BB1AB7A5BB916
:1094200056F8041C684602F07DF9009B042B03D11A
:1094300049462046FFF744FF01355D45D7D1124B21
:10944000204683F81280FFF7EFFD054630B1012377
:10945000237407B0BDE8F08F8046EDE7237C002B36
:10946000F7D0A37B002BF4D0B86A03684FF47A716D
:109470005B689847B86A03689B6B294607B0BDE8EC
:10948000F04F1847CC250020755A0020945A002030
:10949000F0B5002587B000F513762C46012756F865
:1094A000041B41B1684602F03DF9009B1BB107FA6D
:1094B00005F31C43E4B20135032DF0D1204607B07B
:1094C000F0BD00002DE9F04F2DED028B03270E7C3F
:1094D0009FED348A91B005468846B946AC5D0134AB
:1094E000E4B2B4FBF9F303EB4303E41AE4B205EB93
:1094F0008403D3F84C1209B9AC554CE003A802F030
:1095000011F9DDF80CB00BF1FF33022BF4D8304623
:109510002FF05EFC8246304630F05EFB00F11B030C
:109520009A4508D230462EF0CFFE002011B0BDEC97
:10953000028BBDE8F08FAC55284698F810A0FFF7D5
:10954000A7FFDDED057A8DF83100FCEEE77A9DF896
:1095500010208DF8332017EE903A8DF8343006AB9A
:1095600003CB1B88ADF83D305C221B23CDE90032D4
:10957000CDF83500CDF8391009AABF2150468DED40
:10958000098A8DED0A8A8DED0B8A8DF830408DF8B1
:1095900032B02FF087FC013F17F0FF079ED101206A
:1095A000C4E700BF000000002DE9F04F0F7CA1B020
:1095B00006468846032500EB070999F80540013463
:1095C000E4B20323B4FBF3F303EB4303E41AE4B282
:1095D00006EB8403D3F84C1211B989F805400AE070
:1095E00011A802F083F8DDF844A0BAF1030F08DCFB
:1095F000BAF1000FF1DA013D15F0FF05DDD10120D0
:1096000012E0AAF10402032AF5D838462FF0E0FB55
:109610008346384630F0E0FA00F13602934506D230
:1096200038462EF051FE002021B0BDE8F08F89F8B9
:109630000540304698F810B0FFF72AFFDDF848E003
:10964000CDF80CE0DDF84CE0CDF810E0DDF850E0AE
:10965000CDF814E0DDF854E0CDF818E0DDF858E07E
:10966000CDF81CE0DDF85CE0CDF820E0DDF860E04E
:10967000CDF824E03219DDF864E01C9BCDF828E039
:10968000DDF868E092F80AC09DF874109DF8752026
:10969000CDF82CE00E93DDF86CE01E9B8DF83500C4
:1096A0008DF83C108DF83D20CDF830E08DF8344039
:1096B0008DF836A08DF837C02422CDF83E30362301
:1096C000CDE90032C0212C2303AA58462FF0EAFB33
:1096D00091E700007FB58A8B0B464AF2B9518A4266
:1096E00005465FD04AF2BA518A4274D04AF2B85164
:1096F0008A420BD1474A1268D26A92F89C203AB14A
:1097000035F0A8F9444A05212EF0D4FB042479E071
:10971000D3ED007AF5EEC07AF1EE10FAF6D49FEDB3
:109720003F7AF4EEC77AF1EE10FAEFDC93ED017AAE
:10973000DFED3B6A1C6993ED030AB0EEC77AB4EE25
:10974000E67A93ED027AFCEEE77AB0EEC77AF1EEB4
:1097500010FAB4EEE67A17EE903A54BF01260026CE
:10976000F1EE10FA54BF01220022003C18BF012480
:1097700013F0FF0110D18DED030A0292FCF7CCFB30
:109780009DED030A029A234631462846FFF77CFDE9
:109790000028BBD0002435E0134600943246FFF782
:1097A00049FDF5E7D3ED007AF5EEC07AF1EE10FA57
:1097B000ACD49FED1A7AF4EEC77AF1EE10FAA5DC7C
:1097C000FCEEE77A17EE903A13F0FF0108BFFF2195
:1097D000FFF7DAFDDCE7D3ED007AF5EEC07AF1EEC3
:1097E00010FA93D49FED0D7AF4EEC77AF1EE10FAE9
:1097F0008CDCFCEEE77A17EE904A14F0FF0404D1FB
:10980000FFF70EFC204604B070BD2146FFF7F8FBC1
:10981000C0E700BFCC2500209CEC080800007F4377
:1098200000000034F0B58BB00E4614460746FFF733
:1098300093FB543007C884E8070031463846FFF7E9
:109840008BFB90ED057ADFED267AB0EEC77AB4EEA9
:10985000E77AF1EE10FA054611D590ED067AB0EEF2
:10986000C77AB4EEE77AF1EE10FA08D590ED077AF0
:10987000B0EEC77AB4EEE77AF1EE10FA24D43146AE
:109880003846FFF769FB016A426A836AE869D5F8DE
:1098900014E0D5F818C0099001A8CDF804E00291B1
:1098A00003920491CDF814C00693079208930CF02C
:1098B000D9FE98B1214601A80CF028FD84ED000ADC
:1098C000C4ED010A84ED021A31463846FFF744FB25
:1098D00000F1080120460EF081FB01200BB0F0BD25
:1098E000000000342DE9F0472DED048BACB0B0EE54
:1098F000608A0546B0EE409A0F46F0EE418A9046E7
:10990000FCF70AFBDFED8B7AB0EEC87AB4EEE77AAB
:10991000F1EE10FA4BD5B0EEE87AB4EEE77AF1EE5C
:1099200010FA44D523AC2046FBF76EFEF7F704FE91
:109930002146F7F7E3FB064658BB05F049FA90F8D5
:10994000083390F8C42233B1B02303FB020393F829
:10995000A130012B07D84FF0B00909FB020090F8A5
:10996000A130022B0BD835F075F8734A03212EF085
:10997000A1FA30462CB0BDEC048BBDE8F08705F0B1
:1099800027FA90F8C43209FB0300AC300FC884E812
:109990000F00DDED257A9FED691AB8EEE78ADDED5F
:1099A000267AF8EEE78A28EE018A68EE818A04AA10
:1099B00003A902A8F0EE680AB0EE480A03F0D4FC4E
:1099C000064618B935F046F85D4ACFE79FED5D7A57
:1099D000DDED027A9FED5C8ADFED5C8A8DED068A13
:1099E00067EE877A2422002111A8CDED057A8DED4E
:1099F000078A6BF0FDFE9DED031ADDED040ADFF82A
:109A000058A121EE281A68EEE00AB0EE480A11A823
:109A10000CF048FE05A911A80CF078FC24220021C6
:109A20001AA8CDED060A8DED071A8DED050A6BF02B
:109A3000DFFEF7F781FD90ED810A8DED010AF7F762
:109A40007BFD29EE281AD0ED820A9DED010A1AA8A5
:109A50000CF028FE1AA923A80CF046FD05A923A89E
:109A60000CF054FC4FF000098DED050ACDED060A0F
:109A70008DED071A95F822305FFA89F4A3427FF63C
:109A800078AF1FB127FA04F3DB071AD52B1993F926
:109A90002C32B3B1B8F1000F0DD021462846FCF7A7
:109AA000C5FC88B934F0D6FF294A234603212EF09D
:109AB00001FA00265DE721462846FCF731FB002825
:109AC000EBD109F10109D5E708AA214628468DED19
:109AD000088A8DED098A8DED0A8AFFF7A3FE20B969
:109AE00034F0B8FF1B4A2346E0E708A905A80EF0AA
:109AF00025FA0BAA214628468DED0B0ACDED0C0A5E
:109B00008DED0D1AFCF7A0FA9AE807000EAB83E87A
:109B100007001A4621462846FCF742FA23AA2146A6
:109B200028468DED238A8DED248A8DED258AFCF75C
:109B300049FAC6E700000034C0EC080895BFD633E8
:109B4000DBEC080800007A440000000035FA8E3C87
:109B5000F0EC080804ED0808409908080120704757
:109B600001207047436898687047000040680368A8
:109B70009B6C184710B5054B03600446806A10B112
:109B800003685B689847204610BD00BFECED0808ED
:109B9000406803685B6A184733B46C46406884E8E1
:109BA0000C0003689D6A94E80C00AC4602B030BC1F
:109BB0006047000010B50446FFF7DCFF2046FBF7C6
:109BC000C7FF204610BD0000406808F04FBB0000F2
:109BD000406808F0ADBB00004068012308F0A8BB56
:109BE0004068002308F080BB90F84420D20705D5D8
:109BF00090F8421000F12C02FFF780B87047000087
:109C0000F8B504461E460F461546FEF777FF084B8B
:109C100023600023E3622363636394F84430A76204
:109C200065F3410384F8436084F844302046F8BD6E
:109C3000ECED080810B50D4B83630446806A036899
:109C400098221B690021984770B1A06A03682022FE
:109C50001B690121984738B1A06A0368BDE810402C
:109C60001B69012202211847002010BDC5DC6A3F94
:109C700037B50446806A03686A469D680321062357
:109C8000A847D0B1BDF80020BDF8041052BA95B273
:109C900049BAB5F5704F0BB211D013F5805F0ED0F5
:109CA000BDF802305BBA9DB2B5F5704F07D0524295
:109CB0005B42A287E187A4F8403003B030BD0020AA
:109CC000FBE70000806A036801221B690221184734
:109CD00030B585B00446FFF7CBFF05462046FFF7B9
:109CE000F1FF6DB3B4F93C3094ED0E0A06EE903AF4
:109CF000B4F93E3007EE103AB4F9403007EE903A2E
:109D0000F8EEE66AB8EEC77AF8EEE77A01A8CDED8C
:109D1000016A8DED027ACDED037A0EF079F994F8AF
:109D200042102046FFF768F818B1022101A80EF092
:109D300005FA94F842200E2301A92046FFF7CCF83B
:109D400005B030BDFFF7C4BF13B5806A036801AA30
:109D50009C680A210323A04738B10549032201A8C2
:109D60006BF0ECFCB0FA80F0400902B010BD00BF0F
:109D700024ED08082DE9F84300252DED028BDFF8CE
:109D800088819FED5D8A04462E462F46A06A0368AF
:109D900011221B6900210137984700287BD0D8F891
:109DA0000090D9F82800036832215B689847A06AC0
:109DB000036860221B690121984700286BD0A06AC4
:109DC000036801221B6902219847002863D0D9F853
:109DD0002800036832215B6898472046FFF748FF58
:109DE000002858D00135022FEDB256DDB4F93C30D1
:109DF0009FED425A9FED426A07EE903AF8EEE77AFD
:109E0000C5EE276AF0EEE66AF4EEC66AF1EE10FAE5
:109E100041DDF4EEC86AF1EE10FA3CD5B4F93E30FB
:109E2000DFED385A07EE903AF8EEE77A85EEA77A3A
:109E3000B0EEC77AB4EEC67AF1EE10FA2BDDB4EECE
:109E4000C87AF1EE10FA26D5B4F9403005EE903A12
:109E5000F8EEE55AC5EE257AF0EEE77AF4EEC67A2A
:109E6000F1EE10FA17DDF4EEC87AF1EE10FA12D521
:109E700094ED0B6A76EE266A0136C4ED0B6AD4EDDA
:109E80000C6A36EE877A84ED0C7A94ED0D7A77EED3
:109E9000277AC4ED0D7A192F02D0052E7FF476AF04
:109EA000A06A036810221B6900219847052E18D16B
:109EB000D4ED0B6AF1EE047A86EEA77A0120D4ED98
:109EC0000C6A84ED0B7A86EEA77AD4ED0D6A84EDE8
:109ED0000C7A86EEA77A84ED0D7ABDEC028BBDE894
:109EE000F8834FF07E53052DE3622363636394BFD1
:109EF00000200120F1E700BFCDCCAC3F00002E4494
:109F00003333333F00002244CC250020F0B5044613
:109F1000806A036885B05B699847054648B9504B2D
:109F200050491B68986903681B689847284605B024
:109F3000F0BD03689B689847A06A03680A21DB6A42
:109F40009847A06A03689B69984760B9444B4649A3
:109F50001B68986903681B6898472B682846DB686C
:109F600098470025E2E72046FFF7EEFE0028F4D0F0
:109F70002046FFF7FFFE30B9394B3C491B68986912
:109F800003681B68E8E72046FFF754FE0028E4D08A
:109F9000A06A0368DB69984730B9314B34491B68C4
:109FA000986903681B68D7E794F84430A06A43F0C7
:109FB000010384F8443003680321DB6A98472B6867
:109FC0002846DB689847236820469B689847A06A24
:109FD000036807215B6A9847A06A03689B6A9847F1
:109FE00004F1420201462046FEF7D6FE054600284F
:109FF0009CD0A06A94F84210036801919B6A98472C
:10A00000019902462046FEF7CBFE94F8432094F8CF
:10A0100042102046FEF7FAFE94F844309B0705D51F
:10A0200094F8421001222046FEF7CEFEA06A029468
:10A0300003681E6A0F4B039304AB13E90C0043F251
:10A040001541B047064BA06A1B689E6933681F68BC
:10A0500003689B6A9847084902463046B84765E757
:10A06000CC25002028ED08084EED080874ED0808FE
:10A0700099ED0808459D0108C7ED080810B5084B83
:10A08000036004460023086860600B60037A03F0F5
:10A090000703022B02D1C02108F016FA204610BD9A
:10A0A00004EE080810B5044B044640F8043BF9F7E9
:10A0B00025FE204610BD00BF04EE080810B504467A
:10A0C000FFF7F0FF2046FBF743FD204610BD0000E0
:10A0D000F7B503680E4617461BB90024204603B0A7
:10A0E000F0BD0022026008200193FBF729FD054620
:10A0F00010B101A9FFF7C2FF01A8F9F7FFFD002D7C
:10A10000EBD04820FBF71CFD04460028E5D029468B
:10A110003B463246FFF774FD2046FFF7F7FE054643
:10A120000028DBD1236820465B6898472C46D5E79A
:10A1300090F82D100022FEF7E1BD0000F0B50446B6
:10A14000806A036889B05B6A984703689B68984790
:10A15000A06A03680A219B6C9847A06A01230DF14D
:10A160001702002108F0E4F8002838D09DF81730D5
:10A17000082B34D14E4F052500230122A06A32213D
:10A1800008F0B2F83B689B6A1A68526840B90A2125
:10A1900018469047013D15F0FF05EDD145481CE0FC
:10A1A00018461421904706AEFF238DF81830A06A98
:10A1B00001233246322108F0BBF80028EAD09DF88E
:10A1C000183013F00103E5D1A06A0393082232216D
:10A1D00008F08AF8039B58B9374849F09FFAA06AFB
:10A1E00003685B6A98470368DB68984700255CE072
:10A1F000A06A03931A46342108F076F80028EBD0C1
:10A20000039BA06A2422412108F06EF80028E3D0C5
:10A21000039BA06A0822312108F066F80028DBD0F1
:10A22000A06A036803219B6C9847A06A03685B6A75
:10A2300098470368DB689847A06A102108F016F871
:10A24000A36A04F12D0299682046FEF7A5FD054694
:10A2500058B3A36A94F82D109A682046FEF7A0FD23
:10A26000A36A16481A7A597A00919B681449D20851
:10A2700049F054FA94F82C2094F82D102046FEF75B
:10A28000C5FD94F82E302BB194F82D1001222046F4
:10A29000FEF79AFDA06A03689F6A0A4B069407932B
:10A2A00096E80C0042F21071B847284609B0F0BD9C
:10A2B000CC25002094EE080834EE08086BEE080860
:10A2C00063EE080851A3010810B586B004460123C7
:10A2D000806A0DF10302102108F02AF898B39DF866
:10A2E0000330DB072FD5A06A062301AA112108F04D
:10A2F0001FF840B3BDF904309FED146A94F82D2087
:10A3000006EE903ABDF9063007EE103ABDF8083077
:10A310005B421BB207EE903AF8EEE66AB8EEC77AF7
:10A32000F8EEE77A66EE866A27EE067A67EE867AB8
:10A330000A2303A92046CDED036A8DED047ACDED05
:10A34000057AFEF7C9FD06B010BD00BF85EBC13F21
:10A35000FFF7BABFF7B503680D4616461BB90024D0
:10A36000204603B0F0BD002707603020CDE9007320
:10A37000FBF7E6FB044650B1FEF7C0FB0E4B236033
:10A38000019BA362019784F82C6084F82E5001A8E9
:10A39000F9F7B4FC6846F9F7B1FC002CDFD0204691
:10A3A000FFF7CCFE05460028DAD1236820465B681B
:10A3B00098472C46D4E700BFC0EE080810B5044B00
:10A3C000044640F8283BF9F799FC204610BD00BF31
:10A3D000C0EE080810B50446FFF7F0FF2046FBF773
:10A3E000B7FB204610BD000090F831100022FEF7A8
